:020000040800F2
:1000000000000220F1C0000841C1000829C2000818
:100010003DC2000861C2000885C20008000000005F
:10002000000000000000000000000000A9C200085D
:10003000ABC2000800000000ADC2000899C700086C
:100040003DC100083DC100083DC100083DC1000898
:100050003DC100083DC1000873D9000879D90008E6
:100060007FD9000885D900088BD900083DC1000858
:100070003DC100083DC100083DC100083DC1000868
:100080003DC100083DC100083DC100083DC1000858
:100090003DC100083DC100083DC1000891D90008DC
:1000A0003DC100083DC100083DC10008D9D9000884
:1000B000DFD90008E5D90008EBD900083DC10008E8
:1000C0003DC100083DC100083DC100083DC1000818
:1000D0003DC1000855D900085BD9000861D9000866
:1000E000B5D900083DC100083DC100083DC1000868
:1000F0003DC100083DC10008F7D900083DC1000816
:100100003DC100083DC10008F1D900083DC100080B
:1001100067D900086DD900083DC100083DC100083D
:1001200045D000083DC100083DC100083DC10008A0
:100130003DC100083DC100083DC100083DC10008A7
:100140003DC100083DC100083DC100083DC1000897
:100150003DC100083DC100083DC100083DC1000887
:100160003DC100083DC100083DC100083DC1000877
:100170003DC100083DC100083DC100083DC1000867
:100180003DC100083DC1000830B585B00DF04AF80A
:10019000012800D0FEE70DF0E7FC00F0FDFA04F0C6
:1001A0005BFD00F029FB21F019FA144D002455F8ED
:1001B000040F134921F02AFF70B121F043FB1149CC
:1001C000114A51F82400019202900023022001A953
:1001D00003931DF019FA02E00134042CE7D101F079
:1001E00003F838B9084C029001A9012001941DF0D0
:1001F0000BFA01E000F0E0FEFEE700BFFCFFFF1F8E
:100200007BC9030800000020B171030813B50B4639
:100210000979C907024602D51B68185C07E0114638
:100220009C680DF107000122A0479DF807001CBD46
:10023000F8B5164E090174181D46277B069B17F06A
:10024000060F04D1162303604FF0FF30F8BDA068FD
:1002500017F0040F18BF60606768874214D17158A7
:10026000411818696E180438864288BFC1EB000532
:10027000DE6810462A46B0476368A1685A194819D3
:10028000A06062602846F8BD0020F8BD180200207A
:100290000C48012B00EB011103D0022B03D053B902
:1002A00003E04B6800E08B68D2188B689A4205D84F
:1002B0004A60104670474FF0FF3070474FF0FF30F4
:1002C000704700BF1802002000200860704700003F
:1002D000107910F0010004D0024812680901435857
:1002E000D0187047180200202DE9F341184B14462E
:1002F0000A019D180E46297B11F0060F984617D06B
:10030000A868030A8DF8053058F802308DF804000B
:10031000010C070E8DF806108DF80770191F0422C6
:10032000E76801A82346B847227922F0040020712B
:10033000FF211022284622F0E7FF06490B6808EB50
:10034000061600205A1E30730A60BDE8FC8100BF0B
:10035000180200209C02002010B50C4659B10B7801
:100360004BB1084624F038FB012808D12046064945
:1003700023F0A0FF28B905480021016010BD00202E
:1003800010BD002010BD00BF287203089802002095
:100390002DE9F041DFF85CC0069E4FEA01180CEB36
:1003A00008040746257B6168ED071046A26804D45F
:1003B00009233B604FF0FF3519E03579521A93421B
:1003C00038BF1A46ED0708D55CF80830C9183368FD
:1003D0005918154622F0C2FE06E05CF80830B568F0
:1003E000C9183346A8470546626850196060284618
:1003F000BDE8F081180200201B68591801F0F6B919
:10040000C0F34000704700002DE9F0470E680C462D
:10041000154630462946FFF7F9FEFF2854D0B0466E
:1004200000E0904640462946FFF7F0FE284B9A1B15
:1004300002F8080008F101020028F2D1254F7B6084
:1004400008F10406287926F00306FFF7D9FF50B11A
:1004500030462946FFF7DAFEA0F1AA01484240EBF8
:100460000108043600E0804630462946FFF7CEFEFC
:1004700029468146701CFFF7C9FE02029144B01C58
:100480002946C7F80090FFF7C1FE29468246F01CB6
:10049000FFF7BCFE4FEA0A4A01068A4400200AEB35
:1004A0000903B8603873321D3B602879D618FFF70E
:1004B000A7FF10B1033626F00306B8F1000FA8D14C
:1004C00026600448BDE8F0870020BDE8F08700BF43
:1004D00008110020281100202DE9F04F8BB00D46A7
:1004E000019014469A46002630462146FFF78EFEBC
:1004F000FF2803D1CAF8006000205EE00027B81989
:100500002146FFF783FE07F108036A46985410B1AD
:1005100001371E2FF3D106F1040909EB070020F083
:1005200003092079FFF76CFF58B148462146FFF7D1
:100530006DFEA0F1AA014F4247EB010709F1040942
:1005400000E0074648462146FFF760FE2146834605
:1005500009F10100FFF75AFE2146030209F10200EA
:100560009B44FFF753FE2146804609F10300FFF745
:100570004DFE4FEA084C02060CEB0208019802A956
:100580001E22D84409F1040924F056FA48B947B9A3
:10059000149BC5F800906F60C5F8088063B11E60B9
:1005A0000AE0207908EB0906FFF72AFF00289BD014
:1005B000033626F0030697E701200BB0BDE8F08F65
:1005C0002DE9F04F5C4B15461A688BB0082A064699
:1005D0008846149C9A4602D11721016015E008ABA9
:1005E0000093084607AB03A92246FFF775FFA0F169
:1005F000010EDEF1000040EB0E0015F4007309D08F
:10060000290505D520B1112333604FF0FF348EE06A
:1006100080F001036A0502D5A90700D008B933B1FB
:1006200000E0012394F804C05FEA8C7216D5E90754
:1006300006D405F00207002F0CBF0127032700E0B6
:1006400002272A0748BF47F0040717F0060F07D014
:100650000BB90D23D8E72279530703D51E23D3E71F
:10066000002B3ED048B135490D680399099509A87A
:10067000E568083904222346A84703A9224607ABA8
:100680004FF000092E48CDF80090FFF725FF4046B7
:1006900024F0A2F92169DDF81CB04B1C0246CBEB1B
:1006A000030C00F11000844501D21C23ACE759462D
:1006B00001322346E5684046A847404624F08CF9BD
:1006C00007992579CDF814900B1D03EB000C2CF045
:1006D0000300083045F004020390CDF81090227119
:1006E00002E008B902238FE7164B8DF8187000243A
:1006F00053F8082C013206D153F8040C421C02D1E5
:1007000019684A1C05D001341033082CF0D14FF081
:10071000FF340DF10C0C9CE80F000B4D05EB04159C
:1007200085E80F00DAF80020531CCAF80030204694
:100730000BB0BDE8F08F00BF9C020020E6710308FB
:100740002A720308200200201802002010B588B089
:100750000F4C06A801F03CF800210091224602A9A6
:1007600007AB0C48FFF7B8FE2068079BC01801F0E4
:100770002CF8079004E0421C06920CF03BFF20B1DD
:100780000698079B9842F6D9012008B010BD00BF1B
:10079000100000202A720308F8B5114C00252746E6
:1007A00007EB0510FF2110220026013522F0ACFDD9
:1007B00026731034082DF3D1304601F009F80949A9
:1007C000094A0860C0F10160086108480DF076F937
:1007D0000749054A07480DF071F93046F8BD00BFDA
:1007E0001802002010000020007203082C72030879
:1007F000EC710308307203080020014602460DF038
:100800005DB9000010B504460A480021036842F2B1
:10081000107098470130F7D1012C09D1064C1820EF
:100820002368984718202268904721681820884735
:1008300010BD00BFA4020020A0020020024A034B0A
:1008400010601960704700BFA0020020A4020020C1
:100850002DE9F0470124A2B006464FF000084FF4FE
:1008600080651423274693E01FB150480368432056
:100870009847DFF844A14E48DAF80020002190475D
:10088000421C00F08480182800F28180494911FA46
:1008900000F37CD5042808D1444803680620984713
:1008A0000020FFF7AFFF40467CE0182809D13F4900
:1008B00006200A6890470020FFF7A4FF4FF0FF30A2
:1008C00070E00027DAF80030394800219847431CCF
:1008D00031D001AAB8540137842FF3D19DF804A078
:1008E000A24528D1E1439DF80570C8B2874222D1C4
:1008F00000220DF10501134611F8017F082083EA5B
:10090000072313F4004F4FEA43031CBF83F48053C3
:1009100083F021030138F4D10132802AECD19DF813
:1009200086C01B04190CBCEB136F04D19DF887E043
:10093000CAB2964504D01D4801681520884725E0B5
:1009400008F18007FFF75EFFAF420DD905F500758E
:100950003068294622F0D4FE28B90120FFF752FF63
:100960006FF003001EE03060104906200A689047CF
:1009700033680DF1060103EB0800802222F0EEFB44
:100980000AF10104E4B2B8464FF0140900274B46BF
:1009900003F1FF39002B7FF467AF0120FFF732FF2F
:1009A0006FF0020022B0BDE8F08700BFA002002077
:1009B00040420F0080000048A402002008B504490E
:1009C000044822F0FDFC0448BDE8084022F010BEB7
:1009D0004A8C0308398C03084F8C030808B511486A
:1009E00022F006FE104822F003FE104822F000FE1E
:1009F0000F4822F0FDFD0F4822F0FAFD0E4822F0CC
:100A0000F7FD0E4822F0F4FD0D4822F0F1FD0D48EF
:100A100022F0EEFD0C4822F0EBFD0C48BDE808404A
:100A200022F0E6BD978C0308A78C0308CC8C030842
:100A3000EC8C03081E8D0308428D0308738D030898
:100A4000D08D0308038E03082C8E03086A8E0308DA
:100A500008B507F06DFC034803685868BDE8084016
:100A600020F04ABE64000020022810B50C4604D0D5
:100A70000848BDE8104022F0BBBD486800210DF0D9
:100A80003FFA28B104486168BDE8104022F098BCE4
:100A900010BD00BF8D8E0308A68E030870B51948DF
:100AA00022F0A6FD1848194E22F08AFC012000F021
:100AB0006DFC3368451C04465A5D154812F0970FCB
:100AC00014BF2146202122F07BFC3168485D00F0F4
:100AD0000303012B08BF20346E2C11D0792CE1D1F7
:100AE0000C4822F06DFCFFF731FE20B90A4822F0D5
:100AF0007FFD0A4800E00A48BDE8704022F078BD5A
:100B000070BD00BFC58E0308088F03086000002079
:100B1000328F0308368F0308468F0308968F030829
:100B2000C08F030803282DE9F0410C4604D02C485F
:100B3000BDE8F04122F05CBD48682A4921F066FA20
:100B4000804628B96168284822F03AFCBDE8F08167
:100B5000A068264921F05AFA054628B9A168244818
:100B600022F02EFC2C4632E04FF4807022F074FA12
:100B7000044618B91F4822F03BFD28E00027012158
:100B80004FF480724346204621F0E0FB06460121E7
:100B9000204632462B4622F013F9B04203D21648C3
:100BA00022F026FD02E0FF2E3744E8D8284620F048
:100BB00095FF3946114822F003FC08E0284620F052
:100BC00041FE54B12046BDE8F04122F04DBA404606
:100BD00020F038FE002DF1D1F3E7BDE8F08100BF31
:100BE000C78F0308E88F0308EB8F03080A900308F8
:100BF0000D9003082C9003083E90030864900308AE
:100C00000128F8B5064602DD0D4601241DE0104816
:100C1000BDE8F84022F0ECBC55F8040F0D4921F076
:100C2000F5F9074620B90BE0C0B222F093FC384634
:100C300020F098FF431CF7D1384620F003FE03E074
:100C40000548296822F0BCFB0134B442E4D1F8BD68
:100C500075900308E88F0308A89003082DE9F74F63
:100C60000546884617460CF08DFF824600286AD05C
:100C700039482946002622F0A3FB344626E0D9F85D
:100C80000410354822F09CFBD9F8040023F0A4FEA0
:100C9000834604E0202022F05DFC0BF1010BBBF148
:100CA0001E0FF7D999F80C30D90707D52B4822F039
:100CB00087FB013657B10120386007E0D9F80010F2
:100CC000274822F07DFBD9F80010641850460CF03C
:100CD000B3FF81460028D2D150460CF0D1FF214805
:100CE0002946224622F06CFBB8F1000F30D0002ECE
:100CF0002ED028460CF046FF8046D0B928E0327B43
:100D0000D20716D501A8184973682A4620F098FC26
:100D1000002809DD019801213A46FFF79FFF2418BA
:100D2000019822F0A1F904E010487268294622F0E7
:100D300047FB40460CF080FF06460028DFD14046C6
:100D40000CF09EFF04E00A48294622F039FB544685
:100D50002046BDE8FE8F00BFBD900308C190030888
:100D6000C7900308D0900308E8900308EE900308AA
:100D70002C9103082DE9F743002481468846264636
:100D8000012712E058F8045F2249284623F092FA1E
:100D900038B12B782F2B06D029461F4822F010FBA4
:100DA00002E0012600E02C4601374F45EAD300253A
:100DB00026E028460CF0BEFE83685A69FAB19969AC
:100DC000E9B1DB69DBB107684CB1384623F004FEBA
:100DD00021460246384623F095FE80B9274602AAEE
:100DE000002042F8040D31463846FFF737FF02462F
:100DF0002EB1019919B10948394622F0E1FA0135BD
:100E00000CF0ACFE8542D4D30A2022F0A3FBBDE84F
:100E1000FE8300BF51910308549103087A9103089F
:100E200002282DE9F04105460E4601DD49481CE047
:100E30004FF4806022F010F9474F38603C4608B903
:100E4000464812E0464822F0BBFA3846FFF700FD5C
:100E5000B0F100080DDA386822F006F9002318F125
:100E6000040F0CBF3F4840483B60BDE8F04122F012
:100E7000BFBB396808F1FF3001EB0008474608F1B5
:100E8000FF383A781A2AF9D001373848791A22F00F
:100E900097FA022D26D170683549DFF8BC8021F021
:100EA000B5F82368054658B97168324822F088FAC7
:100EB000D8F8000022F0D8F8C8F80050BDE8F0815A
:100EC000FF1A01213A4618462B4621F079FFB84215
:100ED0000CBF29482948716822F072FA284620F090
:100EE000B1FC30E014F094F9054640B9244822F0F2
:100EF0007FFB206822F0B8F82560BDE8F0811BF088
:100F0000C3FF21681F4B28467A1A17F0F1FD0646E9
:100F100020B128464FF0FF3100220BE02846314631
:100F20004FF0FF3233460DF05BFF48B128464FF0DB
:100F3000FF3132460DF0C0FB0146134822F040FA63
:100F4000284614F073F9206822F08EF80021216001
:100F5000BDE8F081AA910308A8020020BD91030812
:100F6000D7910308ED910308FA910308079203084B
:100F700029AD03081B920308339203084D9203081E
:100F8000809203089B920308A292030838B5044696
:100F90000D46074822F02CFB204629461CF034FB66
:100FA000044803685868BDE8384020F0A5BB00BF7E
:100FB000AD920308640000202DE9F0437F4980488A
:100FC00099B022F0FDF907E00A2022F0C3FA7D482B
:100FD0000368586820F090FB0120312201A97A4B68
:100FE00002F014FF0130EFD09DF804100029F3D077
:100FF000012001A903F070F801A823F0EDFC18AD61
:101000002C1814F85D2C0A2A03D001A86F4923F08C
:10101000B5F801AB0AE00D2D08D86FB24FF4C80641
:1010200016FA07F202D5202003F8010C13F8015B31
:10103000002DF0D12C462E4614E0F35D272B01D075
:10104000222B03D144B1AB4207D108E0202B08D1B9
:101050003CB10723F35500E01D46012401E00025C3
:101060002C46013601AF384623F0B6FC8642E4D365
:101070000CB157483BE038460CE0651C06E023F015
:10108000ABFCA11C0246284622F0E0F8617820293A
:101090002846F4D0202123F095F804460028ECD10E
:1010A00001A84C4923F006F9002895D09DF804606A
:1010B000202E14BF01AC0DF10504204623F08CFC5A
:1010C000251815F8012C202A03D02046414923F089
:1010D00055F800230EAF0025DD510433282BF9D13C
:1010E0000DAE0BE000230A2D037003D13A4822F025
:1010F0007FFA71E746F8044F0135441C2046202151
:1011000023F060F80028EDD151E057F8044B002699
:1011100006E0A05D072802D1202109F8061001365B
:1011200057F8049C484623F057FC8642F1D32678B2
:10113000272E01D0222E11D1204623F04DFC23185A
:1011400013F8012CB24209D1601C47F8040C204668
:1011500023F042FC2418002604F8016C08F1010871
:10116000A845D2DB00241D4951F8340001EBC40628
:1011700018B91B4822F03CFA0BE00E9922F0DAFF76
:1011800028B973682BB128460EA9984701E00134AD
:10119000E9E73268002A3FF41FAF7368002B7FF441
:1011A0001BAF1048006828B121F05EFF02E00EAFCF
:1011B0008046D5E719B0BDE8F08300BF4A8C03082C
:1011C000C692030864000020FD9203086F94030890
:1011D00004930308809D03081A930308749303087B
:1011E00034930308A8020020024B00221A60012059
:1011F000704700BFA8020020014B1868704700BF6D
:10120000B0020020014B1868704700BFC0020020E8
:101210000A2808B50AD1074B07491A6809688A42A3
:1012200001D201321A60054B0021196004490A6895
:10123000904708BDC4020020B0020020AC0200208C
:10124000B802002038B504460D4605E0044803689E
:1012500014F8010B9847013D002DF7D138BD00BFB0
:10126000B80200200FB47FB508AB002153F8042B5F
:101270008DF812101B205B218DF804008DF80510ED
:101280000DF106000C2105932AF0FAFF01A823F0C6
:10129000A3FB014601A8FFF7D5FF07B05DF804EBFB
:1012A00004B0704710B5044621460448FFF7DAFF42
:1012B000034B1A68A4181C6010BD00BFE493030818
:1012C000AC02002010B5044621460448FFF7CAFFCF
:1012D000034B1A68141B1C6010BD00BFE893030881
:1012E000AC02002010B5044621460448FFF7BAFFBF
:1012F000034B1A68A4181C6010BD00BFEC930308D0
:10130000C402002010B5044621460448FFF7AAFF96
:10131000034B1A68141B1C6010BD00BFF093030838
:10132000C402002038B50446224604480D46FFF7A3
:1013300099FF0348034B04601D6038BDF493030814
:10134000AC020020C40200200148FFF78BBF00BFA1
:10135000CC95030808B50448FFF784FF0348044A06
:1013600000230360136008BDFB930308C402002040
:10137000AC020020014B1868704700BFAC0200208F
:10138000014B1868704700BFC402002008B504492B
:101390000B689847431C02D0024B1A68904708BD5F
:1013A000BC020020B402002010B5084C20600848A0
:1013B0000160084908480A60084A02990360116000
:1013C0000748084A00230360136010BDB0020020E4
:1013D000C0020020B8020020BC020020B40200209D
:1013E000C4020020AC02002010B54C4B1A68111842
:1013F0004B7813F0970F40F090801B2844D10220C7
:1014000000234FF48071464A02F0B8FE013079D0D3
:1014100002204FF480710023414A02F0AFFE411CCC
:1014200073D0A0F14101032911D8432809D04428E1
:101430000AD040F2011442280CBF20464FF48070BD
:1014400010BD40F2031010BD4FF4817010BDA0F12B
:101450003104052C59D8022000234FF48071304A02
:1014600002F08CFE7E2850D1052C4ED8DFE804F027
:10147000034D4D5006094FF4827010BD4FF4837038
:1014800010BD40F2071010BD0D2809D102204FF405
:101490008071234A002302F071FE4FF4847010BD66
:1014A000092817D009DC032820D002DC01282CD120
:1014B00016E0052817D008280AE015281CD004DCFF
:1014C0000B281CD0142820D113E01A2805D07F281F
:1014D0001BD120E040F2091010BD4FF4867010BD02
:1014E00040F20D1010BD4FF4877010BD40F20F1088
:1014F00010BD4FF4887010BD40F2111010BD4FF4B4
:10150000897010BD40F20B1010BD4FF48A7010BDF1
:1015100040F2051010BD4FF4857010BD6000002032
:10152000A086010028B902204FF480710022002318
:1015300005E0044B02204FF480714FF0FF3202F0BF
:101540001DBE00BFFFFF0F0002460B4602204FF4F6
:10155000807102F013BE02460B4602204FF48071E8
:1015600002F00CBE0146022002F046BE01460220F7
:1015700002F042BE022002F03FBE0000F0B5114D65
:101580000E4600F178470FCD8DB06C460FC40FCDDD
:101590000FC495E80F0084E80F000023ADF10402AA
:1015A000184652F8041F5B180130BB4201D80C28C2
:1015B000F7D11EB103F10062531E336001380DB044
:1015C000F0BD00BF0094030813B50CF017FA022019
:1015D0000822034600244FF4E13100940AF0CCFFC6
:1015E0002146022002F00FFE2146022002F009FEF1
:1015F00009480CF093FD09480CF096FD084809498C
:10160000FFF71CF9084B094A009319205021084B99
:10161000FFF7CAFE1CBD00BF75150008571500086E
:101620006D15000849150008E91300086515000844
:101630002515000804288CBF0020012070470428CD
:1016400004D80F298CBF002001207047002070476C
:10165000D0F1010038BF0020704702288CBF002065
:101660000120704703288CBF0020012070470BF039
:10167000E7BB0F288CBF00200120704740F6FF70A9
:10168000704710B50C4600F081FC037864F3410309
:10169000037010BD08B500F079FC017801F001007D
:1016A00080F0010008BD70B5044600200E4600F031
:1016B00075FCC36EB342054605D090F860106FF319
:1016C000C30180F8601020460BF0E6FBEE6670BDAB
:1016D0000B4A034692E8030082B002AA012B02E9FA
:1016E000030009D802EB830353F8080C430704D026
:1016F00020F00700083000E0002002B0704700BF73
:10170000309403080B4A034692E8030082B002AA11
:10171000012B02E9030009D802EB830353F8080CFC
:10172000420704D020F00700083800E0002002B093
:10173000704700BF3894030810B50446631E08467E
:10174000D9B203290DD80C214B430949CB585BB1C1
:10175000032C114603D1BDE8104000F02DBA984784
:1017600010BD6FF0010010BD6FF0020010BD00BF92
:1017700028AC030838B50446631E0846D9B20329CD
:101780000ED80A490C2505FB03139B685BB1032C9B
:10179000114603D1BDE8384000F03ABA984738BD49
:1017A0006FF0010038BD6FF0020038BD28AC0308AF
:1017B00038B505460C4602F077F9284602F028FABB
:1017C000034608B12046984738BD0021FFF7D6BE32
:1017D00013B5044601A90448FFF7D0FE0CB101304F
:1017E00020600199481C1CBD2BF903080BF0E4BED6
:1017F000002300E001334008FCD11846704710B5C3
:1018000004460846FFF7F4FFC1B22046BDE8104089
:1018100000F048BD034B1870187842B20132FBD17A
:10182000704700BF240000202DE9F8434FF40077F3
:101830000024224D224855F82420511C45F824103C
:1018400055F8242050F824309A42A94621D31D4B44
:10185000DFF87C801978012212FA04F6F6B246EA23
:101860000100187098F800C016EA0C0F03D003208E
:10187000394602F019F9144B1878064203D00021BA
:1018800045F8241005E098F8002022EA060688F8BA
:10189000006001340137042CBFB2CAD10B4B197858
:1018A00048B2421C08D093F800C04FFA8CF10020D7
:1018B000FF2249F821001A70BDE8F883D802002001
:1018C000EC020020E8020020FC020020240000209E
:1018D000E902002001207047B0F5007F06D3A0F593
:1018E000007003288CBF0020012070470B2805D909
:1018F000A0F58073584240EB030070470120704709
:101900002DE9F041A0F50075032D044616461F464B
:101910001CD8002E77F101013BD20A23A2FB030160
:1019200003FB07111C4A00232FF0BEFE064620468B
:101930000F46FFF76FFF194B53F8251000230A4697
:10194000B24273EB0701F6D3BDE8F081B0F5807FBA
:101950001BD156EA07031CD00BF03AF804460D469B
:101960000BF036F8A04271EB050305D24FF0FF32C1
:101970000B4B801841EB0301001B61EB0501B042EA
:1019800071EB0703ECD3BDE8F081BDE8F0410AF04C
:101990000BBFBDE8F08100BF40420F00D80200201D
:1019A000FFFF0F002DE9F843DDE9086790469946EF
:1019B000032100220023044600F036F8464577EB69
:1019C000090305460ED2002200232046062100F01E
:1019D0002BF801220024921944EB0703121843EB61
:1019E000010301E032463B460D4CB2EB080263EBCB
:1019F0000903A2FB040104FB03112A4600232FF074
:101A000053FE0B46074902466FF00100904271EB0E
:101A100003043CBF02460B4610461946BDE8F88356
:101A200040420F00FFFF0F00B0F5807F73B5044602
:101A300015D1062933D8DFE801F00404474709101F
:101A40000C0002B0BDE870400AF0C2BF4FF0FF309A
:101A500001E06FF0010020493BE0012038E0A0F5F3
:101A60000076032E11D9042908D106210022002373
:101A7000FFF7DAFFCDE9000120461EE0052918D066
:101A800002B0BDE870400AF0BFBE062907D8DFE803
:101A900001F0040819190D101D00FFF7BBFE00200E
:101AA00016E00E4850F82630184611E04FF0FF328D
:101AB00000E001220023CDE9002300220023FFF7EC
:101AC00071FF06E00A2003E0054801E04FF0FF3017
:101AD000002102B070BD00BFFFFF0F00D802002040
:101AE00040420F002DE9F047A0F50075032D064692
:101AF00090469946DDF820A047D8B8F1000F79F15B
:101B000001013CD2012717FA05F458EA0903E4B2AF
:101B10000CD1244BE44393F800C0E0B200EA0C017E
:101B20001970214B1A7800EA020424E00A23A2FB70
:101B3000030103FB09111D4A00232FF0B5FD0246E6
:101B40000B4652EA03011DD019491A4B41F82520D2
:101B500018781549BAF1010F0CBFA0432043187043
:101B60000A7822EA040E304681F800E0FFF752FEC0
:101B70000C4B187804431C700020BDE8F08702204D
:101B8000BDE8F0873846BDE8F087B0F5807F05D026
:101B9000CDF820A0BDE8F0470AF062BE0320BDE802
:101BA000F08700BFE9020020E802002040420F0059
:101BB000EC020020FC020020A0F5007238B595B2BE
:101BC000032D0C4611D8012313FA02F20E4B18789C
:101BD0001978D2B202420CBF00200120012C0CBFA8
:101BE0000A4321EA02021A7038BDB0F5807F04D0A2
:101BF000064A936923B1984738BD6FF0030038BD9A
:101C00006FF0020038BD00BFE902002028AC0308D5
:101C1000A0F5007238B595B2032D0C4610D80123FB
:101C200013FA02F20D4B1978D2B20A420CBF00200F
:101C3000012094B193F800C02CEA0201197038BD5C
:101C4000B0F5807F04D0064A136A23B1984738BDA7
:101C50006FF0030038BD6FF0020038BDE8020020CD
:101C600028AC03080249034AB0FBF1F31360704744
:101C700040420F00C80200200249034AB1FBF0F3C2
:101C80001360704740420F00CC020020054906480F
:101C9000D1E900230068121843F10003C1E90023D1
:101CA000704700BFD0020020CC0200202DE9F8438D
:101CB000194C0AF075FED4E9002303E00AF070FE27
:101CC00032463B46D4E9006786EA020887EA030900
:101CD00058EA0903F2D1114B1A6800232FF0E4FCF3
:101CE0000F4B341847EB01056FF00102A24273EB72
:101CF00005010CD2204629462FF0D6FC14461D467D
:101D00000AF056FE0448C0E900890AF059FE204650
:101D10002946BDE8F88300BFD0020020C802002099
:101D2000FFFF0F002DE9F0411446104A0C2652F82F
:101D300020704E43BD194FF001086B701B19D9B2CA
:101D4000B95508FA01F1A86821F0DAFCA86048B991
:101D5000B855E8806880A880D4F1010038BF002021
:101D6000BDE8F0814046BDE8F08100BF74940308EF
:101D7000054B53F820000C2202FB01030022DA80FD
:101D80005A809A80704700BF749403082DE9F04789
:101D90000C254D430B46364951F820607119044615
:101DA0004888D1F808901FFA80F8705D00285CD050
:101DB000CF881FFA87FA4F784FF0010CC01B0CFA3E
:101DC00000F0824509DD2B490A682B49D06822467C
:101DD00020F036F90020BDE8F0870CFA07F404F093
:101DE0000707E01D7C1E09EB0803C010062C05D870
:101DF000DFE804F0201C1814100C080012F8017B16
:101E000003F8017B12F801CB03F801CB12F8014B68
:101E100003F8014B12F8017B03F8017B12F801CBA8
:101E200003F801CB12F8014B03F8014B12F8017BC8
:101E300003F8017B92F800C00138002883F800C045
:101E400002DD01330132D9E7735D4F784C88012000
:101E500010FA03F210FA07F3013A13FA84FC02EACB
:101E60000C074F80CA881318CB80BDE8F08700BFED
:101E70007494030864000020409403080C234B432F
:101E8000064951F82020D05CD11830B191F801C03A
:101E90000122CCEB000012FA00F0704774940308A2
:101EA000044B53F820000C2202FB0103D88880B2B7
:101EB000704700BF74940308F8B50C2404FB01F5C7
:101EC000314951F820607419705DA388A1689BB2F4
:101ED000002852D0B4F806C01FFA8CF000284FD06A
:101EE0006078012717FA00F000F00707CB18C11D32
:101EF000781EC910062805D8DFE800F0201C181449
:101F0000100C080013F8017B02F8017B13F801EBB9
:101F100002F801EB13F801CB02F801CB13F8010B27
:101F200002F8010B13F8017B02F8017B13F801EBB7
:101F300002F801EB13F801CB02F801CB1878013954
:101F40000029107002DD01320133DBE700200BF0C5
:101F500097FDE388591EE1800BF092FD725D637876
:101F6000A188012010FA02F710FA03F2013F12FAD9
:101F700081F307EA0302A280F8BD4FF0FF30F8BDFD
:101F80004FF0FF30F8BD00BF74940308024B1C22D1
:101F900002FB0030704700BF880E002000487047E9
:101FA000100E00202DE9F041FFF7F8FF90F87420A3
:101FB00050F82210426E836ED1F804809A42044693
:101FC00007D190F860E00EF0020C5FFA8CF0002868
:101FD00050D000200BF054FD0026074684F87460B2
:101FE0003546616E31FA05F3DB071AD52846FFF74F
:101FF000CDFF94F8741044F8210094F874300178FF
:10200000203304EB4302436882616FF304110170D3
:10201000434508BF94F8746094F87400421C84F837
:1020200074200135102DDCD194F8745084F875506B
:1020300006E094F87420501C44F8225084F8740090
:1020400094F874C0BCF10F0F4FF00005F1D984F87B
:1020500074500AF04DFF616EA16684F8746094F8C4
:102060006030384665F3410384F86030BDE8F041E4
:102070000BF006BDBDE8F0812DE9F0478A46044625
:10208000FFF784FF05460020FFF788FF06460BF0A8
:102090000AFD00200BF007FD4FF0010980462146A4
:1020A0004846FFF7EBFE09FA0AF787420BD04B468A
:1020B000484621465246FFF735FE4845034611D1B2
:1020C0002146FFF755FEAF82297841F001002870C4
:1020D000736E012515FA04F41C43746640460BF038
:1020E000CFFC2B461846BDE8F08770B50546FFF7D4
:1020F0004DFF06460020FFF751FF0123446E13FAFF
:1021000005F124EA0102426696F800C075606FF39B
:10211000000C86F800C0347844F002013170307849
:1021200000246FF3C3003070B4823278347264F3E9
:1021300082023270294674811846F4600422FFF747
:10214000F1FD28462146BDE870400AF0E9BF37B5E9
:102150000546FFF71BFFB0F80AC0037A01211FFAFA
:102160008CF211FA03F39A42044606D1002343810C
:1021700090F800E04EF008020270E268B4F80AE05D
:1021800023691FFA8EFC33F81C00131AE3602278CF
:1021900002F01001C8B240B1A2691088ADF8060083
:1021A00021786FF30411217005E0012029460DF11B
:1021B0000602FFF781FE62892369BDF806001FFA57
:1021C00082FC23F81C00E368618922691FFA81FE02
:1021D00032F81EC00CEB0300E06061894B1C638188
:1021E0003EBD10B5FFF7D2FE00234381C3600278E5
:1021F00063F3C302037A0270002B52D0012414FA55
:1022000003F303F00701DA1D4C1ED210062C05D88B
:10221000DFE804F03C342C241C140C00002301697A
:10222000002421F81340591C8BB200E000230169FF
:10223000002421F8134001339BB200E00023016920
:10224000002421F8134001339BB200E00023016910
:10225000002421F8134001339BB200E00023016900
:10226000002421F8134001339BB200E000230169F0
:10227000002421F8134001339BB200E000230169E0
:10228000002421F8134001339BB200E000230169D0
:10229000013A0024002A21F8134002DD01339BB2E9
:1022A000BDE710BD70B506460D46FFF76FFE03781B
:1022B000DA07044602D530460AF0EEFD207AA8423D
:1022C0000FD0022125722069A94021F019FA20615E
:1022D00038B9E0602278207260F3C3022270608116
:1022E0003DB93046FFF77DFF01203146FFF740FD45
:1022F000012070BD38B50546FFF748FE2946044663
:102300000120FFF7CDFD80B210B92078C0F3001096
:1023100038BD37B50546FFF739FE00230446284689
:10232000ADF80630FFF7E6FF002834D0227A237894
:10233000AAB103F00801C8B268B32846FFF707FF47
:10234000B4F814C01FFA8CF212B1A08A431EA38203
:10235000E268237A32FA03F1ADF806101BE003F0CD
:102360001001C8B258B1A369B3F800C0ADF806C0F7
:1023700094F800E062F3041E84F800E005E0012018
:1023800029460DF10602FFF797FDA08A82B212B12D
:10239000A38A591EA182BDF806003EBD70B50E4647
:1023A0000446FFF7F3FD05462046FFF7A3FFB042C2
:1023B0000CD2297801F00200C3B23BB12A78D107D0
:1023C00004D52046FFF796FFB042F7D32046BDE87C
:1023D0007040FFF78FBF00000A4B5A6882B95A61FC
:1023E0001A684FF0FF31D96019612AB906484FF0D9
:1023F00058311960C0F8B4214FF480725A609A6065
:102400000020704788050020C0030020064B1A6892
:10241000904203D359685218904202D39B68002B14
:10242000F5D11846704700BF7805002000F108027A
:1024300012F0070302D0534203F00703C018C91A71
:10244000064B41F001029861D9604260411804488E
:1024500028224A600269DA61704700BFC003002089
:1024600088050020F4282DE9F84FAC4C00F2828159
:102470000A2884BF00F10B0525F007052768A74B44
:1024800098BF1025EA0837FA02F188071AD001F040
:10249000010080F001018A1803F1240505EBC20553
:1024A000A8688468A54205D10121914027EA010767
:1024B0001F6005E01B699C42C0F08E86AC60E56041
:1024C000D20041E39E68B54240F22B83002974D0CC
:1024D0004FF0010808FA02FC0CFA08F0464211FA23
:1024E00002F246EA000C0CEA0206714201EA06001A
:1024F000411E0A0B02F0100031FA00F2560906F0F4
:10250000080101EB000C32FA01F0860806F0040223
:10251000D04020FA08F10CEB020601F0020230FA7A
:1025200002F121FA08FCB6180CEA080031FA00F2B0
:1025300006EB000C944403F1240101EBCC06B068D7
:102540008268964205D108FA0CF827EA08071F604E
:1025500005E01B699A42C0F03F86B260D6604FEA40
:10256000CC077B1B45F00306451943F0010246608A
:102570006A60EB50A668694FD6B14FEAD60C4FF0AF
:1025800001083E687A6901EBCC0108FA0CFC1CEAF0
:10259000060F04D14CEA06063E600E4604E08E6843
:1025A0003F69BE42C0F018868A60F2609660D160D2
:1025B000A36065610830BDE8F88F5A68002A00F012
:1025C000B082504200EA02077A1E160B06F0100095
:1025D00032FA00F7790901F0080637FA06F18A089D
:1025E00002F0040731FA07F206EB000C560806F079
:1025F000020032FA00F1BC444F0807F001020CEB74
:102600000006B71831FA02F03A1803EB8201D1F84C
:102610002C114B6823F00300421B08460AE05F6858
:1026200027F00301C5EB010C94452CBF94461846D6
:10263000624619460B69002BF1D14B69002BEED194
:10264000D4F810C06045C0F0C7854719B84280F083
:10265000C385C3688169834206D086686645C0F039
:10266000BB85F3609E601EE0436913B100F1140660
:1026700007E00369BBB100F1100602E003F11406A4
:102680003368D3F81480B8F1000FF7D1D3F8108075
:10269000B8F1000F02D003F11006F1E76645C0F073
:1026A0009B85C6F80080002934D0D0F81C801B4ED2
:1026B00008F14A0C04EB8C0CDCF8048040450BD18B
:1026C000CCF8043093B9C369012111FA03F371689E
:1026D00021EA030373601DE03669B142C0F07C85D6
:1026E0000E6986420CBF0B614B619BB12669B342F8
:1026F000C0F072859961016921B1B142C0F06C8569
:1027000019618B61416929B12669B142C0F06485C4
:1027100059618B610F2A03D8521915E2C0030020BA
:1027200042F0010345F0030545607B60BA50A6689E
:10273000AA4BE6B14FEAD60C03F124051E6859698D
:102740004FF0010805EBCC0508FA0CFC1CEA060F5B
:1027500004D14CEA06061E602E4604E0AE681B69F2
:102760009E42C0F03985A960F1608E60CD60A260A4
:1027700067611FE710F1410F00F2D181666800F137
:102780000B0222F00705002E00F0CB816A42290AD5
:1027900027D0B1F5803F23D2A1F580774FEA1743C8
:1027A00003F0080C01FA0CF1A1F58050070C07F0BA
:1027B0000407B940A1F58043180C00F002036744F8
:1027C00011FA03F007EB030CCCEBD03000F115014C
:1027D00035FA01F303F001010E3001EB400100E096
:1027E0001F2104EB8100D0F82C31002B2ED01F29A3
:1027F0001ABF4FEA5108C8F119084FF000084FF00E
:10280000000C05FA08F8174660465A6822F00302E1
:10281000521BBA4202D292B1174618464FEAD879F3
:102820005A6909F1040953F8293012B19A4201D1C9
:1028300002E062462BB194464FEA4808E5E71846A5
:1028400001E013463A46B3BB002842D16FF00103C2
:1028500013FA01F111EA06032BD0594201EA0300F1
:10286000461E330B03F0100036FA00F3590901F04D
:10287000080633FA06F106EB000C880800F00403A2
:102880009C4431FA03F35E0806F002000CEB0006EC
:1028900033FA00F0410801F0010306EB030C30FAB3
:1028A00003F10CEB010004EB80060020D6F82C317C
:1028B0000FE018460DE0596821F00306711B9142A4
:1028C00028BF11461A6938BF184602B95A6913461B
:1028D0000A46002BEFD1002800F02381A368C5EB46
:1028E000030C624580F01D813C4ED6F810C0604557
:1028F000C0F072844319984280F06E84C168866982
:10290000814206D087686745C0F06684F9608F60B1
:102910001EE0416911B100F1140707E00169B9B186
:1029200000F1100702E001F114073968D1F81480B2
:10293000B8F1000FF7D1D1F81080B8F1000F02D034
:1029400001F11007F1E76745C0F04684C7F8008041
:10295000002E34D0D0F81C80204F08F14A0C04EB34
:102960008C0CDCF8048040450BD1CCF8041091B9F4
:10297000C169012616FA01F17E6826EA0101796033
:102980001DE03F69BE42C0F02784376987420CBF13
:102990003161716199B12769B942C0F01D848E61BE
:1029A000066926B1BE42C0F017840E61B161466966
:1029B0002EB12769BE42C0F00F844E61B1610F2A6B
:1029C0000ED802EB050C4CF00302426000EB0C0247
:1029D000516841F0010353609DE000BFC003002037
:1029E000D10845F0030742F001061F2947605E60E9
:1029F0009A5019D8954E276806F124024FF0010C21
:102A000002EBC1020CFA01F1394203D139433160C2
:102A1000114604E091683669B142C0F0DD839360ED
:102A2000CB609960DA6076E0160A29D0B6F5803F6F
:102A300025D2A6F580714FEA114707F0080906FA7A
:102A400009F8A8F580564FEA164101F0040108FA8A
:102A500001F6A6F580473F0C07F0020709EB010CD1
:102A6000BE400CEB0708C8EBD63707F1150132FA68
:102A700001F606F001090E3709EB470600E01F26B4
:102A80004FF0010CD4F80480DE610CFA06F900273F
:102A900019EA080F5F611F616C4906F14A0C07D102
:102AA00049EA08024A6001EB8C0141F8043F20E04A
:102AB00001EB8C011F2E496802D07608C6F1190778
:102AC00012FA07F600E061464F6827F003079742C5
:102AD00013D0F70F043701EB870851F827C07600B1
:102AE000BCF1000FEFD122699045C0F0758341F829
:102AF00027309961DB609B600DE026698A68B142EE
:102B0000C0F06A83B242C0F06783D3608B60D96043
:102B100000219A609961083040F0788301E04FF01D
:102B2000FF35A268494E954217D8531B0F2B706989
:102B300007D9421943F001017261B3605160D3506B
:102B40005AE30023B360736142F0030182184160CD
:102B5000536843F0010151602CE5F268954208D2B8
:102B6000B069511B431941F00102F160B3615A6031
:102B700042E3FFF731FCD6F8B401DFF8D89010F04B
:102B8000040F72D1B06918B1FFF740FC824620BB38
:102B900000200BF0CDF9421C064660D0D9F8083071
:102BA0005F4203F1290CD9F804305A1E0CEB050ED4
:102BB00010420EEA070705D0391AC2185F4202EA2E
:102BC00007000F18224B9F4249D838460BF0B0F946
:102BD000B042804640F01C836BE0D9F80830F268C0
:102BE00003F12901C2EB010E5F420EEB050018490B
:102BF00007408F4233D838460BF09AF99AE80C0018
:102C000002EB030C6045804640F00283013050D156
:102C100025E00F4B9F424CD805F12906B74248D218
:102C2000D9F8082002F1290C0CEB050E5142C7EB34
:102C30000E0000EA01069E42C7F1000A39D830466C
:102C40000BF076F9013007D0BF1932E0C003002045
:102C5000FEFFFF7F8805002050460BF069F9D4F88D
:102C6000B40140F00403C4F8B431D9F8081001F1FC
:102C7000290E4B420EEB05028D4902EA0300884201
:102C800000F2BF820BF054F9804600200BF050F99F
:102C9000B8F1FF3F00F0B582431C00F0B2828045DE
:102CA00080F0AF82C8EB000705F12800874240F2B0
:102CB000A882D4F8AC31D4F8B061FA18B24288BF17
:102CC0007C4EC4F8AC2188BFC6F8B021A669794B08
:102CD000D6B9D9F80010C3F81080C3F8B881C3F88A
:102CE000BC71C3F8C461196203F1240203F5927345
:102CF000D260926008329A42FAD14046A7F1280188
:102D000015E09B681BB915E003F5DC739B461A6858
:102D1000596802EB010CE045F3D17EE2964209D3FB
:102D2000464507D2C8195860E268A069B918FFF78C
:102D30007DFB55E2236998453CBF5E4BC3F810808C
:102D40005D4B03E09B68002B00F07581196808EB70
:102D5000070E7145F6D165E25E68C3F80080F71989
:102D60005F6008F1080313F0070002D05A4202F036
:102D7000070001F1080313F00702404402D05B4250
:102D800003F007028A18C0EB020C4319C5EB0C06CE
:102D900045F003054560A169464D8A4207D1EA68BE
:102DA000AB61B618EE6046F001065E6002E4696948
:102DB0008A4209D1A9686B61761846F00102AE60BB
:102DC0005A609E51FFF7F6BB516811F0020F40F0B8
:102DD000968021F0030C4FEADC08B8F11F0F1ED8D3
:102DE0009768D1688F4207D1012707FA08F82F6842
:102DF00027EA0801296080E005F1240909EBC808E9
:102E0000474503D02D69AF42C0F0E681414503D06C
:102E10002569A942C0F0E081F9608F606DE0D1685A
:102E2000976991420AD0D2F808802D69A845C0F070
:102E3000D381C8F80C10C1F8088020E0516911B1A5
:102E400002F1140507E01169C9B102F1100502E0B1
:102E500001F114052968D1F81490B9F1000FF7D1E8
:102E6000D1F81080B8F1000F02D001F11005F1E7A0
:102E7000D4F810904D45C0F0AF81C5F80080002F08
:102E80003BD0D2F81CE00B4D0EF14A0804EB880849
:102E9000D8F804904A4511D1C8F80410C1B9D169D5
:102EA000012717FA01F16F6827EA0101696024E040
:102EB000FEFFFF7FC0030020780500202D69AF4290
:102EC000C0F08A813D6995420CBF39617961A1B139
:102ED000D4F810804145C0F07F818F61156925B11C
:102EE0004545C0F079810D61A96155692DB127690A
:102EF000BD42C0F071814D61A9616244664455686C
:102F000025F001015160F10846F001021F295A60C5
:102F10009E5119D8B14D2468012605F1240C0CEB03
:102F2000C10216FA01F1214203D121432960114661
:102F300004E091682C69A142C0F04E819360CB609F
:102F40009960DA60FFF736BB310A27D0B1F5803FD0
:102F500023D2A1F580774FEA174202F0080801FA60
:102F600008F1A1F580552F0C07F00407B940A1F531
:102F70008042150C05F0020208EB070C91400CEBA7
:102F8000020ECEEBD13707F1150536FA05F202F045
:102F900001080E3708EB470100E01F214FF0010741
:102FA000D4F804C0D96107FA01F8002518EA0C0F1B
:102FB0005D611D61894A01F14A0707D148EA0C01A8
:102FC000516002EB870242F8043F1FE002EB8702E8
:102FD0001F29526802D04D08C5F1190516FA05F1EE
:102FE00000E03A46556825F00305B54213D0CF0FEF
:102FF0003D1D02EB850C52F825704900002FF0D1E1
:1030000021698C45C0F0E88042F825309A61DB6088
:103010009B60FFF7CFBA24699168A242C0F0DC80C0
:10302000A142C0F0D980CB609360DA600022996041
:103030009A61FFF7BFBA3046FFF7E8F990E80C0055
:1030400002EB030AAAF1270212F007001CBF50424C
:1030500000F00700AAF12F09814406F1100189450B
:1030600038BFB1464046A7F12801FFF7DFF91B231F
:10307000C9F804309BE80F0009F1080C8CE80F0038
:103080000020C4F8B881C4F8BC71C4F8C401C4F805
:10309000C0C109F11803072043F8040F191D8A4520
:1030A000F9D8B14500F09C80C6EB0902B31842F094
:1030B0000107586820F00101D0081F285960776087
:1030C000B25017D845492268012701F1240E0EEBB2
:1030D000C00317FA00F0104203D102430A601A46F7
:1030E00003E09A6809698A4276D39E60D660B2602E
:1030F000F36075E0110A27D0B1F5803F23D2A1F526
:1031000080774FEA174303F0080801FA08F1A1F5A8
:103110008050070C07F00407B940A1F58043180C54
:1031200000F0020308EB070E99400EEB030CCCEB0A
:10313000D13707F1150032FA00F303F001080E371A
:1031400008EB470100E01F214FF00107D4F804C04D
:10315000F16107FA01F8002018EA0C0F7061306184
:103160001E4B01F14A0707D148EA0C025A6003EBF3
:10317000870343F8046F1EE003EB87031F295B6896
:1031800002D04908C1F1190012FA00F100E03B46F3
:10319000586820F0030C944511D0CF0F381D03EB75
:1031A000800C53F820704900002FF0D1226994451B
:1031B00012D343F82060B361F660B66010E0216975
:1031C0009A688B4208D38A4206D3D6609E60F36029
:1031D0000023B260B36103E01EF006FAC0030020D2
:1031E000E168134B8D420CD29869491B4219D96092
:1031F00041F001019A61516045F003054560FFF718
:10320000D9B91EF0AFFA0C2303600020BDE8F88F97
:10321000B8F1FF3F7FF4FDAC21E5D86800077FF5EA
:103220007DAD87E5DA6812073FF505AF94E500BF8D
:10323000C00300202DE9F041002800F00582914DE7
:103240002E69A0F10803B3422C46C0F0FB8150F870
:10325000047CBA0740F1F68127F0030217F0010F52
:1032600003EB020140F0958050F8087CDB1BB34271
:10327000C0F0E881686983423A447ED0FF081F2F7E
:103280001CD89D68D868854207D12568012616FAA2
:1032900007F725EA070727607BE004F1240C0CEB15
:1032A000C707BD4202D0B542C0F0CC81B84202D0BF
:1032B000B042C0F0C781E86085606AE0DF689D6960
:1032C0009F4207D09868B042C0F0BC81C760B86028
:1032D00038461DE0586910B103F1140706E038695B
:1032E000B0B1103702E000F114073868D0F814C00C
:1032F000BCF1000FF7D1D0F810C0BCF1000F02D024
:1033000000F11007F1E7B742C0F09C81C7F800C098
:10331000002D3ED0DF695B4E4A3704EB8707D7F8B4
:1033200004C063450AD1786090B9D869012515FABF
:1033300000F0756825EA000070602AE03669B54241
:10334000C0F080812E699E420CBF2861686100B385
:103350002669B042C0F0768185611D6925B1B5420C
:10336000C0F070810561A8615D6995B12669B542BB
:10337000C0F068814561A8610BE0486800F0030C6B
:10338000BCF1030F05D1AA60486820F00100486035
:1033900024E08B4280F056814868C50740F1528195
:1033A00010F0020640F0BB80A769364DB9420ED13D
:1033B000E968AB61501840F00101E86059606A6942
:1033C000934240F041816E61AE60BDE8F0816E696C
:1033D000B14209D1A8686B611218AA6042F00101DC
:1033E00059609A50BDE8F08120F00307F8081F28C3
:1033F0001ED88E68C9688E4207D1012111FA00F0EB
:10340000296821EA000028607DE005F1240C0CEB1E
:10341000C000864203D02D69AE42C0F013818142C4
:1034200003D020698142C0F00D81F1608E606AE0B6
:10343000C8688E6988420AD0D1F808C02D69AC45A9
:10344000C0F00081CCF80C00C0F808C023E0486947
:1034500010B101F1140507E00869E0B101F11005B0
:1034600002E000F114052868D0F81480B8F1000FCC
:10347000F7D1D0F810C0BCF1000F05D000F1100555
:10348000F1E700BFC0030020D4F810804545C0F02C
:10349000D980C5F800C0002E35D0D1F81C806B4D06
:1034A00008F14A0C04EB8C0CDCF8048041450BD18C
:1034B000CCF8040090B9C969012010FA01F16868DC
:1034C00020EA010169601EE02D69AE42C0F0BA80B9
:1034D00035698D420CBF30617061A0B1D4F810C065
:1034E0006045C0F0AF8086610D6925B16545C0F0CB
:1034F000A9800561A861496929B12569A942C0F07F
:10350000A18041618861D21942F0010058609A504F
:1035100061698B420AD14D4B9A60BDE8F08120F081
:10352000010042F0010548605D609A50D1081F29F2
:1035300018D846482468012500F1240202EBC10294
:1035400015FA01F1214203D121430160114603E044
:1035500091680069814275D39360CB609960DA60AD
:10356000BDE8F081100A24D0B0F5803F20D2A0F54C
:103570008077390C01F008018840A0F580552E0CA9
:1035800006F00406B040A0F580473D0C05F00205AA
:103590008F19A84007EB050CCCEBD03606F11501CE
:1035A00032FA01F505F001070E3607EB460000E0A0
:1035B0001F204FF001066768D86106FA00FC00255D
:1035C0001CEA070F5D611D61204900F14A0607D121
:1035D0004CEA07074F6001EB860141F8043F1EE00B
:1035E00001EB86011F28496802D04008C0F1190587
:1035F00012FA05F000E031464D6825F003059542CA
:1036000012D0C70F3D1D01EB850751F82560400022
:10361000002EF0D12269974214D341F825309961E8
:10362000DB609B60BDE8F08120698A68814209D334
:10363000824207D3D3608B60D96000219A60996180
:10364000BDE8F0811DF0D0FFBDE8F081C00300208F
:1036500038B568B141EA0004220C130400FB01F5FF
:103660003BB1B5FBF0F0884218BF4FF0FF3500E0EA
:1036700005462846FEF7F6FE044618B100212A4604
:103680001FF042FE204638BDF8B50E46044620B96C
:103690000846BDE8F840FEF7E5BE19B9FFF7CAFDD8
:1036A00035466DE0413105D91EF05CF80C2303600E
:1036B000002565E0334D50F8041CA0F1080228698C
:1036C0008242AC4643D38D0741D521F00307D5197B
:1036D000AA423CD26B68D80739D50A2E86BF06F1BC
:1036E0000B0323F0070310239F4215D3FD1A0F2D60
:1036F0002FD901F00101D01841F0020C4CEA03036C
:1037000045F00301451944F8043C41606B6843F0FF
:103710000101696008301DE0DCF818C019486545F2
:103720001DD1C5687D199D4219D901F0010102EB37
:10373000030CED1A41F00201194345F0010344F86E
:10374000041CCCF80430C0F818C0C56001E01DF0BE
:103750004BFF00201AB190B1FFF76CFD0FE030462F
:10376000FEF780FE054658B13A1F2146964238BF03
:1037700032461FF0F3FC2046FFF75CFD00E02546D3
:103780002846F8BDC00300204FF0FF32002380E838
:103790000C00704703C80022002300F0EFBC0000BB
:1037A000F7B504460E4603211DF048F920460121D5
:1037B0000AF0D8FE18B92046194914F081FC2046B9
:1037C00002210AF0CFFE18B92046164914F078FC01
:1037D000204601210AF02CFF2DF072FD054600F075
:1037E000C8FC18B92046104914F06AFC2046022192
:1037F0000AF01EFF2DF064FD0746FEF76DF818B9BC
:1038000020460A4914F05CFC0023009386E8A000DF
:1038100028464FF4E1310822022308F0ADFEFEBD38
:103820007C94030895940308AF940308BF9403089D
:10383000F7B504460E4603211DF000F9204601218C
:103840000AF090FE10B920461F4906E020460221EA
:103850000AF088FE30B91D49204603B0BDE8F040AB
:1038600014F02EBC204601210AF0E2FE2DF028FDC6
:10387000054600F07EFC18B9204615492A460CE0A2
:10388000204601210AF0D4FE2DF01AFD0746FEF76E
:1038900023F838B90F4920463A4603B0BDE8F04056
:1038A00014F00EBC0C4800234FF0FF3202604FF4BE
:1038B000E131009386E8A00028460822022308F0A0
:1038C0005BFE012003B0F0BD7C94030895940308CF
:1038D000D0940308E79403082800002013B5036878
:1038E000581C10D109480A4B019002218DF8001094
:1038F00002AC14E9030003F1080282E8030018682F
:10390000012120F053F90B601CBD00BF9AFFFF7F1F
:1039100038110020F7B5224B174605460E464FF0EA
:10392000FF32002438E0D5F800C0BCF1FF3F0FD1D2
:103930001C481D4B019002218DF8001002AC14E9C7
:10394000030003F1080282E80300186801211DE06A
:1039500016480168002906DA6968604600F00EFC26
:10396000011E15DA03E04FF0FF33036010E0104A48
:103970000D4F019201268DF8006002AD15E903009C
:1039800007F1080C8CE803003868314620F00EF986
:10399000084A315500230134BC42C4DBFEBD00BFE0
:1039A000FFFF0F009AFFFF7F381100202800002042
:1039B00098FFFF7FA0860100F7B503680133044636
:1039C0000D46174616D10D480D4D019002218DF878
:1039D000001002AC14E9030005F1080282E80300BC
:1039E0002868012120F0E2F8A95D206800F004FCBD
:1039F000013600E00026BE42F6DBFEBD9AFFFF7FE7
:103A00003811002010B5064C2368002B04DAFFF7AC
:103A1000C1FE002802DD2060012010BD002010BD85
:103A2000280000200068013018BF012070474FF0C7
:103A3000FF3303607047000003060BD44209064BB6
:103A4000012100F01F0011FA00F053F82210084382
:103A500043F82200704700BFB405002002060CD4D2
:103A60004209064B012100F01F0011FA00F053F843
:103A7000221021EA000043F822007047B40500201C
:103A800001060CD400F01F030649400901229A40A8
:103A900051F820301A420CBF00200120704700204E
:103AA000704700BFB405002038B504460138C3B2E2
:103AB000032B0D4628D811F0B3FB30B32046FFF797
:103AC000DFFF10B3114B124A187812F8201021B101
:103AD00010481FF08DFD002038BD93F800E093F8EA
:103AE00000C0187802F82E4002EB8C02411C558071
:103AF00001F01F021A7011F093FB074908220223FC
:103B00000CF0EEFA012038BD002038BD440600203C
:103B1000C4050020FF9403081D3B00082DE9F04771
:103B2000284FDFF8ACA03E783A7839780AEB860463
:103B300005461AF82660B4F80290481C00F01F03EE
:103B40003B70002430460AF82240FFF799FFB84640
:103B5000574620B328461C491C4A0AF079FF2846DC
:103B60004FF0FF3132460AF073FF28464FF0FF3125
:103B70000AF0C0FC48B1284649460AF050FE2846E3
:103B8000012122460BF01AF904E028464FF0FF31DC
:103B90000AF022FC28464FF0FF310AF01DFC0020FD
:103BA00009F06EFF98F800C017F82C10044621B9F0
:103BB00028460A460B460CF093FA2046BDE8F0472B
:103BC00009F05EBFB0050020F0D8FFFFA93A000859
:103BD000C4050020034B00221A605A609A60DA6024
:103BE000704700BFB405002008B5FFF7F3FF054894
:103BF000054B00210170054819708022BDE808407E
:103C00001FF082BB44060020B0050020C405002040
:103C10000138C3B2032B9ABF024B53F82000002097
:103C2000704700BFA00500202DE9F04F394B53F835
:103C3000206085B004460F469346002E63D0DFF81F
:103C4000E8A05AF82010D146A9B94FEA86084046A4
:103C500001911FF001FA4AF824000546019938B98C
:103C60002D4801682D48C9681EF096FA28464DE097
:103C700042461FF049FB06F1FF3A4FEA8A020392DF
:103C800038460A2120F09EFA054618B9384620F039
:103C9000A3FE3D18BD4202D8BBF1010F2CD138461E
:103CA000E91B20F0BDFF804638B91B491C480B6852
:103CB000D9681EF071FA404628E01A4F57F82400E0
:103CC000B04210D159F82430194651F8040B029330
:103CD00001911FF0C9F9029A01991046039A1FF049
:103CE000B5FA47F824A057F8243059F82420581C76
:103CF00042F8238047F82400297831B168786F1C96
:103D00000028BDD101E0304600E0012005B0BDE84B
:103D1000F08F00BFD8950308640000203C9503088D
:103D2000819503084806002050060020F0B585B0B4
:103D30001F4606460D46144620F04EFEC71902E007
:103D40000135013C013F4F2FFAD800E0013C231818
:103D5000502BFBD8184A1021684620F0CBF8684653
:103D600020F03AFE01466846FDF76CFA304620F036
:103D700033FE01463046FDF765FA28462146FDF739
:103D800061FA10210D4A684620F0B4F8684620F028
:103D900023FE01466846FDF755FA1021084A3B46C6
:103DA000684620F0A7F8684620F016FE01466846EF
:103DB000FDF748FA05B0F0BDC4950308C99503089E
:103DC000CE9503082DE9F8430E4B0F4F53F82050C2
:103DD000044699468DB1A846002604E058F8040B25
:103DE0001FF042F9013657F824008642F6DB2846D8
:103DF0001FF03AF9002149F82410002247F8242046
:103E0000BDE8F88350060020480600202DE9F04F59
:103E10000E46A84987B01F4651F8203005928246C9
:103E2000ABB9A54C25683846A9681EF0B5F92068DD
:103E300080681DF053FE22680599526830461DF0D7
:103E40004BFF00280CBF4FF0FF35002540E13846FE
:103E500020F0C2FD059B04904FF000085C1E9749BE
:103E600086F80080012250460394FFF7DDFE3846B5
:103E70000499FDF7E7F94546444603E04FF0000892
:103E800000E0D8460120FDF781FAA0F58071814657
:103E9000132900F2C78001A252F821F0693F0008FF
:103EA000693F00084B3F00085F3F0008FB3F0008E8
:103EB0000F4000082540000825400008ED3E00089E
:103EC00025400008213F000825400008ED3E00087D
:103ED0002540000825400008ED3E0008853E00080A
:103EE0000B4000081F400008DB3F0008744A75497A
:103EF00052F82A00431E51F82A0042F82A3050F89E
:103F000023001FF0B1F840F20F12914500F0C2807B
:103F1000B9F5867F00F0DA806A1C40F0BD80D7E0FA
:103F2000002CAFD0002DADD004F1FF392A1B311980
:103F3000013D06EB09001FF089F9002373554C463B
:103F4000384631462A464B4606E0002C9AD0013CC2
:103F5000384631462A462346FFF7E8FE92E7AC4250
:103F600000F081800134F3E7554951F82A30012BE4
:103F700088DD544803F1FF3B50F82A10C8EB0B02D0
:103F800051F822000191009202931FF06DF8304623
:103F900020F0FAFA009B0199B9F5807F14BF4FF029
:103FA000FF320122904441F82300B8F1FF3F029B09
:103FB0003FF464AF9845BFF664AFC8EB0B0B039AB0
:103FC00051F82B10304620F0F1FD039D002474556C
:103FD000304620F001FD04463FE0002D3FF452AF93
:103FE000AC42BFF44FAF013D621CB11830192A1B1F
:103FF0001FF02CF900237355AAE7384631462A46AC
:104000000023FFF793FE00243CE700253570384677
:1040100031462A462B46FFF789FE2C4632E700211F
:1040200031551AE028490A68131893F801C01CF0AA
:10403000970F3FF427AF039B9D42BFF423AFA542E8
:1040400013D1049A6C1CC0B27055A51800214F2DD5
:10405000315502D8FDF7DCF805E0384631462246F6
:104060002346FFF763FE25460CE704F1010B2A1BEC
:104070003119013506EB0B001FF0E8F8002006F8B7
:104080000490314670552A4638465B46FFF74EFE8F
:104090005C46F7E66FF001050A201FF05BFAAB1CE7
:1040A0003FF4D5AE002D13DD735D8BB10022725548
:1040B0000EE000BFD8950308640000202B720308AF
:1040C0004806002050060020600000204FF0FF3519
:1040D000284607B0BDE8F08F0022FFF7A5BD00001D
:1040E0001B4A52F820302DE9F04104461BB3194F0A
:1040F00057F820301BB3184A52F820009046F0B110
:10410000084616491DF082FF0646E0B1002508E08A
:1041100057F82430124953F8252030461DF090FFFF
:10412000013558F824108D42F2DB30461DF08AFB31
:104130000020BDE8F0816FF00100BDE8F0816FF074
:104140000200BDE8F0814FF0FF30BDE8F08100BF14
:10415000D895030850060020480600200A9003085E
:1041600014A60308052801D808F09EBA4FF0FF30C6
:10417000704705288CBF0020012070472DE9F74FBC
:1041800014461D46884654EA0501814609D0194B5C
:104190004FF0FF3284EA020685EA030756EA070178
:1041A00004D103B0BDE8F04FFFF7DCBF404600216B
:1041B00000220023FDF738FC82468B4600220023B4
:1041C0004846FFF7CFFF061E10DA00220023012128
:1041D0004046FDF729FC5B46CDE9000152464046CA
:1041E000FDF7E0FBA04271EB0503E7D3304603B0D7
:1041F000BDE8F08FFFFF0F00052801D808F040BA96
:10420000704700207047CF2801D808F06DBA002011
:1042100070470000014B00221A70704769060020A9
:10422000014B1878704700BF6906002008B50222CC
:1042300003204FF4006108F095F8054B1A7810B18F
:1042400042F0030201E002F0FD021A70187808BD86
:104250002D00002003204FF48061012208F082B875
:1042600003204FF48061002208F07CB80146012051
:1042700008F06CB908B50120FF2108F067F9C0B259
:1042800008BD000013B503204FF40061024608F09A
:1042900069F84FF480610422032008F063F8FFF707
:1042A000DFFF08220120002301920146074A009304
:1042B00008F0B4F8FFF7D4FF0A24FFF7DBFF013C56
:1042C000FBD1034B012018701CBD00BF801A0600F3
:1042D0006906002000000000F7B500234FF480704D
:1042E00001210022FDF7A0FB134DC5E90001FFF7F6
:1042F000C1FFFFF7BFFFFF28044617D000220023AD
:1043000001214FF48070D5E90067FDF78DFB32463F
:10431000CDE900013B464FF48070FDF743FB04A359
:10432000D3E90023824273EB0106E2D22046FEBDB0
:104330001FA107000000000060060020AFF300800E
:1043400010B50446FFF796FF207010BD0000000076
:104350002DE9F743002304460D464FF480700121F8
:104360000022FDF761FB1C4EC6E90001FFF782FF4A
:10437000FF2818D10022002301214FF48070D6E9D4
:104380000089FDF751FB4246CDE900014B464FF451
:104390008070FDF707FB0EA3D3E90023824273EB85
:1043A0000107E3D211E0FE280FD120462646FFF791
:1043B000C7FF701C0234FFF7C3FF023DF5D1FFF7C2
:1043C00059FFFFF757FF012000E00020BDE8FE8302
:1043D0009F8601000000000058060020AFF3008017
:1043E00038B504460D46FFF777FFFF2828D1204651
:1043F000FFF73CFF280EFFF739FF290CC8B2FFF783
:1044000035FF280AC0B2FFF731FFE8B2FFF72EFFF1
:10441000402C04D0482C0CBF8720002000E09520C1
:10442000FFF724FF4C2C01D1FFF724FF0A24FFF7EC
:1044300021FF030605D5013CE4B2002CF7D138BDBD
:10444000FF2038BD38B504460D46FFF745FFFF286D
:1044500020D12846FFF70AFFFD2D1DD00025605D05
:10446000FFF704FF631902355878FFF7FFFEB5F533
:10447000007FF4D1FF20FFF7F9FEFF20FFF7F6FEE3
:10448000FFF7F8FE00F01F01A1F10502504240EBDA
:10449000020038BD002038BD012038BD00000000FA
:1044A0002DE9F04385B0002840F00D81FFF7BEFEF6
:1044B000894B1A7812F0020F1F4601D0187803E1D9
:1044C000FFF7E0FEFFF7C6FE40200021FFF788FF60
:1044D0000128054640F0CD80002200234FF4807073
:1044E0002946FDF7A1FA7D4CC4E9000148204FF4AC
:1044F000D571FFF775FF0128264664D10025FFF727
:10450000B9FE03AB58550135042DF8D19DF80E00C6
:10451000012840F0AE809DF80F10AA2940F0A98034
:1045200077200021FFF75CFF012805D869204FF0B4
:104530008041FFF755FFB8B10022002301214FF45D
:104540008070D6E90089FDF76FFA4246CDE9000197
:104550004B464FF48070FDF725FA5DA3D3E90023A5
:10456000824273EB0105DBD20022002301214FF4CC
:104570008070D4E90045FDF757FA2246CDE90001E5
:104580002B464FF48070FDF70DFA51A3D3E90023B9
:10459000824273EB010E6CD37A200021FFF720FFDB
:1045A000002866D10446FFF765FE03AD28550134A7
:1045B000042CF8D19DF80C2002F04004002C0CBF14
:1045C0000225062556E077200021FFF709FF012884
:1045D00007D869200021FFF703FF01288CBF0125C0
:1045E0000225022D07D177200021FFF7F9FE0128CF
:1045F00006D8692000E041200021FFF7F1FEB8B1A4
:104600000022002301214FF48070D6E90089FDF7D4
:104610000BFA4246CDE900014B464FF48070FDF79E
:10462000C1F92BA3D3E90023824273EB010ED8D248
:104630000022002301214FF48070D4E90089FDF7A6
:10464000F3F94246CDE900014B464FF48070FDF787
:10465000A9F91FA3D3E90023824273EB010408D315
:1046600050204FF40071FFF7BBFE002818BF002553
:1046700000E000251A4B1B4C1D70FFF7F1FDFFF702
:10468000F9FD23780BB1581E20709DB13A7802F0E5
:10469000FE063E70FCF7EBFF134A46080821012096
:1046A00000230191964238BF32460146009307F03D
:1046B000B5FE01E0FFF7AEFD237813B1002D3FF406
:1046C000FFAE387800E0012005B0BDE8F08300BF00
:1046D0003F420F00000000002D000020580600207F
:1046E000680600202C00002020BCBE00AFF3008034
:1046F00008B520B9FFF79AFD024B187808BD0120D4
:1047000008BD00BF2D00002070B50C4616461D46A2
:1047100000283CD1002B3AD0FFF788FD1E480378D3
:10472000D80736D41D4A1178490758BF7602FFF7DB
:1047300091FD012D0ED151203146FFF751FEF0B908
:1047400020464FF40071FFF703FED0F1010538BF9A
:10475000002514E052203146FFF742FE78B920468A
:104760004FF40071FFF7F4FD28B1013DEDB204F5FF
:104770000074002DF3D14C200021FFF731FEFFF72C
:104780006FFDFFF777FD281C18BF012070BD0420C6
:1047900070BD032070BD00BF2D0000206806002002
:1047A000F8B50C4615461E4600284BD1002B49D0C3
:1047B000FFF73CFD264B1A78D00745D41B785907E4
:1047C00044D4244F3878420758BF6D02FFF742FDAA
:1047D000012E0DD158202946FFF702FE50BBFE21C5
:1047E0002046FFF72FFED0F1010638BF002621E05A
:1047F00039788B0707D500217720FFF7F1FD572087
:104800003146FFF7EDFD59202946FFF7E9FD88B94C
:104810002046FC21FFF716FE28B1013EF6B204F552
:104820000074002EF4D10020FD21FFF70BFE0028BC
:1048300008BF0126FFF714FDFFF71CFD301C18BF51
:104840000120F8BD0420F8BD0320F8BD0220F8BD0A
:104850002D000020680600207FB50D461446064650
:10486000002840F09880FFF7E1FC042D17D1237851
:10487000012B0CD003D3022B40F092800AE0FFF70B
:10488000CFFC002800F08980FFF7C4FC05E0FFF7AB
:10489000F9FC02E0FFF7C4FC6070354680E0424856
:1048A0000378DB077BD4FFF7D5FC0D2D6DD8DFE84F
:1048B00005F04607416C6C6C6C6C6C6C6C4D4F5D1C
:1048C00049200021FFF78CFD054600285BD1684692
:1048D0001021FFF73DFD002855D09DF800209DF8E0
:1048E00008309109012907D19DF809001902421CDD
:1048F000501883B29B021BE09DF807209DF806002C
:10490000910001EB931300F0030291029DF8050062
:104910009DF80A2001335B189DF8091000F00F0E76
:104920000EEBD21C01F003000CEB4002D11F8B40B8
:1049300023602BE04FF400752580002526E0FFF76B
:10494000CBFCB0F1FF0518BF01251FE0492000E0B6
:104950004A200021FFF744FDA8B910212046FFF7A7
:10496000F7FCD0F1010538BF00250FE07A200021C7
:10497000FFF736FD48B90546FFF77CFC6055013569
:10498000042DF9D102E0012500E00425FFF768FCC1
:10499000FFF770FC04E0042502E0054600E0032573
:1049A000284604B070BD00BF2D00002000487047AD
:1049B000C05CC53608B5084601F058FD08BD10B505
:1049C0000C4608681EF050FB60681EF04DFB204648
:1049D0001EF04AFB002010BD10B588B091E8110010
:1049E00013491F2306916946079301F011FDC0B9D1
:1049F0009DF80930BBB10699087808B90DF1090195
:104A00009DF80820C2F3001020731E22094820F0F0
:104A1000CDF80849009B61602360BDF80620A260C4
:104A200002E0002400E01C46204608B010BD00BF94
:104A30004C0700200811002070B508200E461EF01B
:104A40000BFB044618B300230360436024201EF0D0
:104A500003FB0546206070B110201EF0FDFA606077
:104A600048B128460EB1317809B90A4900E031460B
:104A700001F098FC58B1206808B11EF0F5FA6068A2
:104A800008B11EF0F1FA20461EF0EEFA002420468E
:104A900070BD00BF287203080D4810B52424012BF7
:104AA00004FB010004D0022B04D073B9144603E0C8
:104AB000846800E0C4681419214601F0E6FB002870
:104AC0000CBF20464FF0FF3010BD4FF0FF3010BD3F
:104AD0006C06002037B504460848242505FB010074
:104AE00011461A4601AB01F017FA20B105232360E5
:104AF0004FF0FF3000E001983EBD00BF6C06002083
:104B000037B504460848242505FB010011461A461E
:104B100001AB01F0A4FA20B1052323604FF0FF3070
:104B200000E001983EBD00BF6C06002038B5094D7D
:104B3000242404FB0155284601F0A0FB2246284608
:104B400000211EF0E1FB044B1868421E1A60002091
:104B500038BD00BF6C060020FC0600202DE9F8439C
:104B6000384F98463B68042B04460D46164602D142
:104B70001721016026E0DFF8D490002089F80000BA
:104B800008462F211FF01EFB18B948462E491FF07A
:104B9000F5FA2E4829461FF0F1FA06F4C062B2F584
:104BA000C06F26F4803301D1B2070ED103F4206622
:104BB000B6F5206F0BD013F400720AD1022B09D97D
:104BC000162323604FF0FF3639E0082202E000226E
:104BD00000E0102213F0030302D142F0010208E0CA
:104BE000012B02D142F0020203E0022BE8D142F095
:104BF0000302174D15492846D2B201F0DBF808B17F
:104C00000223DEE718F0080F1CBFEC68AC6000233D
:104C10001E46104C1D592DB101362433042EF8D1F7
:104C20004FF0FF360A4D242202FB06440FCD0FC47D
:104C30000FCD0FC4396828684B1C20603B6030469C
:104C4000BDE8F883FC060020287203082407002032
:104C5000000700206C060020074908B5002001F07D
:104C600099F8014628B90548054ABDE8084008F00A
:104C700025BF6FF0060008BD6C07002008960308EA
:104C8000E095030810B5002302E0CC5CC454013366
:104C90009342FAD110BD01E000F8011B12F1FF327E
:104CA000FAD2704710F8013B0BB18B42FAD118468B
:104CB0007047002302461846410841EAC01CD15CF7
:104CC000013351FA8CF00B2BC0B2F5D17047F8B517
:104CD00003690D4601F10902002B51D043691F7B86
:104CE000114600241E5D202E0A4613D0052E14BF47
:104CF0003246E5223E0707D5A2F1410C5FFA8CF659
:104D0000192E01D82032D2B201F8012B0134082C1F
:104D10000A46E7D11C7A202C18D02E2201F8012B4C
:104D200008269C5D202C0A4610D0FA0608D5A4F16E
:104D300041025FFA82FCBCF1190F01D82034E4B2C1
:104D400001F8014B01360B2E0A46EAD1DE7A2E72AB
:104D50009C7F93F81FC01E7F210441EA0C615C7F99
:104D600041EA060C4CEA04262E60597E93F818C0DE
:104D70004CEA0124AC80DE7D9B7D43EA0621E9807C
:104D800000241470AE69F6B10369ABB1028C4FF622
:104D9000FF739A4215D0C76909E0002101F04CFC6D
:104DA00060B1EA69511E8C420ADA3055013437F895
:104DB000020B0028F1D104E01C4602E0044600E0AA
:104DC000002400203055F8BD2DE9F041C56A8D4220
:104DD00004460E462AD00379E3B100F1300841467B
:104DE00040782A460123FFF7DBFC10BBA269216A49
:104DF0002071501885420DD2E77809E0A3696078E8
:104E0000ED1841462A460123FFF7CAFC013FFFB2D5
:104E1000012FF3D886B1607804F1300132460123C6
:104E2000FFF772FC58B9E662BDE8F0810020BDE8EA
:104E3000F0810120BDE8F0813046BDE8F08101201D
:104E4000BDE8F08110B504460A46407804F130010F
:104E50000123FFF759FC002832D194F82FC294F8AF
:104E60002EE2194B4EEA0C210AB29A422AD194F84A
:104E7000683094F869E094F866C01A0442EA0E615A
:104E800094F8672041EA0C0141EA022323F07F42B3
:104E90000E4B9A4217D094F8842094F885C094F869
:104EA0008200110441EA0C6E94F883204EEA000C53
:104EB0004CEA022121F07F40C01A18BF012010BD2A
:104EC000032010BD022010BD55AAFFFF464154002B
:104ED00070B500210446FFF777FF054600284FD143
:104EE0002378032B44D16079002841D004F13006A7
:104EF000304629464FF40072E562FFF7CCFEAA2344
:104F000084F82F326123552284F8323084F8173226
:104F1000236984F82E2252204122722184F8300025
:104F200084F8310084F83320180A84F8141284F8C5
:104F3000151284F81622190E1A0C84F81832E36838
:104F400084F8190284F81A22180A1A0C84F81B1221
:104F5000190E84F81C3284F81D0284F81E2284F88D
:104F60001F126078626931460123FFF719FC6571F1
:104F7000002160780A46FFF76FFC003018BF01205F
:104F800070BD08B560B1037853B1C2888A4209D1B7
:104F90004078FFF7ADFB10F0010018BF032008BDFB
:104FA000092008BD092008BD01292DE9F041054669
:104FB0000C465AD9C369994257D20378066A022B24
:104FC00028D0032B36D0012B52D101EB510706EB31
:104FD0005721FFF7F9FE00284AD1FA05D10D6818CC
:104FE000013790F8308006EB57212846FFF7ECFE9A
:104FF00000283DD1F805C70DEF1997F8303048EA81
:105000000320E30702D50009BDE8F0810105080D82
:10501000BDE8F08106EB1121FFF7D6FE40BB240668
:1050200005EBD45595F8312095F830C04CEA0220B4
:10503000BDE8F08106EBD111FFF7C6FEE0B96406CA
:1050400005EBD45595F8323095F8332095F83000BB
:10505000190441EA026848EA000E95F831804EEAE8
:10506000082323F07040BDE8F0810120BDE8F08105
:105070004FF0FF30BDE8F0814FF0FF30BDE8F08128
:1050800001292DE9F04104460D4616466AD9C36947
:1050900099426AD20378076A022B3CD0032B48D08E
:1050A000012B5AD101EB510807EB5821FFF78CFE79
:1050B000002853D14FEAC850C30D15F00105F2B2D4
:1050C00006D0E11891F8300000F00F0141EA021219
:1050D000E31808F1010883F83020012222712046EC
:1050E00007EB5821FFF770FEC0BB4FEAC8514FEAEB
:1050F000D1580DB1360909E004EB0802330A92F8E1
:10510000301003F00F0621F00F02164304EB0803E2
:1051100083F8306022E007EB1121FFF755FEE8B974
:105120002D0604EBD55585F83060360A85F83160D8
:1051300014E007EBD111FFF747FE78B96B0604EBDB
:10514000D355320A310C85F83060360E85F831209F
:1051500085F8321085F8336000E0022001212171CA
:10516000BDE8F0810220BDE8F0810220BDE8F081B9
:105170002DE9F0410546D0F81C800E4629B9C768D4
:105180005FB1474528BF012708E0FFF70DFF012861
:1051900030D9404539D3374600E001273C46013439
:1051A000444502D3012F28D9022428462146FFF77F
:1051B000FBFE30B1411C28D0012826D0BC42EED1E4
:1051C0001BE0284621466FF07042FFF759FFB8B93F
:1051D0002EB1284631462246FFF752FF80B92B698F
:1051E000EC605A1C10D0581E012328616B712046B8
:1051F000BDE8F0810120BDE8F0810020BDE8F0812C
:105200004FF0FF30BDE8F0812046BDE8F081012974
:1052100070B504460E4620D9C36999421DD217E0E5
:1052200020463146FFF7C0FE0546C8B1012814D01C
:10523000013014D0204631460022FFF721FF78B913
:105240002369581C03D0591C0120216160712E462E
:10525000E2699642E4D3002070BD022070BD0120B7
:1052600070BDC2690239931E994205D290F802C0FE
:10527000806A0CFB010070470020704770B50D4636
:10528000C18081680129044638D00368DA699142F7
:1052900034D271B91878032801D1596A49B900226A
:1052A000E2601989A94229D9586A00EB15132361D4
:1052B00019E09E7836010DE02068FFF775FE431C6B
:1052C000014619D0012819D92368DA69904217D20A
:1052D000AD1BADB2B542EFD2E1602068FFF7C1FF70
:1052E00000EB15112161226805F00F0358013032DF
:1052F00015186561002070BD012070BD022070BDD1
:10530000022070BD2DE9F0410F46C1884E1CB6B297
:105310000446002E69D00369002B66D0320759D1AC
:10532000C16801330361006819B90089B0425CD9D2
:1053300050E083785A1E12EA16134BD1FFF734FE61
:105340000128054657D9013058D02068C1698D42DF
:105350003AD3002F49D0E168FFF70AFF054600283D
:1053600046D0012847D0013048D020680021FFF7FF
:105370002BFD0746002841D12068394630304FF4D4
:105380000072FFF788FCD4F8008029464046FFF7FA
:1053900068FFC8F82C0010E04FF0010883F8048083
:1053A00020680021FFF710FD00282AD12368DA6A5F
:1053B000474402EB0800D862FFB223689978B942EB
:1053C000EAD8D86AC71BDF62E56020682946FFF784
:1053D00048FF20612368E68006F00F023033560153
:1053E0009E1966610020BDE8F0810420BDE8F081CF
:1053F0000720BDE8F0810220BDE8F0810120BDE872
:10540000F0814046BDE8F0812DE9F84F00210546C6
:10541000FFF734FF8046002840F08C80FF2634469A
:1054200028682969FFF7D0FC8046002840F0828078
:105430006F693B78002B7BD0E52BFA7A6ED002F0B7
:105440003F02110702D50F2A68D101E00F2A4ED181
:10545000D5F81CB0BBF1000F61D0580605D5EA881D
:105460007E7B2A8403F0BF0401E0A34256D17B7BFC
:10547000B34253D13A7802F0BF0808F1FF300D2152
:1054800001FB00F84FF001094FF0000A2C491AF80F
:105490000130F81817F803E090F801C04EEA0C202C
:1054A000B9F1000F0ED001F0E5F8B8F11D0F8146FB
:1054B00034DC3BF8180001F0DDF881452ED108F10D
:1054C000010803E04FF6FF72904227D10AF1010A6A
:1054D000BAF10D0FDAD197F800C05FEA4C612CD514
:1054E000B9F1000F29D03BF8183033B316E024B9D6
:1054F0003846FFF7DEFB86421CD04FF0FF31AA6929
:105500002984D07A10F0010302D007E00B2B11D0D0
:1055100017F803E0D05C01338645F7D0FF24284616
:105520000021FFF7EFFE804600283FF479AF01E04D
:105530004FF004084046BDE8F88F013CE4B2EEE7C6
:105540009D9603082DE9F04F0B782F2B85B006466A
:105550000F4601D05C2B00D101370024B4603B78AA
:105560001F2B05D830462146FFF788FE746112E1F3
:10557000F0690025029080468146785D6B1C1F28EB
:1055800003931AD92F281AD05C2818D01F2B00F0AB
:10559000FF80012101F050F80446002800F0F88057
:1055A0007F2806D87D482146FFF77CFB002840F085
:1055B000EF8029F8024B039DDFE7042400E000247C
:1055C000029A02EB450306E033F8022D202A01D0AF
:1055D0002E2A03D1013D002DF6D1D9E0029B0021F6
:1055E00023F815100B22B0692021FFF754FB4FF070
:1055F000000A01E00AF1010A38F8023B202BF9D039
:105600002E2BF7D0BAF1000F01D044F0030402981A
:1056100000EB450306E0013D04D14FF0000B0823E9
:10562000D94605E033F8028DB8F12E0FF3D1F4E737
:10563000029A32F81A80B8F1000F5ED0B8F1200F4C
:105640000AF1010A04D0B8F12E0F04D1AA4502D004
:1056500044F00304ECE79B4501DAAA4512D10B2B79
:1056600002D144F0030448E0AA4502D044F0030408
:1056700043DC4FEA89015FFA81F9AA460B234FF018
:10568000080BD5E7B8F17F0F10D9404600210193F0
:1056900000F0D2FF019B804618B1414A101810F863
:1056A000808C44F00204B8F1000F06D03D4801930D
:1056B0004146FFF7F7FA019B20B144F003044FF095
:1056C0005F0814E0A8F1410081B2192902D849F01D
:1056D00002090CE0A8F1610E1FFA8EFCBCF1190F53
:1056E00005D8A8F1200249F001091FFA82F8B16932
:1056F00001F80B800BF1010B9AE7B2691078E528ED
:1057000001D105211170082B04BF4FEA89095FFA06
:1057100089F909F00C030C2B04D009F0030CBCF13F
:10572000030F01D144F00204A2070AD409F00309CF
:10573000B9F1010F08BF44F01004042B08BF44F076
:105740000804B069C4723046FFF75EFEB169CA7AD8
:1057500002F00403DBB228B104281CD1002B08BFDF
:10576000052018E0BBB9736993F80BE05FEACE60DF
:1057700010D5597D187DDA7E93F81AC0039D40EA52
:1057800001284CEA02297F1949EA0845B560EFE68D
:10579000062000E0052005B0BDE8F08F8D960308D7
:1057A0000D960308969603082DE9F041FF2605465D
:1057B0003446042765E02868FFF706FB0746002803
:1057C00063D168690378002B67D0E52BC27A51D08A
:1057D0002E2B4FD002F03F02110702D50F2A49D1DC
:1057E00001E00F2A3CD15F0605D5EA88467B2A8472
:1057F00003F0BF0401E0A3423CD1437BB34239D163
:1058000090F80080EF6908F03F02531E0D214B43D2
:105810004FF0010E0022224912F801C000EB0C01EA
:1058200010F80CC091F801804CEA0821BEF1000F7D
:1058300006D01D2B1EDC27F813108E46013303E023
:105840004FF6FF7C614515D101320D2AE3D1007876
:1058500041061FD51D2B0DDC002227F8132019E06F
:105860001CB9FFF726FA864211D04FF0FF3EA5F88B
:1058700020E00CE0FF2428460021FFF743FD074607
:1058800018B92969002996D10FB100232B61384638
:10589000BDE8F081013CE4B2EDE70427F5E700BF85
:1058A0009D96030873B51E4614460B220546FFF766
:1058B000E9F9052E0AD97208218834F8023F42EA34
:1058C000C63011FA80F6B6B2002BF4D107230A21B4
:1058D000B6FBF1F001FB106630360DF8036086B2BE
:1058E000013B002EF3D10DF1080C0CEB03027E20DE
:1058F00002F8080C00E001369E4202DAA95D202978
:10590000F9D1072B07DC0DF1080E0EEB0300013374
:1059100010F8082C00E02022AA550136072EF0DDF1
:105920007CBD00002DE9FF418569C7690C22044652
:10593000294601A8FFF7A6F99DF80F30DB071CD513
:105940000020E8720126E061284601A93A46334664
:10595000FFF7A8FF2046FFF757FD804630B9013614
:10596000B6B2642EF0D14FF00708A8E0042840F04A
:10597000A6809DF80F10E972E7619DF80F2090074F
:1059800004D401270DE001339BB200E0002337F877
:1059900013000028F7D103F119010D2291FBF2F752
:1059A000BFB220460021FFF769FC8046002840F086
:1059B00086800646054620682169FFF705FA80467D
:1059C00000287CD163691B78E52B00D033B905B979
:1059D000E6880135ADB2BD4201D174E005462046EE
:1059E0000121FFF78FFC80460028E4D067E02046C5
:1059F0003146FFF743FC8046002860D1A069FFF7DD
:105A000058F90646681E85B220682169FFF7DCF95F
:105A10008046002853D16369D4F81CE05E730F21DF
:105A2000EAB20D27D972511E794318739876D87649
:105A30000746DFF8A8C04FF6FF78404517F80C80FE
:105A400018BF3EF8110003EB080C03F808004FEAFA
:105A5000102818BF01318CF8018001374FF6FF7C08
:105A6000002808BF60460D2FE3D1604502D03EF804
:105A7000110008B942F040021A70236801221A711D
:105A800020460021FFF73EFC8046C0B9013DADB283
:105A9000002DB9D119E06569414628462022FFF75B
:105AA000FAF82846A1690B22FFF7ECF8A36993F8EE
:105AB0000BC00CF018022A732068012101714046C6
:105AC00004B0BDE8F081012D91D120682169FFF774
:105AD0007BF980460028F2D1DDE700BF9D960308E0
:105AE000F8B5036815461A78303A092A07D85C7861
:105AF0003A2C04D102330360002A40F01F81A048F1
:105B000004680C60002C00F01B81217861B1607882
:105B1000FEF7EEFDC30707D4002D00F0138110F04F
:105B2000040018BF0A20F8BD002020706070FEF746
:105B3000B7FCC10700F1088115B1420700F10681E9
:105B400000212046FFF77EF9012818D194F8F221B0
:105B5000002A00F0FF8094F8F82194F8F93194F8C5
:105B6000F6E194F8F7C1110441EA036040EA0E0639
:105B700046EA0C2620463146FFF764F900E000268D
:105B8000032800F0E580002840F0E48094F83C1001
:105B900094F83BC04CEA0120B0F5007F40F0DC8077
:105BA00094F8477094F8465055EA07230ED194F8BC
:105BB000567094F8575094F8542094F8553039049E
:105BC00041EA056040EA020E4EEA032394F8405091
:105BD00094F83E2094F83F1094F8420094F841C0A5
:105BE00094F8447094F843E0A361E5706B4342EA93
:105BF000012194F83D5072184CEA00205EEA072714
:105C00002262A57020810ED194F8527094F853C08E
:105C10003F0447EA0C6E94F850704EEA070E94F871
:105C200051704EEA0727791A0009C3EB010CC0EB4B
:105C30000C0EBEFBF5F1023140F6F675A942E161AA
:105C400006D94FF6F675A94200F28880022500E0D9
:105C50000125991861621218D0184FF0FF332361A3
:105C60000023032DA06223715FD194F8610094F8A2
:105C700060E063714EEA002172186261607804F19D
:105C800030010123FEF740FD00284ED194F82F1279
:105C900094F82E023B4B40EA01220FFA82FC9C450D
:105CA00043D194F8323094F833E094F830001A0479
:105CB00042EA0E6194F83120334B41EA000C4CEA81
:105CC000022E9E4531D194F8162294F8173294F89A
:105CD00014E2100440EA036194F815222B4841EACB
:105CE0000E0C4CEA022181421FD194F81E1294F846
:105CF0001F2294F81CE20B0443EA026094F81D1280
:105D000094F81B2240EA0E0C94F81A024CEA012384
:105D1000E360010494F8183294F8190241EA026E23
:105D20004EEA030C4CEA00212161194A25701188C2
:105D300000204B1CE0621380E380F8BD0B20F8BD0F
:105D40000C20F8BD2846F8BD0320F8BD0A20F8BD98
:105D50000120F8BD0D20F8BD0D20F8BD94F85E506F
:105D600094F85FC0290494F85C5041EA0C6E94F8F2
:105D70005D104EEA050C4CEA0125656203256AE7D1
:105D8000DC09002055AAFFFF525261417272416145
:105D90009C09002048B9064A136803B1187009B17C
:105DA00000230B701160002070470B20704700BF6C
:105DB000DC0900202DE9F0418EB004460EA8002336
:105DC00002F01F0540F8341D236002A905F01E02F1
:105DD000FFF786FE002840F099804E480BA90891F5
:105DE0000990019902A8FFF7ADFB15F01C0F54D0E4
:105DF00060B1042840F08A8002A8FFF793FD0028D4
:105E000040F0848045F00805079E33E0690778D4A8
:105E1000079E002E79D0F27A12F0110375D12A076D
:105E200028D5F07E96F81A8096F815C096F814E0FA
:105E3000737548EA00214EEA0C2702983375B37651
:105E4000F37633777377B377F377012351EA074714
:105E50000371D0F82C8007D03946FFF7D8F9002815
:105E600054D1029A013FD76002984146FEF7ACFF39
:105E700000284BD12B071CD50023F372FEF796FDAB
:105E8000029BB073010AF173020C0121000E3274FF
:105E9000707445F0200519710BE0002836D1079E7B
:105EA000002E30D0F37AD8062DD4A90701D5DA0711
:105EB0002BD4029B0799D86A2162E061A57196F8FC
:105EC00015C0327DF07EB17E42EA0C2E41EA002CF4
:105ED0004CEA0E422261B07FF17F96F81CE002048A
:105EE00042EA0160727F236040EA0E0C4CEA022015
:105EF000E060FF210020A060E171A061DA88A2804B
:105F000004E0082002E0042000E007200EB0BDE815
:105F1000F08100BF9E0900202DE9F84F9946044604
:105F20000023C9F8003088460068A1881746FFF7AB
:105F300028F80546002840F08F80A379190600F163
:105F40008880DA0740F18780E668A068361AB74291
:105F500038BF3E467AE0A268D305D90D00294DD15D
:105F6000206894F807C081788C450CD30AB9206961
:105F700002E06169FFF718F801280BD9431C43D0F0
:105F800000226061E271D4F800B061695846FFF701
:105F900068F920B9A07960F07F05A57159E0E3792F
:105FA000770A00EB030A25D09BF802E09BF801007A
:105FB00007EB030CF44588BFC3EB0E07414652467E
:105FC000FBB2FEF7A1FBF8B921680B796BB1CA6A85
:105FD000CAEB020ABA4508D24FEA4A2A08EB0A007D
:105FE00030314FF40072FEF74DFEE0793918E1715F
:105FF0007F0221E05F1CC4F818A0E7712068A16946
:10600000A768FEF7E1FE30B194F806E06EF07F0578
:10601000A571012520E0A068FA05C105D70DCB0DBB
:106020002268C7F50077BE4238BF37463033D118F3
:1060300040463A46FEF726FEA268D019A060D9F87D
:106040000010CB19B844C9F80030F61B002E82D1DD
:1060500002E0022500E007252846BDE8F88F2DE97B
:10606000F84F9A4604460023CAF800308846006874
:10607000A1881746FEF785FF0546002840F0BB8043
:10608000A3791A0600F1B4809B0740F1B380E06861
:10609000C74228BF00279EE0A268D305D90D00297A
:1060A0006FD1206894F807C081788C4515D332B938
:1060B000216959B9FFF75CF80146206103E0616985
:1060C000FFF756F80146002900F08880012915D015
:1060D000481C5CD000226161E2712068A369C16A3A
:1060E000994204D10021FEF76FFE00284FD1D4F869
:1060F00000B061695846FFF7B4F820B9A07960F0A4
:106100007F05A57174E0E3797E0A00EB030927D0CF
:106110009BF802E09BF80100F218724588BFC3EBC0
:106120000E0641464A46F3B2FEF73AFB8346002884
:106130002DD12068C16AC9EB0109B1450BD24FEAE4
:106140004929303008EB09014FF40072FEF79AFD3F
:10615000236883F804B0E279B018E071760230E089
:10616000A168E368994207D358463146FEF72CFEF2
:1061700068B92668C6F82C90E279C4F81890501CCB
:10618000E0712068A169A668FEF71EFE28B1A1791A
:1061900061F07F05A57101252DE0A3682168F20556
:1061A000D805D60DC6F50076C20D3032B74238BFDD
:1061B0003E46881841463246FEF764FD23680120BA
:1061C0001871A2689319A360DAF800008119B0442D
:1061D000CAF80010BF1B002F7FF45EAFA368E2680F
:1061E000A079934240F0200188BFE360A17102E0F2
:1061F000022500E007252846BDE8F88F38B504469B
:106200000068A188FEF7BDFE002836D1A379990663
:1062100033D52068E169FEF7D7FD00282DD1256A26
:10622000E87A40F02001E972E2682A77A389180A27
:106230006877E189A977E27BEA772369AB76208AE0
:10624000010AE976628A2A75638A180A6875FEF778
:10625000ADFB010A020C030EE9752A76A8756B7670
:1062600094F806C020682CF020010122A17102716F
:106270002068BDE83840FEF72BBE38BD10B5044697
:10628000FFF7BCFF00B9206010BDF8B504460D460D
:106290000068A188FEF775FE064600287FD1A27926
:1062A00011067BD4E3689D4204D902F00202002A61
:1062B00008BF1D460021FF20A368E071A160002DEA
:1062C00059D0206887787F026BB1013B6A1EB2FB10
:1062D000F7FCB3FBF7FEF44505D378420340A36017
:1062E000ED1A61690AE0216939B9FEF741FF012819
:1062F000014636D0421C12D020616161002939D09C
:106300001EE0A2792068930704D5FEF731FF01460D
:1063100018B918E0FEF748FE0146481C05D1A179DE
:1063200061F07F06A671012639E0012919D920689C
:10633000C369994215D2A3686161DA19A260ED1BA5
:10634000BD42DED800E03D46A2686F0A5019ED0557
:10635000FFB2ED0DA060E7716DB12068FEF781FF1F
:1063600020B9A17961F07F06A67117E0C519013740
:10637000E77100E00D46A368DA05D00D18B1A169F8
:106380008D4218BFA561E068834208D994F806E001
:10639000E3604EF0200C84F806C000E00226304690
:1063A000F8BD000010B586B0044606A8002240F8EB
:1063B000141D2146FFF794FB30BB144B0199E36198
:1063C00003A8A0612046FFF7BDF8C0B963697BB19F
:1063D000DA7AD00617D5597D93F814C0DA7E93F88F
:1063E0001AE04CEA01204EEA022C4CEA0041A1607E
:1063F0002068C3880021A3802046FEF73FFF0428C1
:1064000008BF052000E0052006B010BD9E09002051
:106410007FB504460E460068A188FEF7B2FD05462A
:10642000F0B9114B01A8A061E36120461EB92946CD
:10643000FEF724FF13E0FFF7B7F9042801D1256127
:1064400000E060B920463146FEF741FC00212046BD
:10645000FEF758FF042802D10021216100E0054623
:10646000284604B070BD00BF9E0900202DE9F04F02
:1064700091B010AB04A943F8340D01221846FFF780
:106480002FFB82460446002840F0BD8069480DA9D4
:106490000A910B90039904A8FFF754F8824600284C
:1064A00000F0AF80042840F0AE8004982146FEF74B
:1064B0005FFE0546002800F0AA80012800F0AA80AF
:1064C000013000F0AA80ABE0049C29462046FEF78C
:1064D000C8FE04F1300731464FF400728146384659
:1064E000FEF7D9FB102620210B2238464FF02E0A4A
:1064F000FEF7D1FB84F83B6084F830A0FEF756FA33
:1065000083B21A0AA9B24FEA15480B0A84F846006A
:106510008DF8092084F847204FEA104B4FEA1822E3
:106520000646000E009084F8490084F84B308DF840
:106530000B2084F8452004F15000202284F848B054
:1065400084F84A5084F8448039468DF80A30019521
:10655000FEF798FB049A84F851A01078069B032854
:1065600003D1516A8B4208BF00231A0C190A100A82
:1065700084F86A3084F86B1084F8642084F865002D
:10658000002413E001230021C0F82C900371FEF7D2
:106590001BFC01468246002835D138464FF4007274
:1065A000FEF779FB013409F10109E4B2049882781D
:1065B000A242E7D804A8FFF7B5F9824620B10498B3
:1065C0002946FEF724FE1EE0099B9DF8090000996C
:1065D000D8759DF80B009DF80AC058751022DA7224
:1065E0000498019A597601219E7583F818B09A761D
:1065F00083F81BC083F814800171FEF769FC8246A2
:1066000001E04FF0080A504611B0BDE8F08F4FF09E
:10661000070AF8E74FF0020AF5E74FF0010AF2E740
:1066200004982146FEF7D0FB0646824600283FF438
:106630004BAFE8E79E0900207F2815D931B1FF282C
:1066400011D88038094B33F810007047084B33F8E5
:10665000022F824203D0013189B28029F7D101F1A2
:106660008000C0B270470020704700BFAA960308A0
:10667000A8960308064A002300E0013332F8021FFF
:1066800021B18842F9D1034A32F81300704700BFA4
:10669000A89703088A99030801604860704738B5D5
:1066A0000C4609680546FFF7F7FF20462946BDE876
:1066B0003840FFF7F1BF000038B5054610201CF048
:1066C000CBFC044650B91BF04DF803462046196830
:1066D00001F0D8FD054801F053FF04E01DB1AA68A0
:1066E0008260E968C160204638BD00BF6A9B03082C
:1066F00070B5074E346808E0256860682946FFF7E2
:10670000CBFF20461CF0B0FC2C46B442F4D170BD47
:10671000F409002008B50749074A096812680748C4
:106720001CF04EFE064B07481968BDE808401CF0F7
:1067300047BE00BFE8090020E00900207B9B03085A
:10674000400A00209E9B0308014B1868704700BF59
:10675000080A0020054B06481A68511C0268196097
:106760009142C8BF1A601868704700BF080A00202D
:10677000300A0020014B1860704700BF080A002053
:10678000014B1868704700BF300A0020014B187891
:10679000704700BF440A0020014B01221A70704765
:1067A000440A0020014B1878704700BF3C0A0020C3
:1067B000014B1870704700BF3C0A0020014B18784D
:1067C000704700BF040A0020014B01221A70704775
:1067D000040A002003490B6801309842C8BF00201A
:1067E000704700BF300A0020013844BF014B1868D1
:1067F000704700BF300A002008B50A4B0022194636
:1068000000E00132834202D01B688B42F9D132B1E1
:106810008B4204D1044801F0B3FE4FF0FF32104622
:1068200008BD00BF0C0A0020B09B030810B5144837
:10683000144A154C002303701370236853B913498D
:10684000134A4FF4FA400860124913600B601CF0C1
:1068500003FC206024685CB91AF084FF03462046DC
:10686000196801F00FFD0C4801F08AFE204610BDAA
:10687000064A2046002112681CF046FD012010BD8A
:10688000040A0020440A0020400A0020E8090020F1
:10689000340A0020E0090020C09B030808B50A481C
:1068A00003680021586802220B461DF087F9FFF7A4
:1068B000BDFF40B105480146FFF7EEFE0448014622
:1068C000FFF7EAFE012008BD640000200C0A00204A
:1068D000F40900205020704770B5194C194A2368FC
:1068E00083424FEA400515DA174909685E18AE423F
:1068F00005DB1168013383420968FBDB1BE0134BA6
:106900005B68136001E05B6801398142FBDC216058
:10691000136012E0AB4206DC116801E04968013BFC
:106920008342FBDC07E009490023116001E00968AC
:1069300001338342FBDB23601160106870BD00BF30
:10694000EC09002038000020300A00200C0A00204A
:1069500010B504460846FFF7BFFF01462046FFF783
:106960009EFE024B1868421C1A6010BD300A0020BF
:106970002DE9F74F814600200D460192FFF79CFE5E
:106980002A4604460A2148461CF076FB0546002CA0
:1069900032D020B91A4801F0F3FD28462DE0DFF887
:1069A00074A0DFF874B0DAF80060C9EB000815488D
:1069B000CBF80060036806EB08079F4204DB12482F
:1069C00001F0DEFD002018E0104A106849464246FA
:1069D00080191CF0C3FB20460199A660C4F80C8006
:1069E000CAF80070FFF7B4FF0949CBF800700B68D4
:1069F0005A1C0A60681C00E02046BDE8FE8F00BFFC
:106A0000E99B0308E8090020F79B0308400A0020DF
:106A1000080A0020E0090020340A0020F8B50446E6
:106A20000846FFF7D7FEFFF757FF06462046FFF759
:106A300053FF094F0446FFF75BFE09E02046FFF7CE
:106A40003BFE054638B13946FFF729FE24682F463C
:106A5000B442F3D10120F8BDF409002070B513E071
:106A6000084611F80C59012D17D11360836844684A
:106A70001D6807E02046266803F018F820461CF041
:106A8000F3FA3446AC42F5D10D4A0E48136800685B
:106A90000C24591E04FB0101144613F1FF33DFD20D
:106AA000094A0A4811680A4A016000232360094B19
:106AB00009491868094B10600A781A7070BD00BF48
:106AC0001C0A0020F0090020080A002030000020E5
:106AD00034000020300A00203C0A00202C0A00204C
:106AE00010B5094CFFF704FEFFF7B8FF206808B1A6
:106AF0001CF0BAFA05490648064A002303602360E1
:106B00000B601360012010BD400A0020340A0020F1
:106B1000E0090020E809002008B5FFF79FFF054ABB
:106B20000548064B4FF0FF311160002201601A70DA
:106B300008BD00BF34000020300000202C0A0020D7
:106B40002DE9F04F89B0544C03905448544A0368DF
:106B500021680093534B10781C680191002C02901F
:106B60009A4607DD504E3268002A03DB4F4D2968F4
:106B7000002904DA4E4801F003FD002089E00020DE
:106B8000FFF7AAFE04F1FF394A4C4FF00C0B2268C4
:106B90000BFB09F802EB080312F808C02746BCF10A
:106BA000030F2DD8DFE80CF00207111158689B681D
:106BB0004068196822E059684868FFF76DFD216850
:106BC00001EB08029068016818E009F1FF390BFB3E
:106BD00009FB5A44596850680968FFF75DFD23684E
:106BE00003EB080003EB0B01826889685068FFF72C
:106BF00053FD206800EB080358689968FFF74CFDC7
:106C00000C2101FB09FE206810F80E30B9F10109D2
:106C100083F0010400F80E40B6D5002213469446D6
:106C20001AE0D7F800B00BEB0C0898E807000DF15C
:106C3000140989E80700E41A0C214C43A3449BE89B
:106C4000070088E807003868041999E8070084E815
:106C5000070001330CF10C0CDAF80020541EB4EBE1
:106C6000430FDEDC039B0BB100F0A0FD30680B4A44
:106C7000296810600848009B01600F49029891F84C
:106C800000C03360019A064B08702A6083F800C088
:106C9000012009B0BDE8F08F300A0020080A00206A
:106CA0003C0A00201C0A0020300000203400002094
:106CB000099C0308F00900202C0A00207047704747
:106CC00073B50D46044616461AF04CFD00230360CA
:106CD00001A928460A221FF06DFB019B206006B126
:106CE0003360AB4201D1074805E01AF03BFD006874
:106CF000222805D1044801F043FC0020206000E078
:106D000001207CBD199C03082E9C0308F8B50B6874
:106D1000934204460D4622DAB2F5007F02DB571299
:106D2000BF0201E04FF40077206818B139461CF02B
:106D3000E7FC02E038461CF08FF9064658B91AF015
:106D400011FD01463046096801F09CFA054801F042
:106D500017FC3046F8BD2F6020600120F8BD0120EF
:106D6000F8BD00BF6A9B03081D4B98422DE9F04116
:106D700003D11C481CF03CFC0DE01B4A83681168E1
:106D8000994216460AD0194913600A68934205DBF6
:106D9000174801F0F5FB0020BDE8F081C568154CEF
:106DA00015496F1C20463A46FFF7B0FF804630B9C0
:106DB000124839461CF004FB4046BDE8F0811049FA
:106DC00037680A682068D1192A461CF0C7F9236879
:106DD000002058557F1937602068BDE8F08100BF5A
:106DE0000C0A00204C9C0308340A0020E80900200B
:106DF000729C0308280A0020E4090020829C0308F2
:106E0000400A0020F8B50B68934204460D4622DA8A
:106E1000B2F5007F02DB5712BF0201E04FF40077AA
:106E2000206818B139461CF06BFC02E038461CF0B3
:106E300013F9064658B91AF095FC01463046096820
:106E400001F020FA054801F09BFB3046F8BD2F60A9
:106E500020600120F8BD0120F8BD00BF6A9B030837
:106E6000F8B50B68934204460D4622DAB2F5007F6E
:106E700002DB5712BF0201E04FF40077206818B11F
:106E800039461CF03DFC02E038461CF0E5F80646A9
:106E900058B91AF067FC01463046096801F0F2F96A
:106EA000054801F06DFB3046F8BD2F6020600120E1
:106EB000F8BD0120F8BD00BF6A9B03082DE9F84F1B
:106EC000254D264C264F90462A680C2601328146D5
:106ED0008A46204639467243FFF7C2FF8346F8B917
:106EE0001AF040FC03465846196801F0CBF91D48DA
:106EF00001F046FB206860B3FFF7B0FD20681CF08E
:106F0000B3F81948194AC4F800B04FF0FF310160D6
:106F1000C5F800B0C7F800B011605846BDE8F88F5A
:106F20002F6822687E43404602F80690216801EBF4
:106F30000609FFF7D1FCC9F80800206800EB060835
:106F40005046FFF7C9FC2368C8F8040001379819B8
:106F50002F60BDE8F88F00BF1C0A0020F009002058
:106F6000240A00206A9B030830000020340000201F
:106F70002DE9F843154E3468B44205D1144801F0A8
:106F8000FFFA0020BDE8F883124D00272860204654
:106F9000FFF792FB8046B8B1296801F10109C5F8F5
:106FA0000090FFF7D5FC17B1C7F8088006E0384617
:106FB00049464A46FFF782FF074628B12468064B38
:106FC0000120B4421870E2D1BDE8F883F409002032
:106FD000AC9C0308080A00203C0A00202DE9F84F69
:106FE0000546084614460E469946FFF7F3FB6F1E0A
:106FF000BC42804601D0B4420AD14046FFF76CFC47
:1070000082463846FFF768FC284B80461E603FE00A
:10701000022039464246FFF751FF002843D0204660
:10702000FFF7D8FB214602460220FFF747FF002862
:1070300039D04046FFF750FCAC42834608DA384668
:10704000FFF74AFC07462046FFF746FC804607E06C
:107050002046FFF741FC80463846FFF73DFC0746D7
:10706000D8F800A039684046FFF716FBDBF80400AB
:107070005146FFF711FB38465946FFF70DFBAC426E
:1070800002DA751B013500E0002508486419046028
:10709000B9F1000F04D0D8F80000514600F0FAFB17
:1070A000034901200870BDE8F88F00BF080A0020DE
:1070B0003C0A00202DE9F84304460D461646FFF72A
:1070C000ADFC20B3012021462A46FFF7F7FEF0B1C0
:1070D0002846FFF77FFBFFF7FFFB671E8046384619
:1070E000FFF7FAFB81461EB10068414600F0D2FB73
:1070F00048464146FFF7D0FA06490748074B076064
:107100002A1B0D68D4432C1901200C601870BDE8AF
:10711000F88300BF300A0020080A00203C0A002043
:107120002DE9F84F0746084688469346FFF752FB7D
:10713000FFF7D2FB82463846FFF7CEFB0025044618
:1071400019E02046FFF710FE0646002839D0DFF888
:107150007C90E2681C494846AA18FFF7D7FD002832
:107160002FD0D9F80000E268401931461BF0F6FF35
:10717000E3682468ED185445E3D1144C124905F135
:10718000020920464A46FFF7C1FDD0B1104A2368E4
:107190001188384659535A464146FFF78BFF80B154
:1071A0000C4D20687A1E2A604946FFF7E1FB40B18A
:1071B000296800200A46FFF781FE10B10649012028
:1071C0000870BDE8F88F00BF200A0020380A0020B0
:1071D0006F940308080A00203C0A00202DE9F047BC
:1071E000804691460D46FFF777FBC8EB05041F4F1D
:1071F0000134C1450646C7F8009007DBA94505DA0A
:10720000C8EB0900441CC9EB050500E000254FF060
:10721000000826E03046FFF74FFA814620B3396870
:1072200001F1010AC7F800A0FFF792FBB8F1000FC7
:1072300002D0C8F8089006E0404651465246FFF793
:107240003DFE804680B10A4B366801221A7014F167
:10725000FF34DFD23968481CFFF73EFB2C46064658
:107260000025002CF3DC0120BDE8F087080A00208F
:107270003C0A00202DE9F3412B4B0025044616461D
:10728000019519609846BEB901A800F00BFD206079
:10729000002843D0019B23B1C11811F8010C0A2822
:1072A00016D02248036858681AF026FA019AD2F1DB
:1072B000010038BF002034E02368197800292FD05E
:1072C00000220192019A985C511C0A280191F9D17F
:1072D0000199022906D1236818782E2802D1023399
:1072E00023601DE02068D8F800200F4FFFF740FB17
:1072F000B8B125B13868FFF7EFFAA86006E0396841
:1073000028460A46FFF7DAFD054650B12168019B81
:10731000074AC818012120601170B4E7304600E028
:107320000120BDE8FC8100BF080A002064000020A5
:107330003C0A002038B50446002505E000EBC500F6
:10734000013540681BF090FEA36820689D42F5DB84
:1073500018B11BF089FE002121600022A26038BD17
:1073600008B11CF0CDB908461BF076BE70B50446D6
:1073700008460E461DF030FBE268811805460131D3
:107380006068FFF7EDFF50B1E16860606A1C40186B
:1073900031461DF00BFCE3685D19E560012070BD0E
:1073A0002DE9F041044610460D4616461DF014FB2B
:1073B0008046A068411CC9002068FFF7D1FFB0B12A
:1073C000A368206000EBC30740F83350002008F1A9
:1073D000010578602946FFF7C3FF40B131462A46D0
:1073E00078601DF0E3FBA1684A1CA2600120BDE8A3
:1073F000F08100002DE9F04F8FB098469DF8603085
:107400000691089300230129044604920360436017
:107410008360C36040F37481002A00F07181B8F189
:10742000000F00F06D8101250293019300E03D46BD
:10743000049951F825603378AF00002B00F01481D7
:107440002D2B727840F01081002A00F00D81069BF0
:107450006F1C9F42B4BF51F8273000232D2A40F003
:10746000C180B278002A00F01E814FF0000A01E0CE
:107470000AF1010A06EB0A0082780AB13D2AF7D127
:107480000B924FF0FF3100220A9703922746934652
:1074900005910993A94644462AE065682DB328461C
:1074A000B11C52461DF02EFBF8B928461DF094FA87
:1074B000504529D0059D6B1C12D0059907980C25C5
:1074C0004D4308EB050258F8053083420BD192F882
:1074D00008C00398227A944518BF0120039004E065
:1074E000CDF814B001E0012303930BF1010B0C3430
:1074F00025680795002DD0D13C46099B0A9FDDF8F1
:1075000014B0079A4D4604E03C46099B0A9F4D463D
:107510000122039959B152B97F492046FFF726FF4E
:1075200031462046FFF722FF20467C4987E0BBF129
:10753000FF3F0AD17A492046FFF718FF314620461F
:10754000FFF714FF2046774979E00B980C2202FBE5
:107550000BFB18B308EB0B052B7A53B97249204685
:10756000FFF704FF69682046FFF700FF20466F49D8
:1075700026E0012B0AD106EB0A01CB7833B96A4920
:107580002046FFF7F3FE2046696815E00AF1030E76
:10759000204658F80B1006EB0E021EE008EB0B0617
:1075A000307A012815D10BB11A7862B95E492046AC
:1075B000FFF7DCFE71682046FFF7D8FE5C492046E5
:1075C000FFF7D4FE4DE0AF1C204658F80B101A46CA
:1075D00003E058F80B10574A2046FFF7E1FE002859
:1075E0003FD18EE001279946F15D00238DF83410DC
:1075F0008DF8353051B1424604E0814203F10C026E
:1076000000F08280106813460028F6D120464A49CF
:1076100011E0013517461B7AD3B127B1F05DF2199D
:1076200008B120460FE0012B12D14B4620460BB18A
:107630001A783AB94149FFF799FE20460DA9FFF79C
:1076400095FE0DE04A46FFF7ABFE002861D158E0F9
:107650002046384AFFF7A4FE002852D0002FC3D19D
:107660002F466568DDB11EE0089981B9029E019838
:107670000136B100FFF774FE00283FD0049A019054
:10768000D359029F029640F827306F1C07E020462E
:1076900000213246FFF784FE002832D06F1C069886
:1076A0008742FFF6C4AE65680DB9019E0BE0204627
:1076B000FFF740FE1CE02046002156F8042BFFF7A0
:1076C0006FFEF0B1013502998D42F4DB3E46002594
:1076D0000BE0049B03EB870C20465CF8052000219F
:1076E000FFF75EFE0136043558B1069A9642F0DB8C
:1076F000019B2BB118461BF0B7FC01E0089800E095
:1077000001200FB0BDE8F08F0137F25D002A80D074
:1077100081E70135A4E700BFD79C0308BB9C0308A1
:10772000CA9C0308DE9C0308E09C0308EB9C03084A
:10773000079D03082B7203081E9D0308319D030853
:1077400010B50446FFF7F6FD606818B11BF08CFC1D
:10775000002363600020E06010BD406870478068CF
:10776000704738B50D1E044607DBFFF7F8FF85426A
:1077700005DA236853F8350038BD002038BD0020F5
:1077800038BD000038B50D1E044608DBFFF7E7FFE3
:10779000854206DA236803EBC505686838BD0248F0
:1077A00038BD014838BD00BF2B72030810B50A4C24
:1077B000FFF785FA206808B11BF056FC074A084914
:1077C000084800231360084A23600B6003601360BD
:1077D000BDE81040FFF772BA580A00204C0A00209A
:1077E000480A0020540A0020500A0020F0B50E4933
:1077F0000E480F4B0D6806681F6800222B46BB42DF
:107800001C4602DB0B600020F0BD06EB850C01334B
:107810005CF802C00432BCF1000FF0D0006850F8F0
:10782000240001340C60F0BD480A0020580A0020F2
:10783000540A0020F8B5134C134D0646FFF73FFAE3
:1078400020681249421C92002846FFF7DBFA0746DF
:1078500068B919F087FF03463846196800F012FD31
:107860000B4800F08DFEFFF729FA3846F8BDFFF708
:1078700025FA20682A68411C42F820602160012016
:10788000F8BD00BF540A0020580A0020500A00200A
:107890006A9B0308F0B50F4B0F4A1C681368164625
:1078A00010E00133A342A8BF002305EB830755F87E
:1078B00023C0844502D100223A6002E00132A24294
:1078C000EFDB0068884203D0044D00222D68F6E704
:1078D0003360F0BD540A00204C0A0020580A0020F2
:1078E0000346002001E080F00100013902D45A5C17
:1078F0005C2AF8D0704700002DE9F04F04468BB0A9
:1079000008469246FEF766FFFEF7E6FF0290204625
:10791000FEF7E2FF0746002C40F0B981904800F0E6
:107920002FFE2046B8E13846FFF71EFA054600282C
:1079300000F0B281611C20460391FEF71BFF894ACB
:10794000894C10685168D7F80CB004AE03C6107AA1
:10795000616830702068227A07AB03C31AF004060E
:107960001A7006D0FEF7F0FE014680481BF028FD95
:1079700008260195B94632E1019F17F8014B1AF02C
:10798000020F019713D12868826891684B1E93609B
:10799000002B826807DA976893699F4228DB10689A
:1079A0000470286806E1126814702B6813E100F077
:1079B000CDFD0136864205DD2E686D48B1681AF0AE
:1079C000EBFB0126A4F12007F9B25E2914D85C2C48
:1079D00012D02868674B81688A68551E8D60002D1B
:1079E000826807DA95689769BD4201DB1268DFE0BB
:1079F0002146E9E01268ECE0214604A81CF0E2FB15
:107A0000804628685B4B81688A68013A771C8A60E7
:107A1000002A826814DAD2F808E091698E450BDBFF
:107A200012685C20107018688268136819780A2937
:107A300003D0013313600BE05C2124F033FC07E03A
:107A400010685C2101701B6898680268511C016015
:107A5000002C39D0B8F1000F36D028684549866827
:107A6000B5686C1EB460002C826822DA9369946851
:107A70009C4204AB12DBC3EB08050DF1280C0CEBA8
:107A80000506126816F80C0C1070086882681368F6
:107A900019780A290AD0591C116013E0C3EB0804B5
:107AA0000DF1280E0EEB040313F80C1C24F0FAFB66
:107AB00008E0136898F80C401C700D68A868066808
:107AC000721C02603E468AE028682A4B81688A68F8
:107AD000571E03368F60002F826815DA9169976808
:107AE0008F424FEA94110BDB106830310170186837
:107AF0008268136819780A2903D0013313600CE0F7
:107B0000303124F0CFFB08E01268A1093031117048
:107B1000186881680F687A1C0A602868154B8168AC
:107B20008A68571E8F60002F826825DA91699768EE
:107B30008F424FEAD4010DDB126801F007003030AC
:107B4000107018688268136819780A2905D0013303
:107B500013601CE001F00701303124F0A3FB16E0B4
:107B6000B09B0308589D0308619D0308519D0308BD
:107B7000559D030864000020E008176800F0070125
:107B8000303139701A6897683868411C3960286844
:107B9000434B81688A68551E8D60002D826804F011
:107BA000070414DA95689769BD420BDB126830341C
:107BB000147018688268136819780A2904D05C1C4C
:107BC00014600CE004F1300124F06CFB07E0126853
:107BD000303414701B689B681968481C1860BBF12E
:107BE000010B2F4D7FF5C8AE4F4600F045FB002836
:107BF00026D11AF0020F23D02868826893685C1E91
:107C00009460002C826813DA91689469A1420BDBBE
:107C100012682420107028688268136819780A296D
:107C200003D0013313600BE0242124F03BFB07E079
:107C30001368242119702A6894682068411C216007
:107C40002868174B81688A68541E8C60002C8268F3
:107C500013DA946891698C420BDB12680A20107069
:107C600018688268136819780A2903D001331360F1
:107C70000BE00A2124F016FB07E014680A212170AA
:107C80001A6894682068411C21603F68039C029B2D
:107C90009F427FF448AE01200BB0BDE8F08F00BFDB
:107CA000640000202DE9F84305464FF0FF3800241A
:107CB00000E0A0460120F9F769FB0746013028D112
:107CC0003D4E3368586819F0F9FD074698B119F030
:107CD00049FD01463948096800F0D4FA384800F0F7
:107CE0004FFC3068406819F007FD002D60D000227D
:107CF0002A6015465CE03368586819F0FDFC44457D
:107D0000D7D1304B0CB11868075505B12C601D68F0
:107D10004EE02C4E2C493046A21CFEF7F7FFB14630
:107D200020B9002D44D02860054641E0FF2F31DD09
:107D3000B7F5857F13D1002CBCDD306800270755CF
:107D4000013C3368214820221A5531681BF038FB6A
:107D500031681F480F5531681BF032FBAAE740F22B
:107D600009118F4207D109201BF0F4FB376809265F
:107D70003E5501349EE7B7F5847F9BD115481BF033
:107D800037FC31680A2008550134336800221A553F
:107D90005DB90BE038461BF0DDFB36683755013422
:107DA000002F87D1FEF7F8FC84E72C60D9F800504B
:107DB0002846BDE8F88300BF64000020769D0308D4
:107DC0006A9D0308680A00205C0A00207C9D030865
:107DD000829D0308DAB003082DE9F34707460E46F3
:107DE00092460068002400E02C4610F80490651CC0
:107DF000B9F10A0FF8D1012D5AD02146FFF770FDD5
:107E0000002855D0DFF8BC802C4940462A46FEF7B2
:107E10007DFF00284FD0D8F8000039682A461BF0B3
:107E20009DF9D8F800301B1903F8019CBAF1000F36
:107E300000D0013C01A8FFF735FF054600283AD0E5
:107E4000019A2AB1801810F8019CB9F10A0F04D0E8
:107E50001B4800F095FB00202DE0DFF868801749F3
:107E60004046A218FEF752FF28B3D8F80020294652
:107E70001019019A1BF072F90199012904EB01050F
:107E80000ADDD8F800806C1E40462146FFF728FD29
:107E900010B108EB0403C7E70A4C084920466A1CE6
:107EA000FEF734FF38B121680020485523683B6055
:107EB00006B135600120BDE8FC8700BF6C0A0020D8
:107EC000869D0308640A00202DE9F04F037887B0EF
:107ED000212B0390884606D002F0BEFA75491AF0AD
:107EE00095F8064640B919F03DFC0146039809682B
:107EF00000F0C8F97048C6E04046FEF7EDFC834646
:107F0000FEF744FC0490FEF73BFC05904046FEF76C
:107F100031FC00252F46A946002468486849A21C68
:107F2000FEF7F4FE002800F0C0807268DFF88CA134
:107F3000501E0028706008DA624B314618681BF04A
:107F40009DFC0346013004D10DE0316811F8013B7E
:107F50003160DAF800000355013413B9FEF71CFC58
:107F6000DBE70A2BD9D1DAF80010544A0020085573
:107F7000591C20D130460292019319F09FFC029ABD
:107F8000019B60B19A4619F0EDFB02460020116892
:107F900000F078F94C4800F0F3FA504687E054B10D
:107FA00015680A21295513681D196870FEF7EEFB44
:107FB00000B901340125DAF800A0BAF1000F74D03D
:107FC00034B3FEF77CFE60190290FEF7BDFB029908
:107FD00002465046FEF7CCFC98B1DBF800B0B9F190
:107FE000000F02D0C9F808B00EE0FEF7ADFB8246E4
:107FF000FEF7AAFB514602464846FEF75FFF814660
:1080000010B9FEF75BFE50E03F19FEF757FE83E71D
:10801000059BC3EB0802544244EB0204B8F1000F85
:108020000AD04CB147B1049931B1FEF7C7FB18B182
:1080300024480368254807E04DB114B1FEF7A6FBBC
:1080400028B9204A22481368D9681AF0A5F8FEF723
:108050009DFB28B1049B1BB915B10CB9013706E093
:10806000002F08BF012514B10DB1FEF7ADFB30465E
:1080700019F0E8FB50B119F075FB01460398096847
:1080800000F000F9134800F07BFA0EE000F0F2F87F
:1080900030B90C4A104910683A46C06819F0D0FF50
:1080A000FEF752FBC8EB000001E04FF0FF3007B0D5
:1080B000BDE8F08F7BC903089D9D0308700A00206E
:1080C000600A002064000020B49D0308CB9D0308D3
:1080D000DD9D0308EF9D0308079E03082DE9F74F78
:1080E0001D4603780190212B0E46144606D002F05F
:1080F000B3F9314619F08AFF074640B919F032FB4F
:1081000001460198096800F0BDF83D485FE020464F
:10811000FEF7E2FB214606462A463A481BF050F994
:10812000A0464FF0000A36E03046FEF71DFE8346BB
:1081300020B9314634481BF043F934E0D6F80C90AE
:10814000FEF71EFB804505D1FEF720FB10B1FEF7C0
:1081500035FB20B90A200BF8090009F101094B464B
:1081600013E01BF8010B0093394619F0A9FF013009
:10817000009B0AD119F0F6FA02460020116800F0BF
:1081800081F8224800F0FCF90DE0013BE9D53668A2
:10819000CA4408F10108B8F1000F01D0A845C3DDB9
:1081A000BAF1000F07DA1A4821462A461BF008F9EF
:1081B0004FF0FF3021E0384619F044FB50B119F080
:1081C000D1FA03460198196800F05CF8114800F0F4
:1081D000D7F9EDE700F04EF830B90F480168524684
:1081E000C8680E4919F02CFF24B1AC4204DC2C1BEA
:1081F000601C02E0204600E00020BDE8FE8F00BFCA
:108200000C9E0308249E03083A9E0308679E0308F9
:10821000799E03089C9E030864000020079E0308C3
:1082200038B50D46034668B102785AB10B4C0C497B
:1082300020680C4AC06819F003FF23680A20D96837
:1082400019F03EFF4DB1054B074A19681268C8681E
:108250000649BDE8384019F0F3BE38BD640000207F
:1082600020B703083BCD0308740A0020309F0308A1
:108270000120704700207047014B1878704700BFFD
:10828000780A002038B50D460C490B780246A3B990
:108290000B4C30B1007820B123680A49D86819F036
:1082A000CFFE22682846D4681CF08AF906490246A7
:1082B0002046BDE8384019F0C3BE38BD7A0A002018
:1082C00064000020579F030814A6030800B591B06E
:1082D00001A920F037FB40B9029A02F47041A1F5E0
:1082E0000043584240EB030000E0012011B000BD04
:1082F00010B50C490B78044683B10278212A08D0C6
:1083000009491BF0D7FF20B120462F211BF05AFF4F
:1083100030B1064800F034F9002010BD012010BD36
:10832000012010BD790A00204DBF03085C9F03089F
:10833000F0B50D46A5B006466349644C782202A804
:108340001AF00CFF2868002320603146009320A813
:108350002A4602ABFFF74EF8014608B95C4808E030
:1083600020A8FFF7FAF9002857D020A8FFF7F5F961
:108370000121FFF755FFA1E0294620A8FFF7F1F9F9
:108380002946064620A8FFF7FDF9002E4CD06C2E9A
:1083900040D006DC562E29D0682E10D0472E33D17F
:1083A0000AE0722E18D002DC702E2DD111E0732E4F
:1083B00015D0762E28D116E00122464B11E0464911
:1083C00046481AF0FDFF464821681AF0F9FF454873
:1083D00016E001F053FB1EE00122434B01E0434B4A
:1083E00001221A7017E001F05BFB14E03A49404AA1
:1083F00040481AF0E5FF404840491AF0E1FF404884
:108400001BF0F6F800205CE03E480021FFF708FF73
:10841000032056E00127013501E00746054620A864
:10842000FFF79DF98542A7DB374900201AF092FD3E
:10843000FEF734FA002835D140E0294620A8FFF79E
:10844000A1F9324904461BF035FF20B92749012222
:108450000A70AD1826E02046FFF74AFF90B10021D0
:108460002046FFF731FD002803DA0020FFF72EFF3A
:1084700030BB94F800C0BCF1210F18D0204600F0AA
:1084800071F814E0224802682248D16819F084FE8D
:10849000237813B1204800F073F80020FFF716FF8F
:1084A00070B904E020A8FFF75AF98542C5DB20A87F
:1084B000FFF746F9384601F011FB02E0012000E029
:1084C000022025B0F0BD00BFB89E0308740A00204A
:1084D000749F0308780A0020A19F0308869F030861
:1084E000A89F0308C59F0308790A00207A0A002084
:1084F00030A2030829A2030834A2030889A20308B2
:108500008EA2030855A303082B7203082ECD03087F
:1085100064000020DDA5030876A3030810B5074B0F
:108520001B680246104612F8011B5C18647814F0B0
:10853000080F01D00A29F5D110BD00BF600000204E
:10854000014B1860704700BF3C000020014B1868C9
:10855000704700BF40000020014B1868704700BF03
:108560003C00002010B5054C01464FF480722046B7
:108570001CF01CFB002384F8FF3010BD900A002083
:1085800010B50649064C002818BF01465022204667
:108590001CF00CFB002384F84F3010BD2B72030835
:1085A000080C0020002808B504DD0348FFF7E8FFA9
:1085B000012008BD002008BDC1A3030808B5064A74
:1085C0001168081843781B0704D40448FFF7D8FF44
:1085D000012008BD002008BD60000020D4A30308CE
:1085E0002DE9F34704460020FEF774F9064620689B
:1085F000FFF794FF206003780A2B00F0F38002A9B4
:10860000002541F8085D204669460122FFF7E4FB9A
:10861000002800F01781236893F80090B9F1210F2A
:1086200040F0DB80581C2060FFF722FE08B187482D
:10863000DFE0204601A90122FFF7CEFB002800F071
:108640000181834E019A8349276830460132FEF743
:108650005DFBB046002800F0F580356885F8009095
:10866000012590E0212B42D1974212D0DFF8E09112
:1086700078496E1C48463246FEF748FB002800F059
:10868000E1802368D9F8001013F801CB01F805C088
:1086900056E0714E3368B1462BB1FFF7EDFD38B1AE
:1086A0003268507820B96D48FFF76AFF0025CAE0AC
:1086B0006B4F67483B686749EA18FEF727FB0028BD
:1086C00000F0C0803968336805E05E78D8F8007043
:1086D00013467E550135D9F800005A1C00EB010EF7
:1086E0007245F2D32768791C21602E464AE0252B7B
:1086F00028D15C48067826B95B48FFF741FF35462C
:10870000A1E001F0A9FE07461CF066F9844601903D
:1087100050494F4805EB0C02FEF7F8FA002800F02C
:1087200091802E4605E017F8015BD8F8002095559A
:108730000136019B581E0190002BF4D127687B1C49
:1087400023601FE0DFF80891424905F1020A48461C
:108750005246FEF7DBFA002874D02368D9F80020CF
:108760001E785655236819466E1C11F801EBBEF1B0
:108770005C0F216006D15878D9F800109D1C8855EF
:10878000256056463546226813780A2B7FF46AAF77
:1087900001E05A1C2260236818780A28F9D02E4C70
:1087A000324920466A1CFEF7B1FA00284AD0D8F8B0
:1087B000001020682A461AF0D1FC2368284A0021BC
:1087C00059553B781560212B01D0252B03D1256805
:1087D000681C1AF00DFF256835E00098B0420BDDEB
:1087E000234806E0FFF748FD30B91E490D781DB952
:1087F0001D48FFF7C5FE26E01E481F49721CFEF704
:1088000085FAF8B1002305E01068C15425686A1C98
:10881000013322602168174A09780A29F4D11068C7
:108820000025C55401E001332360236893F800C09C
:10883000BCF10A0FF7D01068FFF75AFD10B10D4ACE
:10884000156800E005462846BDE8FC875C9F0308E4
:10885000B80C0020040C0020900B0020EEA30308AD
:10886000800A0020900A002002A40308940B002034
:1088700016A40308880A0020840A00200148FFF794
:108880007FBE00BFB09B03082DE9F3470546FDF707
:108890005BFF7A4F7A4B386018600026984628684C
:1088A000FFF73CFE28608146FDF74EFF0123009054
:1088B00000E000232968DFF8DCA10C78DAF800205A
:1088C00010194278520709D5002B00F0AA8068469B
:1088D0002A46FEF7F5F90028EBD1C9E02C2C00F070
:1088E00088800FD8252C00F0848005D8202C16D045
:1088F000242C3CD0092C02E0272C60D02B2C40F0FB
:1089000087800CE02F2C3BD004D82D2C07D02E2CA8
:108910007ED12CE03B2C6CD03F2C79D130E0481C30
:108920002860FFF7FBFD28600146DAF80020007898
:10893000131893F801C05FEA4C700DD501A82A46C0
:10894000FEF7BEF9002800F093800199009B2D2CC2
:1089500008BF49425B1808E02B2C02D1009C631C25
:1089600003E02D2CA5D10098431E0093A1E7002B16
:1089700057D04A1C2E2C2A6046D1FDF7E5FE45E073
:1089800023B919463F481AF01BFD4AE0A4F12F0114
:10899000D1F1000E4EEB0101284601F05BFB0028EF
:1089A0000146009003DA38481AF00AFD60E02B68AF
:1089B0001878A0427FF47DAF01332B6079E7002B5C
:1089C0002FD0481C28604B78613B8A1C192B2A60E9
:1089D00005D92E48FFF7D4FD4FF0FF3004E02C49B5
:1089E00051F82300FDF708FF00280090BFF661AFA3
:1089F0003EE06BB14B1C01363B2C2B6002D1FDF7E6
:108A0000A3FE00E001203860FDF7BAFE009050E7B9
:108A1000494530D0009C002C03DBFDF7B1FE8442B9
:108A200002DDFFF72BFF23E00098013600280FDB63
:108A30002A6839681378C8F800102C2B386003D0E6
:108A40003B2B05D1FDF796FE2868441C2C6026E7D9
:108A5000012E02D03B68834202D03A68C8F8002059
:108A600010F1020F14BF30464FF0FF30BDE8FC8715
:108A70006FF00100ECE74FF0FF30E9E7980B0020C2
:108A8000580C002028A4030843A4030860A403088A
:108A90009C0B00206000002010B50B4B12B90B4A54
:108AA000186011601B68002B07DD08480468A342AA
:108AB00003DCFDF765FE844203DDFFF7DFFE0020E7
:108AC00010BD012010BD00BF580C0020980B0020E5
:108AD00038B50446FDF738FE0546FDF735FE22465B
:108AE00001462846BDE83840FFF7D6BF2DE9F843D8
:108AF000164E174DD6F800802F688946FFF7C4FE42
:108B0000041E1FDBFFF7B8FB30B12CB91148FFF78B
:108B100037FD2046BDE8F8832D680D4C002D03DBA2
:108B2000FDF72EFE854204DDFFF7A8FE0020BDE81C
:108B3000F8832368C6F80080C9F800302760012058
:108B4000BDE8F8830020BDE8F88300BF580C002082
:108B5000980B002077A4030808B5026813786C2BE3
:108B600003D10B6843F002030AE06E2B03D10A68BD
:108B700042F0040304E0702B07D10B6843F00803B4
:108B80000B6003685A1C0260E7E7511C0A2B016066
:108B900004D00348FFF7F4FC002008BD012008BD05
:108BA0008CA403082DE9F04387B04FF00009044678
:108BB00088461646CDF80890FFF766FE071EC0F2FD
:108BC00054862068FFF7AAFC0346206013F8015B77
:108BD000692D236000F0528239D8572D00F0C784E8
:108BE00024D8482D00F01D8216D8452D00F0CA80EB
:108BF00010D8232D00F0188607D80A2D00F0F7852D
:108C0000212D40F0188600F0DBBD3D2D40F013868D
:108C100000F0C4BD472D06E0502DC0F00C86512D4C
:108C200040F21083562D40F0068620E1652D00F0BD
:108C30009F8006D8632D4DD07CD8612D40F0FB85F8
:108C400033E0672D00F0138100F2EB81E8E0722D34
:108C500000F0238312D86D2D00F0C28205D86B2D51
:108C600000F04C8200F2788222E2702D00F07482D3
:108C700000F2E8826E2D40F0DE856DE2762D00F088
:108C8000F68005D8742D00F03C8400F25C8444E347
:108C9000782D00F0F184C0F06A84792D00F00B8506
:108CA0007A2D40F0C88500F035BD204602A9FFF7B7
:108CB00053FF002800F0DC850EB9FDF7CFFE964982
:108CC000204609683246FEF7D5FA002840F0B985FB
:108CD00000F0D1BD9148026880460AB901250560BF
:108CE0008D4D2B680BB9012129603846FFF7F0FE46
:108CF000002800F0C385204602A9FFF72DFF0028B9
:108D000000F0BF850EB9FDF7A9FED8F8000029686C
:108D10003246FEF7CFF9002800F0B685FDF714FDC6
:108D2000324601462046FEF7A5FA002840F0898524
:108D300000F0ADBD3846FFF7CBFE002800F0AA8555
:108D4000204602A9FFF708FF002800F0A6850EB90B
:108D5000FDF784FE704A7148116800683246FEF7DC
:108D6000A9F9002800F09C85FDF7F4FC00F069BD2E
:108D7000FDF718FD30B1FFF77DFA18B918F1030FB0
:108D800040F091853846FFF70DFC002840F08E85B5
:108D900023681878FFF712FC002840F08A852046E7
:108DA000FFF71EFC0446002800F08685FDF7E8FC6E
:108DB000324601460120FEF77DF9002800F07F854C
:108DC000FDF78EFE002800F07D85FDF72FFD0028C1
:108DD00000F07B85237823B1212B02D02046FFF7BA
:108DE000C1FBFFF749FA58B1217849B94C480278DC
:108DF00032B94C48FFF7C4FB6FF0010000F030BE01
:108E00002178474B002914BF204618460021FFF760
:108E10005BF80028C0F25C85FDF77EFE002079E259
:108E20003846FFF7BFFB002840F0558522681078D0
:108E3000FFF7C4FB002840F051852046FFF7D0FB28
:108E4000002800F04E850378212B06D13648FFF725
:108E500097FB6FF0010000F003BE0BB1FFF782FB40
:108E60002F4801F0F9FA1AF0C3FB00F0EABC36B162
:108E70002E48FFF785FB6FF0010000F0F1BD672D74
:108E800006D0A5F1470CDCF1000141EB0C0300E03A
:108E900001230493FDF774FC3A4601460120FFF7D5
:108EA000FBFD002800F020851C4A1B4B11681A6846
:108EB0009DF81030204600F0D9FF002800F01785FB
:108EC000472D06D0A5F15605D5F1000E4EEB050550
:108ED00000E00125049535B1204602A9FFF73CFECC
:108EE000002800F007859DF81060029F8EB9FFF7FB
:108EF000C3F920B120680E491BF0DCF9D0B1002184
:108F000020460A46FEF768FF002800F0F684256830
:108F100011E000250FE000BF980B0020580C002046
:108F2000900A002002A40308A6A40308BAA4030818
:108F30006F9403089A4DFDF791FDFEF757FC00284A
:108F400000F07F84FDF758FCFDF714FCFDF7FCFBF7
:108F50000028C0F2D584002E54D0FDF7F5FB8046E2
:108F6000FDF7F2FB3A4601464046FEF7C5FC0028F5
:108F700000F0C98405A8FEF795FE2060002800F0E7
:108F8000C584059B002B40F37485C21812F8011CA0
:108F90000A29EFD100F06DBD8248FFF7F1FA6FF0BA
:108FA000010000F05DBD012B05D17F491BF082F966
:108FB0000028C2D00DE0022B0BD17C491BF07AF9BE
:108FC00038B9FDB97A48FFF7DBFA6FF0010000F01D
:108FD00047BD204605A90022FEF7FEFE002800F04E
:108FE0009884744D059B744928465A1CFDF78EFEE3
:108FF000002800F09184059A2868216801321AF04F
:10900000ADF82D68256007E0002101222046FFF71A
:10901000C9FD0028C0F28384216808780028F3D1B4
:109020008BE73846FFF7BEFA002840F07B842046E5
:1090300002A9FFF791FD002800F07784482D0AD19E
:109040005E4B93F800E0DEF1010C38BF4FF0000CEE
:1090500083F800C001E0682D04D058480278002A47
:1090600000F0EF83564A1178002900F0EA83554852
:1090700055490368D86818F0E3FFE2E3534D2A68C6
:109080000AB901212960204602A9FFF765FD0028E1
:1090900000F04E840EB9FDF7E1FC2B682046591E06
:1090A0003246FEF7E7F8002840F0CB8300F043BCDF
:1090B000FDF74AFB0546FDF747FB3A46411C2846AB
:1090C000FFF7EAFC002800F03984204602A9FFF7E8
:1090D00043FD002800F035840EB9FDF7BFFC3C4885
:1090E0003A4A00681168884200F0AB833246FEF7C6
:1090F00017F8002840F0A58300F026BC334D4378D4
:109100002D680493811C21602DB9FFF7B7FB6FF028
:10911000010000F0A5BC204602A9FFF71DFD0028B4
:1091200000F015842846FDF7D7FB049B613B192B03
:1091300006D92848FFF724FA6FF0010000F090BC30
:10914000254A52F8234011461CB9244A14680134B8
:10915000146041F8230074E36C2D01D1022304E074
:109160006E2D01D1042300E0082338460493FFF755
:10917000AFFC002800F0EE83204602A9FFF7ECFCCC
:10918000002800F0EA8312481049029B049A006804
:1091900009681A43FEF7B0FB002840F0FC82DFE3C9
:1091A000A3A40308869D03086F940308D6A40308AC
:1091B000EEA30308B00C0020BC0C00207C0A0020A9
:1091C000080C00206400002014A60308980B00205F
:1091D000580C002060A403089C0B0020B40C002055
:1091E0003846FFF775FC002800F0BD83204603A930
:1091F000FFF77CFC002800F0B983984D039B2A6898
:1092000093420ADB964801688B4206DA9548FFF7DD
:10921000B7F96FF0010000F023BC204602A9FFF768
:109220009BFC002800F0A5830EB9FDF717FC8C4BC2
:1092300028681968039A3346FDF7D0FE002840F0ED
:10924000008399E33846FFF7ADF9002840F0978393
:10925000204602A9FFF780FC002800F09383502DE0
:109260000AD1814991F800E0DEF1010C38BF4FF0DE
:10927000000C81F800C0E4E2FDF794FA40B1FEF77B
:10928000F9FF28B9712D03D118F1030F40F07D8348
:10929000FDF726FC4FF0FF30E2E34078FFF78EF950
:1092A000002840F075831FB9FDF76AFA6C4A106018
:1092B0002046FFF795F90446002800F06C830EB9AC
:1092C000FDF7CCFB694D287828B92378212B02D0F3
:1092D0002046FFF747F9FEF7CFFF48B1217839B9AB
:1092E0002A782AB96248FFF74BF96FF00100B7E31B
:1092F00094F800C05A4B5D481968BCF1000F18BFC4
:109300002046FEF7E1FD00280390C0F2478300F0FD
:1093100098820120FDF74CFA93E24D46554A2168A8
:1093200010680B78C21892F801E05FEA4E720ED511
:1093300051482246FDF7C4FC002800F032834F4B11
:10934000186820F0100145F0080519601FE0702B27
:109350000ED004D80A2B05D0672B11D105E0722B53
:109360000ED108E045F0080511E045F0010504E0E4
:1093700045F0020501E045F004054A1C226006E0C4
:109380005DB13F48FFF7FCF86FF0010068E325B1DD
:10939000236819780A29C1D165E3002505E0394819
:1093A000FFF7EEF86FF001005AE315F0010802D064
:1093B000314A00201060236819780A290AD093F8EE
:1093C00001C0BCF10A0F05D12F48FFF7D9F86FF0A3
:1093D000010045E30DB168070FD5204600F072FE8D
:1093E000002800F0E18245B920462449224A33464C
:1093F00000F088FD002800F0E982DFF88090D9F8BD
:10940000003016B143F0010301E023F00103C9F875
:109410000030B8F1000F05D0D9F8000080F010033B
:10942000C9F80030A90707D5D9F8003083F0080142
:1094300021F00602C9F80020206803786E2B08D0BE
:10944000702B23D06C2B2AD1D9F8002042F00203D4
:1094500020E0D9F8001041F004031BE0580C002074
:10946000980B0020D9A403087B0A0020900A002052
:1094700002A4030860000020AC0C00208C0A00202D
:109480008CA40308EDA4030806A50308D9F800304E
:1094900043F00803C9F800302268501C20603846A9
:1094A000FFF716FB002800F09482204602A9FFF780
:1094B00053FB002800F090820EB9FDF7CFFA8948DF
:1094C00089498A4B009600680968D9F800201B6812
:1094D000874C00F015FE002800F08182226812F00F
:1094E0000E0F00F0AE81FDF72FF90546FDF72CF9C0
:1094F000226801462846FEF7FFF9002840F0A181C6
:1095000070E23846FFF7E4FA002800F06E82204649
:1095100003A9FFF7EBFA002800F06A82204602A9AF
:10952000FFF71AFB002800F066820EB9FDF796FAE5
:109530006C496D4B0868039A1968FDF74FFE0028C7
:1095400040F07F815AE23846FFF72CF8002840F0BF
:109550005882204602A9FFF7FFFA002800F0548243
:109560003046FDF7EDFA002840F06B814FE243787A
:10957000712B049301D0512B01D10230206022685D
:109580001078FFF71BF828B15A48FEF7F9FF6FF083
:10959000010065E22046FFF723F8044628B9564843
:1095A000FEF7EEFF6FF001005AE23FB9FDF7E8F871
:1095B00020B94D4B4B4E1F6037600DE0FDF7E0F8D2
:1095C0003A4601460120FFF767FA28B94B48FEF7F3
:1095D000D7FF6FF0010043E2494E317829B9207876
:1095E000212802D02046FEF7BDFFFEF745FE48B118
:1095F00022783AB933782BB94248FEF7C1FF6FF0B1
:1096000001002DE221783E483F4B364A002918BF21
:109610002046354C3D491268572D08BF194623682E
:10962000FEF75CFD00280446039005DA3848FEF793
:10963000A7FF6FF0010013E2FDF7A2F8844203D107
:109640000020FDF7B5F80CE0FDF7ACF848B1FEF7E7
:1096500011FE30B9049A712A03D118F1030F40F0BA
:10966000D981049B712B02D0512B40F0EA80FDF789
:1096700037FA4FF0FF30F3E11B4D2B68002B04DB72
:10968000FDF77EF82968884204DAFFF7F7F86FF0F3
:109690000100E5E1204602A9FFF75EFA002800F08C
:1096A000BC810EB9FDF7DAF92868FDF761FC0028E6
:1096B00040F0C780B4E13846FFF70AFA002800F00E
:1096C000B281204602A9FFF747FA002800F0AE81D8
:1096D0000448054A00681168FDF7A0F9002840F029
:1096E000B080A6E1580C0020980B0020AC0C0020A4
:1096F0008C0A002020A503083BA5030850A50308F9
:10970000900A002002A40308B8B4030829AD030896
:1097100066A50308A64B01251D60FDF715F88046D8
:10972000FEF7AAFD18B9D6F1010538BF00250120C2
:1097300008EB05013A46FFF7AFF9002800F07C81FD
:10974000216808783138C2B2082A09D804A822460C
:10975000FDF7B6FA002800F072810498FEF7F0FEDB
:10976000204602A9FFF7F8F9002800F06B81FDF709
:1097700007F8904C0546FEF7EFFE246821188D424D
:1097800002DAFCF7FDFF01462046029AFEF7B4F824
:10979000002800F05A810021029152E0204602A9DF
:1097A000FFF7DAF9002800F0538117B1814B1968EF
:1097B00002E0FCF7E5FF01467F4819F001FE40E0BA
:1097C0007E487B4C19F014FF7A4A216812687C4865
:1097D00019F0F6FD042019F03FFC044619F044FC92
:1097E0002146784819F0ECFDFCF794FF29E0704D14
:1097F00001242C60FCF7A8FF0546FEF73DFD18B9D3
:10980000D6F1010438BF0024012029193A46FFF798
:1098100043F9002800F01F816648006800220146D5
:10982000FEF76AF868B919E1236813F8011B0A29E1
:109830002360F9D105E06448FEF7A2FE6FF0010055
:109840000EE10298002800F00B81FCF77DFF044632
:10985000FCF77AFF029A01462046FEF74DF80028F1
:109860000CBF6FF001000020FAE06FF00100F7E09C
:109870006FF00100F4E06FF00100F1E06FF0010023
:10988000EEE06FF00100EBE06FF00100E8E06FF058
:109890000100E5E06FF00100E2E06FF00100DFE0C1
:1098A0006FF00100DCE06FF00200D9E06FF0010022
:1098B000D6E06FF00100D3E06FF00100D0E06FF070
:1098C0000100CDE06FF00100CAE06FF00300C7E0D7
:1098D0006FF00100C4E06FF00100C1E06FF0010023
:1098E000BEE06FF00100BBE06FF00100B8E06FF088
:1098F0000100B5E06FF00100B2E06FF00100AFE0F1
:109900006FF00100ACE06FF00100A9E06FF0010022
:10991000A6E06FF00100A3E06FF00100A0E06FF09F
:1099200001009DE06FF001009AE06FF0010097E008
:109930006FF0010094E06FF0010091E06FF0010022
:109940008EE06FF001008BE06FF0010088E06FF0B7
:10995000010085E06FF0010082E06FF001007FE020
:109960006FF001007CE06FF0010079E06FF0010022
:1099700076E06FF0010073E06FF0010070E06FF0CF
:1099800001006DE06FF001006AE06FF0020067E037
:109990006FF0010064E06FF0010061E06FF0010022
:1099A0005EE06FF001005BE06FF0010058E000BF87
:1099B000580C0020980B00208FA7030874A50308FB
:1099C0009DA50308BBA50308CCA503086FF0010003
:1099D00046E06FF0010043E06FF0010040E06FF0FF
:1099E00001003DE06FF001003AE06FF0010037E068
:1099F0006FF0010034E06FF0010031E06FF0010022
:109A00002EE06FF001002BE06FF0010028E06FF016
:109A1000010025E06FF0020022E06FF001001FE07E
:109A20006FF001001CE06FF0010019E06FF0010021
:109A300016E06FF0010013E06FF0010010E06FF02E
:109A400001000DE06FF001000AE06FF0010007E097
:109A50006FF0010004E06FF0010001E06FF0010021
:109A600007B0BDE8F08300F0F9F900287FF49DAC61
:109A700095E4002B7FF497AAFFF78EBA10B5014644
:109A8000054C064801220270204650221BF08EF839
:109A9000002384F84F3010BD5C0C00207B0A0020AE
:109AA000014B01221A7070477C0A002030B5094929
:109AB000094A0B6802F1680407E052F8045B85422A
:109AC00003D1002542F8045C013B0BB1A242F4D162
:109AD0000B6030BDB40C00209C0B002030B587B06B
:109AE0000023019003930493FDF7E9F85F481AF00F
:109AF00057F8044610B9FDF7E1F80AE05C48016840
:109B00005C48C96818F048FB5B48FEF739FD4FF028
:109B1000FF34574D2A68906817F0E0FF002C0CDAEC
:109B200056490B784BB12A685549D068554A18F008
:109B300087FA2868C06817F0D1FF53490B7843B102
:109B40005248534919F03CFC494A1068806817F0A4
:109B5000C5FF05A8FEF7A6F80290002840D0059B97
:109B600033BBFCF71FFE00283AD0FEF783FB054607
:109B7000002835D13E4C47482368D96818F00CFBC3
:109B80004548FEF7FDFC2846FEF7A0FB58B13B48D0
:109B90000178002964D02368049AD8683F49394B7A
:109BA00018F04EFA5CE0FCF703FE6FF00204B0E739
:109BB000C11811F8012C0A2A05D03948FEF7E0FC3B
:109BC0006FF00104A5E7049B581C0490214602A8ED
:109BD0000022FEF7E7FF044600289AD0421C01D17C
:109BE000039840E0C31C09D1214D2A482A68D16856
:109BF00018F0D2FA2848FEF7C3FC1BE0043013D15A
:109C00001E48017800292DD00020FEF75FFB18B117
:109C1000174B049A1B6816E015490A681849D06862
:109C2000184A18F00DFA1DE0114D1A482B68D96832
:109C300018F0B2FA0020FEF749FB50B10F4A107835
:109C400080B1049A2B68D86814490E4B18F0F8F9C3
:109C500008E0019D002D7FF45CAF0121039158E7DE
:109C6000022000E0012007B030BD00BF48100020F6
:109C700064000020DCA50308E0A503087C0A00209E
:109C800014A60308080C00207B0A002030CB030830
:109C90005C0C0020DDA50308EAA5030803A6030861
:109CA000869D030810B505E010F8014B944208BFEB
:109CB00000F8013C0139F7D510BD0A220023FFF757
:109CC000F1BF00220A23FFF7EDBF00002DE9F041AC
:109CD00002681378202B94B0074601D154484CE019
:109CE0000A2B08D0561C066052780A2A03D09A42E2
:109CF00001D0344646E04F4C236813B94E48FEF776
:109D00003FFC206891E05B2A2DD162785E2A01D069
:109D1000013400E0023420785D281DD11BE05B2A6D
:109D200019D16578A5F12E02D1B20F2913D8434875
:109D30004FFA82FC10FA0CF10DD5224612F8020FF0
:109D400002E00A290DD00846144612F8011B5D29CD
:109D5000F7D1A842F7D1013422785D2A11D00A2A1E
:109D6000DDD1374809E05C2A0BD194F801E0BEF15F
:109D70000A0F01D0013404E03248FEF701FC002054
:109D800053E0013422789A4201D00A2ABBD12E4DE9
:109D90002E49A61B2846721CFCF7B8FF002844D0A9
:109DA00032462868396819F0D9F92B6800229A558B
:109DB0003C60FCF7EBFC18B128683146FFF781FFE7
:109DC000D5F80080B8F1000F2ED01A4D296811B1D6
:109DD0001F4A107890B14FF4067019F03DF904460F
:109DE000286058B917F0BEFC034620461968FEF7F4
:109DF00049FA1848FEF7C4FB204616E0144E2868BE
:109E00000027377041460B4E00F08CFF50B11249CD
:109E100068461AF03FFB6846FEF7B2FB306819F05F
:109E200023F93760286800E0404614B0BDE8F081AF
:109E300006A50308E80C002018A603080000098006
:109E40002CA6030845A60308EC0C0020C80C002033
:109E5000E00C00206A9B03085CA60308024B18680C
:109E6000003018BF01207047D40C00202DE9F743C3
:109E70001F46036893F80090B9F1200F04460E4680
:109E8000904602D0B9F10A0F04D11D48FEF778FBC5
:109E9000002033E0FFF71AFF054600282ED0236884
:109EA0001A784A4501D1581C2060FDF77FFC3046E6
:109EB000FCF712FD04461EE02046FCF755FF8146E4
:109EC000E0B1FCF763FC18B14846E168FFF7F9FE22
:109ED0000022494628461346009200F025FFD0F1A3
:109EE000010138BF0021B94203D12046FDF7A2FC91
:109EF00020B1246801364645DEDD0120BDE8FE8341
:109F000006A503082DE9F04F85B0002701930368EB
:109F100093F800A01760BAF10A0F04460D46934665
:109F20000F6004D1464A08201760086084E0036887
:109F300003971E4616F8019B06605978414E252965
:109F400048D193F802C0CC4544D19A1C02603368D2
:109F500013B93D48FEF714FB30684FE0DFF8E480AA
:109F60003A49B71C40463A46FCF7D0FE002864D078
:109F70002268D8F80000134613F8011B8155701CA5
:109F80000A29236003D1577837BB226029E05C2976
:109F900022D113F801EBD8F80010BEF10A0F01F836
:109FA00000E0236016D1019B2BB113E02848026822
:109FB000506817F0A1FB03A8FDF774FE206000288D
:109FC0003BD0039B002BF1D004DDC31813F8011C18
:109FD0000A29EBD13E4600E00646226817784F4535
:109FE000BCD1184F19493846721CFCF78FFE20B3BC
:109FF0003968134B0020885538681E60E8B1236823
:10A000001A780A2A01D1082315E0524501D15A1CB9
:10A01000226021680B78A3F1310C5FFA8CF00828DC
:10A0200004D858462246FCF74BFE06E0672B03D1C6
:10A030000131216010232B60012005B0BDE8F08FB5
:10A04000C00C0020CC0C0020EDA40308D00C002094
:10A05000640000202DE9F3410E46FFF737FE054668
:10A06000FCF772FB044635B3204616B1FCF7B2FB91
:10A0700001E0FCF7B9FB0446B0B1FCF72DFC8046CB
:10A08000FCF772FE0746B0B1FCF780FB20B1384602
:10A09000D8F80C10FFF715FE002228463946134663
:10A0A000009200F041FE40B1FCF74EFB8442DBD150
:10A0B0000348FEF765FA4FF0FF342046BDE8FC8107
:10A0C00068A6030838B50446FCF7F9FD2046FFF7FB
:10A0D000FDFD044650B1084D2868844206D008B101
:10A0E00018F0C2FF054B2C6001221A70FCF7E6FD48
:10A0F000201C18BF012038BDD40C0020E00C00202B
:10A100002DE9F04FAFB00C919DF8E01008900138A8
:10A11000079209930D91FCF72DFB00220492069201
:10A1200080E1FCF717FBFCF7D7FB0446FCF71CFEAD
:10A130000646002800F08A81FCF728FB18B130465B
:10A14000E168FFF7BEFDE46800230A94974C009392
:10A150002068314610220EAB00F0E6FD002840F0EA
:10A160005E8135468246074604460596099B0E9E4B
:10A1700023B10AF1010A534540F096800EB1761BD7
:10A1800001E04FF0FF368A4F8A4904EB0608384653
:10A190004246FCF7BBFDB946002800F057813B68FA
:10A1A00029461819324618F0D9FF804982480A68B2
:10A1B000D2F8087244460B97834607685CE03B7808
:10A1C000262B1CD10E980F9A7A49C5EB000808EB94
:10A1D000020377480393A218FCF798FD039B00281D
:10A1E00000F03481264607E015F80840D9F8001041
:10A1F00008F101088C5501369845F5DB3AE05C2BF7
:10A2000027D17B78302B07F1010823D9392B21D8AE
:10A210000B9F303BBB421DDC0EAF07EBC30057F872
:10A220003310426862484F1BBB1862490393A2185F
:10A23000FCF76CFD039B002800F00881264605E032
:10A24000EC5DD9F800200137945501369F42F7DBC9
:10A250000FE0B846564F5749661C38463246FCF761
:10A2600055FD002800F0F28098F800C0386800F82A
:10A2700004C0474601373446504ADBF800001368F3
:10A28000391A99429BDB4A4D4A492846621CFCF721
:10A290003DFD002800F0DA8000202968844208553E
:10A2A000C0F2D48001271BE00F9B41484149F618BA
:10A2B000761B04EB06084246FCF728FD002800F058
:10A2C000C580FCF763FA18B128463146FFF7F5FC64
:10A2D0003748026829461019324618F03FFF4446B5
:10A2E0000F9B0E9DED182978A1B11FB1079EF106B5
:10A2F0000DD563B100222D4B00921868294610221B
:10A300000EAB00F011FD00283FF430AF02E0059ED7
:10A31000012700E0059E0A9826493618C5EB060875
:10A3200004EB0809224809F10202FCF7EFFC0028BF
:10A3300000F08C80B8F1000F08DD0F9E36B9079948
:10A34000CA0603D51E48FEF71BF92DE0FCF71EFADE
:10A3500018B128464146FFF7B0FC154E3168424619
:10A360000819294618F0FAFE164833680288444452
:10A370001A53002F53D009F10109B9F1000F62DB24
:10A380004DD03568FCF79BFCFCF7DEF90446FCF782
:10A39000DBF90D9A0146204605EB0907FCF78AFE1A
:10A3A00090B90646FCF78AFC30464FE0D40C0020FA
:10A3B000C40C0020E40C0020CC0C0020C00C0020B9
:10A3C00071A603086F9403080024FCF7BDF9494601
:10A3D00002462846FCF7CCFA054618B9FCF76EFC95
:10A3E000284633E02CB1FCF7AFF9FCF775FAA06012
:10A3F0000FE0FCF7A9F90646FCF7A6F9314602463C
:10A400002046FCF75BFD044618B9FCF757FC2046D4
:10A410001CE0BD42D9D1FCF751FC01220492069800
:10A42000431C06930C9B089806991A1A91427FF7D1
:10A4300078AE049949B9079AD30706D40548FEF7C0
:10A440009FF8049802E0002000E001202FB0BDE852
:10A45000F08F00BF68A6030810B504461AF0BCFAD6
:10A460000B49421C0B48FCF751FC78B1002201E07B
:10A470000132013407490B68981823785C2B04BF1C
:10A48000637801340370002BF2D1086810BD00BF5F
:10A49000D80C0020DC0C0020D0F80032FF2B03DDAC
:10A4A000044BC0F814327047C154591CC0F8001254
:10A4B000704700BF8CA60308D0F80432FF2B03DDE1
:10A4C000054BC0F814327047C21882F80011591CAD
:10A4D000C0F80412704700BFABA6030801680A4623
:10A4E00012F8013B6E2B02600ED006D8532B11D010
:10A4F000642B15D0302B16D10AE0732B0DD0742BA2
:10A5000004D0722B0FD110E00A2070470920704749
:10A51000002070474FF4805070474FF470607047D0
:10A520004FF488507047087870470D20704700003E
:10A5300008B5D0F800329A4205DB0748074A084BB5
:10A540004A2117F0A7F89A1AFF2ACABF054B4254AE
:10A55000C0F8143208BD00BFCAA60308A9A80308A2
:10A56000DCA60308F2A6030838B50C1E054609DD73
:10A570000021FFF791FF28462146A21EBDE8384082
:10A58000FFF7D6BF38BD00002DE9F04F85B00EAD06
:10A5900006460C461746984695E820065FE1D6F831
:10A5A00000329C4205DB9748974A984B4FF4D07194
:10A5B00006E0FF2C06DD9348934A954B40F2A1112B
:10A5C00017F068F8112900F23F81DFE811F03B0134
:10A5D0001200B1002D00BA00D000FA000E01EB000D
:10A5E000F2005E0069008000750050008800950050
:10A5F000A3003046E11C3A464346D5F800B08DE84A
:10A600002006FFF7C1FF58B13019C5F800B04178F6
:10A610003A463046611843468DE82006FFF7B4FFFE
:10A6200033199A78A41819E196F810C279487A4932
:10A630000CF001033219002B0CBF03460B462868AF
:10A6400092F802B0C0EB080CE34500F3A88092F842
:10A6500001E00EF58072B11838185A469847002864
:10A6600040F09D80296801EB0B032B6098E0304699
:10A67000A11C3A464346D5F800B08DE82006FFF706
:10A6800083FF48B1C5F800B006E0304621463A469F
:10A690004346009500F02AF9321950782418DEE07C
:10A6A0003046A11C3A4643468DE82006FFF76CFF72
:10A6B000002840F0D980E8E73046A11C3A464346DE
:10A6C0008DE82006FFF760FF002840F0CD8030467F
:10A6D00021463A464346009500F032F9DCE72B6804
:10A6E00043452CDA4D4917F803C00A6802EB0C0009
:10A6F000417811F0080F19E02B6843451FDA474AEB
:10A70000F85C11680A18507810F0080017D101336E
:10A710002B6054E02B68434511DA404817F803C01A
:10A72000026802EB0C01487810F0040F07D002E039
:10A730002B68434503DA01332B6000203FE03848A3
:10A740003DE02A6842452ADA3119002391F801B028
:10A750000BF5807006EB000B8878B95C04E01BF801
:10A7600003C08C4517D001338342F8DB17E02A6819
:10A77000424514DA3319587800F5807106EB010B65
:10A780009878B95C002304E01BF803C08C4506D020
:10A7900001338342F8DB01322A60002000E02048C8
:10A7A00003345BE029681E4B002914BF18460020C3
:10A7B00005E028681A4A404514BF104600200134BD
:10A7C0004CE0B9F1000F0BD033190AF1FF315B787F
:10A7D000994207DD2A68B81849F83300002002E0E2
:10A7E000484600E00F48023438E0B9F1000F27D0A6
:10A7F00031194B78534519DB0248034A0A4B40F2A2
:10A800002D21DDE6CAA60308B9A803081BA7030883
:10A810002DA7030801310208E9AC00086000002000
:10A8200068A6030809A703085FA70308296859F861
:10A83000330009EBC30207EB010CC0EB0C035360C0
:10A8400002340CE001340AE02246094818F0B8FD51
:10A850000848094A094B40F23A21B1E620B9315D76
:10A8600000297FF49CAE084605B0BDE8F08F00BF1C
:10A870007BA70308CAA60308B9A803089EE2030839
:10A880002DE9F04387B08946002106461746DDF8DA
:10A89000388005911D4623B118464FEAC80218F0CA
:10A8A00033FDD6F80C42B4B105AB8DE82801304633
:10A8B00000214A463B46FFF767FE11E006AB3046F3
:10A8C00043F8044D00218DE828014A463B46FFF736
:10A8D0005BFE013400E00448BC4201DA0028EDD1FF
:10A8E00007B0BDE8F08300BF68A603082DE9FF4765
:10A8F0000C9C07460E4691469A46256811E0BB1906
:10A90000D4F80080597801900290711838464A4670
:10A9100053460094FFF738FEC4F80080002808BFB3
:10A920004546002001900290B11C38464A465346E5
:10A930000094FFF729FE0028E1D02560BDE8FF87DD
:10A940002DE9F04385B006460C9C0D461746984607
:10A95000D4F800900DE07319D4F800905978019064
:10A960000290691830463A4643460094FFF70CFEC1
:10A9700058B1002001900290A91C30463A46434647
:10A980000094FFF701FE0028E5D0C4F8009005B060
:10A99000BDE8F08370B504460D4600211646FFF76A
:10A9A0007BFDD4F80022701920186119521B18F091
:10A9B0004DFCD4F800329E19C4F8006270BDF8B5A1
:10A9C0000D46415C03290446164615D1AF1CC35DF4
:10A9D000012B11D95A1EC255FFF75EFD6019E35DC8
:10A9E00041782046C918FFF757FD20460121FFF79F
:10A9F00053FDD4F80052033D204629460222FFF7BA
:10AA0000C9FF2046691C2A466655BDE8F840FFF795
:10AA10008FBD00002DE9F74FD0F80832D0F8007252
:10AA2000019304460D463E464FF0000829680A4649
:10AA300012F8013B2E2B2A6028D00DD8292B00F0CC
:10AA40009E8005D8242B1CD0282B74D0A3B1D1E034
:10AA50002B2B00F2CF809EE05C2B4ED006D83F2BF4
:10AA600000F0AC805B2B40F0C58014E05E2B05D07D
:10AA70007C2B40F0BF80A7E02960E3E0204608215E
:10AA800001E020460921FFF707FDCFE7D4F8006277
:10AA900020460221F7E74878D4F80062D4F804A2EF
:10AAA0005E2804D1023129604FF0050B1DE04FF004
:10AAB000040B1AE0581C5C2A286004D05D2A20464A
:10AAC00010D15946B2E02846FFF708FDC1B28146D1
:10AAD000204629B9FFF7F0FC20464FEA292102E081
:10AAE000494600E01978FFF7E7FC2B681A78002A3E
:10AAF000E0D1554BC4F8143298E72846D4F80062E8
:10AB0000FFF7ECFC10F47F4F8146204602D04FEA5D
:10AB10002921B8E70321FFF7BFFC2046D4F804122F
:10AB2000FFF7BAFC20460121FFF7B6FC2046494654
:10AB3000FFF7C2FC7AE7D4F80812D4F8006201F1FA
:10AB4000010920460621C4F80892FFF7A5FC20461B
:10AB50004946FFF7A1FC20462946FFF75BFF2A681C
:10AB600012F801CBBCF1290F2A6001D0374B0FE05E
:10AB700020460721FFF790FC2046494683E72960DD
:10AB800020464146FFF7F0FC019800285AD1304B8F
:10AB9000C4F8143256E00B7891F801E02A2B14BF68
:10ABA0000B220A22BEF13F0F05D1023129600A2A89
:10ABB00014BF0D220C222046314602E020463146C9
:10ABC0000E22FFF7FCFE31E741462046FFF7CCFCA2
:10ABD000204639460322FFF7DDFE01233A46E355BE
:10ABE0002046F91807F10208FFF7A2FCFF2204F83B
:10ABF00008201BE72960D4F80062D4F804A206E01C
:10AC00000BF10100286049462046FFF755FCD5F8B6
:10AC100000B09BF80090B9F1000F05D00D484946EF
:10AC200019F0D0FA0028EBD020460321FFF734FCBE
:10AC300020465146FFF730FCD4F804122046CAEBF8
:10AC4000010120E7BDE8FE8F93A70308AAA7030828
:10AC5000BDA70308D1A7030813B500220191C0F8CE
:10AC60001422C0F80C22C0F80822C0F80422C0F850
:10AC700000220B785E2B044602D10121C0F80C1291
:10AC800020460621FFF708FC20460021FFF704FCC0
:10AC900003E0204601A9FFF7BDFE019B18780028BC
:10ACA000F7D1A278012A03D120460421FFF75CFCEA
:10ACB00020460721FFF7F0FB20460021FFF7ECFBC1
:10ACC00020460021FFF7E8FBD4F814021CBD000069
:10ACD00004490B681A18517801F00303012B08BFCF
:10ACE00020307047600000202DE9F84304460D46EF
:10ACF0001746A2B1002614F806804046FFF7E8FF89
:10AD00008146A85DFFF7E4FFB9EB000008D1B8F178
:10AD1000000F05D00136BE42EDD1BDE8F8831046E4
:10AD2000BDE8F883FFF798BF2DE9F04117469DF87D
:10AD30001820044680F8102208461E460D4619F0D9
:10AD40004BFE03461A462046294633460697BDE881
:10AD5000F041FFF795BD000040F0BE61024B41F4A9
:10AD60002020D860704700BF00ED00E010B5C37828
:10AD70002BB3184AD4684278E14301F4E0631B0A1C
:10AD8000C3F1040C5FFA8CF412FA04F10F2454FAA4
:10AD900003F2847890F800C0C9B202EA040343EADF
:10ADA00001020D4B0CEB0301120181F80023037823
:10ADB000012203F01F00590912FA00F306E002789D
:10ADC0000123510902F01F0083402031024840F85E
:10ADD000213010BD00ED00E000E100E021F0604C0A
:10ADE0002CF07F02024B42EA00019960704700BFDD
:10ADF00000ED00E008B501214FF4807000F092FDF5
:10AE00004FF480700021BDE8084000F08BBD0000C9
:10AE100030B543680A6823F0407424F480750B79D8
:10AE200045EA020C4CEA03244460CD680A69846850
:10AE300045EA02038D680A4A43EA050C04EA020364
:10AE40004A794CEA030C4CEA42038360097DC26AEA
:10AE50004B1E22F47002D9B242EA0153C36230BDE4
:10AE6000FDF7FFC000210123016001714171816084
:10AE7000C16001610375704710B5094A094C5368F8
:10AE800003EA040C90E8120021438468C06841EA98
:10AE9000040343EA000141EA0C03536010BD00BF04
:10AEA00000230140E030FCFF836811B143F001034F
:10AEB00001E023F0010383607047092970B54FEA70
:10AEC00041040BD964181E3CC6680725A54026EA34
:10AED0000505A34045EA0304C4600AE00669641856
:10AEE0000725A54026EA050513FA04F445EA0403FC
:10AEF0000361062A0CD8013A02EB8202446B1F233D
:10AF0000934024EA030C91404CEA0102426370BD75
:10AF10000C2A4FEA82030CD89A18046B233A1F2399
:10AF2000934024EA030C11FA02F24CEA0201016395
:10AF300070BD9A18C46A413A1F23934024EA030C57
:10AF400011FA02F24CEA0201C16270BD836811B1CC
:10AF500043F4807301E023F4807383607047836857
:10AF600011B143F4007301E023F400738360704770
:10AF700008B50B4B984207D14FF00070012100F04B
:10AF8000C5FC4FF0007006E04FF08060012100F03A
:10AF9000BDFC4FF080600021BDE8084000F0B6BC69
:10AFA00000640040026822F002030360026842F07D
:10AFB000010303604FF480334268D20701D4013BA0
:10AFC000FAD1436813F0010358D08A790368012A43
:10AFD0000CBF43F0800323F080030360CA79036849
:10AFE000012A0CBF43F0400323F0400303600A7AB8
:10AFF0000368012A0CBF43F0200323F02003036001
:10B000004A7A0368012A0CBF43F0100323F01003AF
:10B0100003608A7A0368012A0CBF43F0080323F017
:10B0200008030360CA7A0368012A0CBF43F00403D3
:10B0300023F0040303608A7891F803C093070A7928
:10B0400043EA0C6343EA024391F805C00A8843EAE5
:10B050000C5C511E4CEA0103C361026822F001013D
:10B0600001604FF480334168CA0701D5013BFAD132
:10B07000436803F0010080F00100704718467047F4
:10B0800070B5837A01229A40394BD3F8004244F0DC
:10B090000101C3F80012D3F81C42D1430C40C3F89D
:10B0A0001C42047BC4B9D3F80C4201EA0406C3F87D
:10B0B0000C62847AB0F802C0C68848344CEA06456F
:10B0C00043F83450857A2B4BB0F804C00488ED0067
:10B0D000EB1844EA0C445C60037B012B19D1244B30
:10B0E000D3F80C4242EA0406C3F80C62847AB0F842
:10B0F00002C0068848344CEA064543F83450857A45
:10B100001C4BB0F804C0C488ED00EB1844EA0C44B2
:10B110005C60C47A164B1CB9D3F804420C4002E0C0
:10B12000D3F804421443C3F8044203892BB9104BEB
:10B13000D3F814422140C3F814120189012905D122
:10B140000B4BD3F814121143C3F81412407B01289F
:10B1500005D1074BD3F81C120A43C3F81C22044B39
:10B16000D3F8002222F00100C3F8000270BD00BF36
:10B17000006400404066004000238371C371037285
:10B1800043728372C3728370C3700322022101234E
:10B19000027141710380704770B5826852010346A5
:10B1A00007D48268120106D48068C00050D50220FE
:10B1B00002E0002000E0012000F1180632019D5855
:10B1C00005F001049C500C7A9D582CB90C6891F83C
:10B1D00009C04CEA445405E04E6844EAC60646EA13
:10B1E00005044D7A25439D508E7A00F1180406F02F
:10B1F0000F0224018A721A19556825F00F0656604D
:10B20000556891F80AC04CEA050656604A7B91F8E9
:10B210000EC0CE7A150445EA0C650A7B45EA060C99
:10B220004CEA022603EB0012C2F888614D7C8E7C4A
:10B2300091F810C02D0445EA0665CE7B354345EAFA
:10B240000C21C2F88C111A5942F00101195170BD3C
:10B25000042070BD30B501F11B042301C55805F071
:10B260000405EDB21572C35815B95B0D136001E00A
:10B27000DB08536024010319045904F0020C82F81E
:10B2800009C05C6804F00F0C82F80AC05C68230AED
:10B29000D37400EB0113D3F8B841D472D3F8B8419A
:10B2A000240A1473D3F8B841240C5473D3F8B8416A
:10B2B000240E9473D3F8BC41D473D3F8BC41240A50
:10B2C0001474D3F8BC41240C5474D3F8BC311B0E55
:10B2D000937421B9C26842F02001C16030BD016998
:10B2E00041F02003036130BD09B9C06802E00129C3
:10B2F00003D1006900F00300704700207047000090
:10B30000016821F0010303600021212301604160F5
:10B310008160C160016143612C4B98421CD02C4B71
:10B32000984220D02B4B984225D02B4B98422AD0C4
:10B330002A4B98422FD02A4B984233D0294B98421F
:10B3400037D0294B984204D14FF03D5243F8AC2CF2
:10B350007047264B984203D13D2043F8080C7047B4
:10B36000234B984204D14FF4746143F8201C70477A
:10B37000204B984204D14FF4741243F8382C704794
:10B380001D4B984204D14FF0746043F8500C704745
:10B390001A4B984203D11A4943F8641C7047194B61
:10B3A000984203D1184A43F87C2C7047174B9842B7
:10B3B00003D1174843F8940C7047164B984204BFCA
:10B3C0004FF03D5243F8AC2C704700BF1060024074
:10B3D00028600240406002405860024070600240B5
:10B3E00088600240A0600240B860024010640240E1
:10B3F0002864024040640240586402407064024085
:10B400003D00002088640240400F0020A0640240FC
:10B4100000003D20B86402400268164B10B502EAF5
:10B42000030CCC680A684B6922438C691343CA69D0
:10B4300023430C6A1A434B6A22438C6A13434A6BB8
:10B4400023438C6B1A4342EA040343EA0C02026072
:10B450004469CB6A24F007020C6B44EA030C4CEA03
:10B46000020242610B6943604A6882608B68C36074
:10B4700010BD00BF3F801CF0002303604360836069
:10B48000C360036143618361C3610362436283629A
:10B49000C3620363436383637047036811B143F07E
:10B4A000010301E023F001030360704730B5074B4F
:10B4B000074A084C084DA04288BF13460D4011F0C2
:10B4C000005F14BFDD609D6030BD00BF00600240C2
:10B4D000006402400F6402407D0F7D0F0B0607D50C
:10B4E000436912B143F0800301E023F0800343611C
:10B4F000802909D001F01E01036812B119430160CF
:10B50000704723EA010202607047000030B5074B24
:10B51000074A084C084DA04288BF13460D4011F061
:10B52000005F14BFDD609D6030BD00BF0060024061
:10B53000006402400F6402407D0F7D0F10B58379D7
:10B540000268002B2DD01C4B1C6824EA02021A60F2
:10B550005C68016824EA01025A6004790168E21813
:10B560001468214311609A68016822EA01029A6016
:10B570000168DA6822EA0102DA604179026810297A
:10B5800008D199680A439A60D968026841EA0200C2
:10B59000D86010BD01F1804C0CF59E331868024351
:10B5A00007E0007900F1804303F59E33196821EA32
:10B5B00002021A6010BD00BF003C014000230C22B3
:10B5C00003600371427183717047000003494B6946
:10B5D00018420CBF00200120704700BF003C014012
:10B5E000014B5861704700BF003C014005490A68A3
:10B5F0004B69034004D010420CBF0020012070476B
:10B6000018467047003C0140014B5861704700BF2D
:10B61000003C0140044B1A69002A03DA034904483C
:10B6200059605860704700BF003C024023016745E5
:10B63000AB89EFCD014BD860704700BF003C0240A2
:10B640000C4BDA68D0030ED4D868C1060DD4D96883
:10B6500011F0EF0F0BD1DA6802F00203002B0CBFE0
:10B6600008200720704701207047052070470620FA
:10B67000704700BF003C024007B508238DF8073033
:10B68000FFF7DEFF8DF807009DF807000128F7D0CF
:10B690009DF807000EBD000070B504460E46FFF78A
:10B6A000EBFF082813D10A4D2A6922F44070286163
:10B6B000296941F480732B612A6942F001002861F5
:10B6C0002680FFF7D9FF296921F001032B6170BDA6
:10B6D000003C024070B5044641B1012908D002295E
:10B6E00014BF4FF440764FF4007603E00E4601E0BD
:10B6F0004FF48076FFF7C0FF08281ED10F4D286950
:10B7000020F440732B612A6916432E61296921F0C8
:10B71000F80028612B6943F0020214432C61296967
:10B7200041F480302861FFF7A7FF2B6923F0020264
:10B730002A61296921F0F8032B6170BD003C0240A9
:10B74000F0B500231A4601240D6894402540A54217
:10B750002ED10327066817FA03F4E44304EA060728
:10B7600007600E7907689E403E4306600E79013EF1
:10B77000F6B2012E14D8866804EA060787604E796F
:10B7800087689E403E438660466826EA0506466016
:10B790008D79466895401FFA85FC4CEA06054560A0
:10B7A000C5682540C560CC79C5689C402C43C46001
:10B7B00001320233102AC6D1F0BD00234FF6FF71CB
:10B7C0000160037143718371C3717047036919424A
:10B7D0000CBF002001207047006980B270474069AB
:10B7E00080B2704701837047418370474161704761
:10B7F00030B501F00705C9080831AB000F2450F837
:10B8000021509C4025EA040440F8214050F8214092
:10B8100012FA03F31C4340F8214030BD10B5254B0C
:10B820009A6802F00C02042A03D0082A03D0224BA3
:10B8300024E0224B22E05C685968620201F03F017B
:10B840000AD55A681D4B47F6C07C02EA0C04A209CF
:10B85000B3FBF1F3534309E05A6847F6C07402EAB8
:10B860000403154C9B09B4FBF1F14B43114C616887
:10B8700001F44032D40BA11CB3FBF1F30D4903607A
:10B880008C6804F0F00213090D4A0468D35C34FAA2
:10B8900003F343608C6804F4E054A40A145D33FAA3
:10B8A00004F48460896801F46041490B525CD34020
:10B8B000C36010BD003802400024F40000127A007A
:10B8C00044000020044B1A6B09B1104301E022EA46
:10B8D00000001863704700BF00380240044B1A6C28
:10B8E00009B1104301E022EA00001864704700BF6C
:10B8F00000380240044B5A6C09B1104301E022EABF
:10B9000000005864704700BF00380240044B1A6AB8
:10B9100009B1104301E022EA00001862704700BF3D
:10B9200000380240044B5A6A09B1104301E022EA90
:10B9300000005862704700BF0038024008B5154B40
:10B9400098420BD101214FF48050FFF7EBFF4FF4E9
:10B9500080500021BDE80840FFF7E4BF0E4988424F
:10B9600007D14FF480400121FFF7D0FF4FF4804012
:10B9700009E00A4A90420BD14FF400400121FFF741
:10B98000C5FF4FF400400021BDE80840FFF7BEBFEF
:10B9900008BD00BF0030014000380040003C0040BE
:10B9A0000B88B1F802C0028810B58C884CEA030CF1
:10B9B000CB884CEA040C0C894CEA0303B1F80AC0AA
:10B9C00023438C8943EA0C0C4CEA0403CC8902F42F
:10B9D000415243EA040C42EA0C030380B0F81CC055
:10B9E0002CF4006213041A0C82830B8A038210BDAC
:10B9F000038819B19BB243F0400303E023F04002F7
:10BA000011040B0C03807047808980B270478181DC
:10BA10007047038919420CBF0020012070470000C5
:10BA20001B4A038890420ED01A4A90420BD0B0F1C4
:10BA3000804F08D0184A904205D0184A904202D050
:10BA4000174A904206D14FF68F7203EA020C4B88D8
:10BA50004CEA0303134A904209D0134A904206D09D
:10BA60004FF6FF4203EA020C0B894CEA0303038002
:10BA70004B68C362064B0A889842028502D0054A89
:10BA8000904201D1897A018601238382704700BFE9
:10BA90000000014000040140000400400008004094
:10BAA000000C00400010004000140040416270474C
:10BAB000C1627047406A7047008D80B2704703884A
:10BAC00019B19BB243F0800303E023F0800211041C
:10BAD0000B0C03807047038819B19BB243F001033C
:10BAE00003E023F0010211040B0C038070470000F7
:10BAF000028C22F0010370B51E04340C0484068C01
:10BB00008488058BB1F80CC025F0730213041A0C5D
:10BB100026F002031E04330C0D884E882A4346EAA1
:10BB20000C051FFA85FC134DA8424CEA030302D012
:10BB3000114DA84218D14FF6F77603EA0605CB89D6
:10BB40004FF6FB7645EA030C8B880CEA0606334376
:10BB5000B1F810C04E8A4FF6FF45254046EA0C0466
:10BB60001FFA84FC4CEA05048480028389684163DF
:10BB7000038470BD0000014000040140B0F820C003
:10BB80002CF0100230B515042C0C0484B0F820C041
:10BB90008488038B23F4E64215040B882A0C2CF0CE
:10BBA000200542EA03222B048D89B1F802C01B0C48
:10BBB00043EA0513124DA84243EA0C1302D0114D7B
:10BBC000A84217D14FF67F7503EA050CCB894CEAE2
:10BBD0000315B1F804C04FF6BF732B4043EA0C13B2
:10BBE0004FF2FF35B1F810C025404C8A45EA8C056C
:10BBF00045EA84048480028389688163038430BDBC
:10BC00000000014000040140B0F820C02CF4807214
:10BC100030B515042C0C0484B0F820C08488838BC4
:10BC200023F0730215040B882A0C2CF400751A43B8
:10BC30002B048D89B1F802C01B0C43EA0523134D78
:10BC4000A84243EA0C2302D0114DA84217D14FF26B
:10BC5000FF7503EA050CCB894CEA0325B1F804C053
:10BC60004FF6FF332B4043EA0C234CF6FF75B1F837
:10BC700010C025404C8A45EA0C1545EA041484801E
:10BC800082838968C163038430BD00BF0000014026
:10BC900000040140B0F820C02CF4805230B51504E7
:10BCA0002C0C0484B0F820C08488838B23F4E642F3
:10BCB00015040B882A0C2CF4005542EA03222B04AD
:10BCC0008D89B1F802C01B0C43EA0533094DA84227
:10BCD00043EA0C3302D0084DA84205D14BF6FF755C
:10BCE00025400C8A45EA8414848082838968016433
:10BCF000038430BD000001400004014000230380A4
:10BD00004380838083608381C38103824382704741
:10BD1000B0F818C02CF0080213041A0C41EA020310
:10BD200003837047B0F818C02CF4006213041A0C97
:10BD300042EA012303837047B0F81CC02CF00802CC
:10BD400013041A0C41EA020383837047B0F81CC045
:10BD50002CF4006213041A0C42EA01238383704717
:10BD6000B0F8443021B16FEA43436FEA534301E036
:10BD700059044B0CA0F84430704783899BB20AB138
:10BD8000194301E023EA010181817047038A1942C6
:10BD90000CBF002001207047C94301827047038A0D
:10BDA000828911EA030092B203D011420CBF002035
:10BDB00001207047C94301827047828822F07003D6
:10BDC0001A04130C8380B0F804C01FFA8CF241EA05
:10BDD000020383807047000008B5234B984205D1C9
:10BDE00010200121FFF79EFD102037E01F498842F7
:10BDF00007D14FF400300121FFF788FD4FF40030E8
:10BE000009E01B4A90420BD14FF480200121FFF73B
:10BE10007DFD4FF480200021BDE80840FFF776BD8E
:10BE2000144B984207D14FF400200121FFF76EFD1B
:10BE30004FF40020EFE71049884207D14FF48010FB
:10BE40000121FFF763FD4FF48010E4E70B4A9042B5
:10BE500009D120200121FFF765FD20200021BDE848
:10BE60000840FFF75FBD08BD0010014000440040DE
:10BE700000480040004C00400050004000140140C9
:10BE800030B5B0F810E02EF440521304CA881B0CF1
:10BE900013430382B0F80CC02CF4B05E2EF00C02F9
:10BEA000B1F804C013040A890D46498942EA0C021C
:10BEB00042EA010E1B0C1FFA8EFC4CEA0301818141
:10BEC000828A22F440731904AA890B0C43EA020106
:10BED00085B0044681826846FFF7A0FC1C4B9C425B
:10BEE00002D01C48844201D1039B00E0029BA2893E
:10BEF0000FFA82FC4FF01901BCF1000F2A6801FB18
:10BF000003F101DA520000E092006423B1FBF2F188
:10BF1000B1FBF3F21201100903FB1011A0890FFA13
:10BF200080FEBEF1000F06DAC9003231B1FBF3F337
:10BF300003F0070305E009013231B1FBF3F000F033
:10BF40000F0343EA020CA4F808C005B030BD00BFDF
:10BF50000010014000140140838919B19BB243F4E1
:10BF6000005303E023F4005211040B0C838170474B
:10BF7000CA05D10D818070478188C805C00D704702
:10BF8000CBB210B55B09012401F01F0114FA01F1D5
:10BF9000A34201D10C3004E0022B01D1103000E0AB
:10BFA000143003680AB1194301E023EA010101607A
:10BFB00010BD038819420CBF002001207047C943FF
:10BFC0000180704710B5CCB20122640901F01F0353
:10BFD0009A40012C01D1838903E0022C0CBF038A13
:10BFE000838A9BB20088134082B243B1080A0123BE
:10BFF00013FA00F111420CBF0020012010BD1846B9
:10C0000010BD0000344B186840F001021A60002295
:10C010009A60196821F0847C30492CF480301860D3
:10C020005960186882B020F480211960DA600092AB
:10C030000192186840F480321A60274B1A6802F4A3
:10C04000003101910098421C0092019919B90098A1
:10C05000B0F5A06FF1D11A6812F4003118BF0121B8
:10C060000191019B012B30D11B4B1A6C42F0805087
:10C070001B4A1864116841F4804010609968996007
:10C08000986840F400429A609968164A41F4A050BA
:10C0900098605A60196841F0807018600E4B1968FA
:10C0A0008A01FBD5104A40F205711160986820F0B2
:10C0B000030199609A6842F002009860064883681C
:10C0C00003F00C0CBCF1080FF8D1084A4FF00061E6
:10C0D000916002B0704700BF003802401030002469
:10C0E0000070004008544007003C024000ED00E0B2
:10C0F000002100F004B80C4B5B58435004310B484E
:10C100000B4B42189A42FFF4F6AF0A4A00F003B80C
:10C11000002342F8043B084B9A42FFF4F9AFFFF7C3
:10C1200071FFF4F731F8704718F70308000000209A
:10C130000C020020180200204C120020FFF7FEBF66
:10C14000704700002DE9F84FD0F800B0C469D0F86E
:10C1500004A0D0F80890D0F80C800769466985697A
:10C160001E4817F045FA59461D4817F029F951465F
:10C170001C4817F025F949461B4817F021F941469C
:10C180001A4817F01DF93946194817F019F93146C0
:10C19000184817F015F92946174817F011F92146E4
:10C1A000164C174817F00CF92168164817F008F9D3
:10C1B000154A1648116817F003F91549154809681A
:10C1C00017F0FEF814480168144817F0F9F8144BFA
:10C1D0001448196817F0F4F8FEE700BFBFA8030879
:10C1E000D4A80308DDA80308E6A80308EFA80308FD
:10C1F000F8A8030802A903080BA9030838ED00E01A
:10C2000014A903081EA9030828ED00E029A90308C2
:10C210002CED00E034A9030830ED00E03FA903084D
:10C220003CED00E04AA903081EF0040F0CBFEFF339
:10C230000880EFF30980FFF785BF704708B500203D
:10C24000202100F01DFA00204D2100F019FA0020F5
:10C250004D2100F015FA0020212100F011FAEEE73F
:10C2600008B50020202100F00BFA0020422100F048
:10C2700007FA0020462100F003FA0020212100F0F7
:10C28000FFF9EEE708B50020202100F0F9F90020C1
:10C29000552100F0F5F90020462100F0F1F90020C9
:10C2A000212100F0EDF9EEE770477047704700007C
:10C2B0000C4A034610B552F820005BB1052B09D09B
:10C2C000062B07D0072B05D00749084C082B08BFC1
:10C2D0000C4600E0044CFFF7EFFB013094FBF0F05C
:10C2E00010BD00BFACAA0308007A030A00BD010517
:10C2F00030B5194B85B0044653F8205058B1052885
:10C3000009D0062807D00728144B05D0144A08285E
:10C3100018BF134600E0114BB3FBF1F2531E4FF66A
:10C32000FF71002002918B4238BF1946ADF804100E
:10C33000ADF80C00ADF806008DF80E0001A92846F6
:10C34000FFF76EFB28460121FFF7C5FB2046FFF7EC
:10C35000AFFF05B030BD00BFACAA0308007A030AE6
:10C3600000BD010573B52C4B164653F820506846A6
:10C370000C46FFF722FA0B2E4BD8DFE806F00B1025
:10C380002E171E333D400626151C2846A1B2FFF786
:10C390002DFA3CE02846A1B2FFF724FA37E0284600
:10C3A000A1B2FFF721FA32E04FF6FF7400200094AB
:10C3B0008DF8040027E04FF6FF7400940221012459
:10C3C0008DF804408DF8051010E0284614B9FFF7E9
:10C3D00003FA1FE0FFF703FA1CE02846A1B2FFF7BB
:10C3E000F5F917E0009401248DF8074028466946C6
:10C3F000FFF7A6F920460DE00094022301E0009427
:10C4000000238DF8073028466946FFF799F9012087
:10C4100000E000207CBD00BF1CAA03082DE9F04FFE
:10C420000C4699464149424B002808BF194689B03D
:10C430000546B1FBF2F0F5F7DBF9C0B2072834BFCF
:10C440000746072700263B4B3B4953F825803B4ACC
:10C4500005EB450001EB000A525D1AF80610404654
:10C460000136FFF7C5F9032EEDD13549354E31F8C8
:10C4700015004FF0000A02224FF0010B06A90690AA
:10C4800040468DF81D208DF81C208DF81EA08DF8DB
:10C490001FB0FFF755F956F825603046FFF74EFA02
:10C4A00030465146FFF7A4FA139B1299ADF804A049
:10C4B000102B0CBF4FF4006CD446234BADF808C0D2
:10C4C000544514BF4FF482745446D14514BF4FF005
:10C4D0000209D146B1EB0A0018BF012033F817C09A
:10C4E000ADF80C0007214FF40072ADF8141030467F
:10C4F00001A9ADF80E20ADF810C0ADF80640ADF8BA
:10C500000A90ADF812A0FFF74BFA30465946FFF7F4
:10C510006FFA0748054A5F44554514BF154605465E
:10C5200055FA07F009B0BDE8F08F00BF80DE800249
:10C5300000BD01058CAA0308E2AA0308A4AB030806
:10C54000DCAA0308E0A9030838AB0308084B10B5C0
:10C5500053F8204089B22046FFF759FA20460121BE
:10C56000FFF757FA0028F9D02046FFF74DFA10BD23
:10C57000E0A9030870470000F0B587B000250091DE
:10C580000C21052A0446ADF80C500C98ADF80A10A1
:10C5900008DB082A06DD092A04D14FF48052ADF8E1
:10C5A000042002E00026ADF8046020B14FF40050F2
:10C5B000ADF8060001E0ADF8060013B1012B0AD179
:10C5C00004E04FF48063ADF8083007E04FF4C06733
:10C5D000ADF8087002E00021ADF80810204A214EA5
:10C5E000175D56F824602049204D095D30463A46D3
:10C5F000FFF7FEF855F824501D4B2846195D3A46C2
:10C60000FFF7F6F81B48022130F814208DF81510BA
:10C6100000278DF814108DF816703046012704A9F4
:10C6200004928DF81770FFF78BF8134B8DF8177085
:10C6300033F8140004A904902846FFF781F80F4A44
:10C6400052F824402046FFF7C7FB20466946FFF713
:10C6500017FC20463946FFF77FFC384607B0F0BD8F
:10C660001EAB030898AA030855A903086CAA03087F
:10C6700014AB030858AB03084EAB0308FCAA03082D
:10C6800070B506460D46074B53F8264080212046DC
:10C69000FFF78FFC0028F6D020462946BDE8704001
:10C6A000FFF766BCFCAA030852EA030170B5044612
:10C6B0000C4E08D156F8204020212046FFF779FC87
:10C6C00068B1204608E056F8245020212846FFF79C
:10C6D00070FC0028F7D02846FFF74EFC70BD4FF0E5
:10C6E000FF3070BDFCAA0308274B0228F7B50446AB
:10C6F00053F820500F464FF0000044D802228DF826
:10C7000005208DF80400C1B9AA8A22F440731904E7
:10C710001E4A1F4B080CA88232F8141033F814007C
:10C7200041EA000202A91B4893B241F8083D50F8C3
:10C7300024006946FFF704F824E011F002060DD04A
:10C74000124B144E33F8141002A840F8081D56F886
:10C7500024006946FEF7F4FF4FF40076FB070ED580
:10C760000B4B0C4A33F81410022000918DF8040092
:10C77000694652F8240046F48076FEF7E1FFAA8A63
:10C780001643AE820120FEBDFCAA030810AA0308CE
:10C7900064AA030880AA030808B5F5F745F8BDE8C0
:10C7A0000840F5F773BA0000F7B51F46144B16465C
:10C7B00053F82050FFF77CFDA0FB062300FB073356
:10C7C0001946104600230F4A24F06EFF0024064647
:10C7D0000F4628462146FFF769F9019402E00198C7
:10C7E000431C01930199C729F9D92846FFF762F93B
:10C7F00000230246B24273EB0701F6D3FEBD00BF31
:10C80000ACAA030840420F00144B13B553F8203074
:10C81000062911D8DFE801F00412161A10101D00C5
:10C8200018460021FFF742F9002301E00198431C5C
:10C8300001930199C729F9D900200CE01846FFF7A8
:10C8400039F908E01146FFF753FD04E0FFF730FD2A
:10C8500001E04FF6FF7000211CBD00BFACAA030829
:10C86000F0B51D46484B144653F8207054EA0503B2
:10C8700087B0064608D1384602210022FFF77DFA2C
:10C8800000203880B8806EE038B1052805D0062831
:10C8900003D0072801D0082803D137A1D1E900012E
:10C8A00002E037A1D1E9000100FB05F304FB0133ED
:10C8B000A0FB04015918354A002324F0F5FE010CB1
:10C8C00001315EB1052E09D0062E07D0072E304B60
:10C8D00005D0304A082E18BF134600E02C4BB3FB9E
:10C8E000F1F13046FFF704FD3046FFF7E1FCA0FB15
:10C8F000042300FB0533194610460023234A24F085
:10C90000D3FE04460D4654EA05032ED0B4F5803F0D
:10C9100075F100032BD200213846FFF7DCF801A89F
:10C92000FFF7ECF9002100200122ADF80410ADF86A
:10C93000100001A93846ADF806200394FFF7D8F897
:10C9400038462146FFF7B4F838460821FFF7E0F9EA
:10C950000C99114B384699550021FFF7A7F8384636
:10C960000121FFF7B8F8002002E0012000E00220DA
:10C9700007B0F0BDAFF30080007A030A00000000AA
:10C9800000BD010500000000ACAA030840420F00F2
:10C99000007A030A00BD0105FC100020AFF30080FF
:10C9A000024948688B680021C01A704710E000E017
:10C9B000024B186820F002021A60704710E000E095
:10C9C000024B186840F002021A60704710E000E065
:10C9D000F5F76CB970B509228AB00C463648374E67
:10C9E0000021FEF705FF012109223348FEF700FF71
:10C9F0000221012003228DF824108DF82510002536
:10CA00008DF8270008A92C4808928DF82650FEF7CB
:10CA100097FE2B4B9C4209D8324652F8040F2B4606
:10CA20000135844204D3042DF7D102E0042500E04F
:10CA30001D462448FEF79CFA05A8FEF79DFB224BF5
:10CA4000224A585D515D224B224A8DF817008DF81D
:10CA50001810585D515D8DF819000024ADF81410C0
:10CA600018488DF81A4005A98DF81B408DF81C4018
:10CA70008DF81D408DF81E408DF81F408DF8164032
:10CA8000FEF790FA012301A88DF80E408DF80F40B3
:10CA90008DF81030ADF80440ADF80640ADF8084010
:10CAA000ADF80A40ADF80C408DF81130FEF7E8FA09
:10CAB00056F825000AB070BD000C024024AB0308F4
:10CAC0003F420F0000640040DAA9030848AB0308A6
:10CAD00019AB0308EBAA03087FB5089812B1012A25
:10CAE00008D103E08DF80C20019103E004228DF8B9
:10CAF0000C20029100218DF80D1003F00701DA1DC2
:10CB00008DF80E304B1ED210062B05D8DFE803F04F
:10CB1000352E272019120B000DF10F0310F801CB51
:10CB200003F801CB01E00DF10F0310F801EB03F85E
:10CB300001EB01E00DF10F0310F8011B03F8011BDD
:10CB400001E00DF10F0310F801CB03F801CB01E078
:10CB50000DF10F0310F801EB03F801EB01E00DF10B
:10CB60000F0310F8011B03F8011B01E00DF10F0387
:10CB700010F801CB03F801CB01E00DF10F0390F8A1
:10CB800000E0013A002A83F800E002DD01330130C1
:10CB9000C4E701A90248FEF7FFFA07B000BD00BFD5
:10CBA00000640040F0B587B00D4634480C9E00216B
:10CBB00014461F46FEF798FB002859D02F48002145
:10CBC00001AAFEF747FB9DF80C3013B9019A2A60C1
:10CBD00002E0029B2B60012323709DF80E3003F0CE
:10CBE0000701DA1D481E3B70D210062805D8DFE881
:10CBF00000F0352E272019120B000DF10F0313F84A
:10CC0000010B06F8010B01E00DF10F0313F801CB46
:10CC100006F801CB01E00DF10F0313F801EB06F864
:10CC200001EB01E00DF10F0313F8011B06F8011BE6
:10CC300001E00DF10F0313F8010B06F8010B01E001
:10CC40000DF10F0313F801CB06F801CB01E00DF154
:10CC50000F0313F801EB06F801EB01E00DF10F03F0
:10CC60001978013A002A317005DD01360133C6E733
:10CC70004FF0FF3000E0012007B0F0BD006400403D
:10CC800008B50648FEF718FF044B054AD96A01307B
:10CC900092FBF0F04B1CB0FBF3F008BD0008004025
:10CCA00000BD01051FB50E4AB2FBF1F31A0C044694
:10CCB000501CB3FBF0F1481E0023029001A9094863
:10CCC000ADF80420ADF80C30ADF806308DF80E301C
:10CCD000FEF7A6FE2046FFF7D3FF04B010BD00BF4D
:10CCE00000BD0105000800402DE9F047044688B06A
:10CCF00088464148414E00211746FEF7ECFE3E486B
:10CD00000021FEF7D3FE16F804A03D48012606FADE
:10CD10000AF54FF00209069506A900258DF81D9029
:10CD20008DF81C908DF81E508DF81F50FEF708FDF1
:10CD30004A4633485146FEF75BFD41462046FFF721
:10CD4000B1FF314680462C48FEF7B9FE6023ADF8AE
:10CD50000430294B198CADF808508AB204FA09F056
:10CD600052FA00F101EA0600ADF80600DA6AADF801
:10CD7000105091194F436420B7FBF0F7BFB24FF446
:10CD800080730397ADF81430032C2FD8DFE804F03C
:10CD9000020B141D01A91848FEF7AAFE1648082127
:10CDA000FEF7B6FF19E001A91348FEF7E7FE1248A7
:10CDB0000821FEF7B7FF10E001A90F48FEF724FF96
:10CDC0000D480821FEF7B8FF07E00B4801A9FEF760
:10CDD00061FF09480821FEF7B9FF01210648FEF767
:10CDE000BFFF05480121FEF776FE01E04FF0000885
:10CDF000404608B0BDE8F0870008004016AA0308C6
:10CE0000000C0240054B8200B3F820C0012111FA4A
:10CE100002F040EA0C021A84704700BF000800408C
:10CE2000064BB3F820C0820001211FFA8CFC11FAD6
:10CE300002F02CEA00021A84704700BF000800408C
:10CE400000487047007A030ABFF34F8F054A06482F
:10CE5000D36803F4E06141EA0003D360BFF34F8F6E
:10CE6000FEE700BF00ED00E00400FA05836823F050
:10CE7000405241EA020383607047836811B143F076
:10CE8000804301E023F0804383607047013901292A
:10CE90008CBF00200120704770B50646F5F776F884
:10CEA00005460020F5F77AF829786FF3000129701C
:10CEB000436E012212FA06F623EA06064666456E1E
:10CEC000044685B9026F084B294653F82200FFF744
:10CED000CDFF0648C570FDF749FF94F8600065F383
:10CEE000C30084F8600070BDF0AA0308E0100020C1
:10CEF00073B50020F5F752F84B4D026F0446002140
:10CF000055F82200FFF7B2FF216F55F821000021EC
:10CF1000FEF71CF8206F002155F82000FDF7C4FF34
:10CF2000FDF768FF03238DF8043000238DF80730E8
:10CF300027E094F874603D4B54F82610486894F844
:10CF4000741033F810203A4B02AE46F8082D54F80E
:10CF500021004268694653F82200FEF7F1FB94F87D
:10CF6000746094F8741054F82630206F4A1C55F8F9
:10CF700020001979D2B20023FDF79FFF94F8746066
:10CF8000731C84F8743094F874C094F87520944538
:10CF9000CFD3002684F8746094F875202549206F5B
:10CFA0000A7555F82000FDF733FF216F55F8210071
:10CFB0000121FDF779FF31461F48FEF76EFA1E4842
:10CFC000FEF79EF994F875301C491B480B6104F17B
:10CFD00040028A60FEF720FA01211748FEF75DFA49
:10CFE00001211748FDF7BBFF206F012155F82000F4
:10CFF000FDF7ACFF102101220F48FEF76FFA94F8FD
:10D000006030DA070DD594F8600000F00801CBB26B
:10D010003BB1226F044B4FF0805153F82200FFF7D1
:10D0200025FF01207CBD00BFF0AA03085AA9030810
:10D0300064AB0308E410002010640240A410002038
:10D040000020014038B50020F4F7A8FF314905461B
:10D050003148FEF75BFA002335E095F8742055F867
:10D0600022402178237A41F01000207043B12178CA
:10D0700001F00800C3B21BB96068F5F768F80EE06C
:10D08000B4F814C01FFA8CF2012A08D90120616893
:10D09000A269F4F77BFE23786FF3041323706068B2
:10D0A000F5F728F9A28A91B2884209D394F800C012
:10D0B0000CF0040E5FFA8EF010B96068FFF7ECFE1A
:10D0C00095F87430013385F8743095F8741095F83C
:10D0D00075209142C1D3002085F8740095F8602036
:10D0E00002F00801CBB20BB1F4F75CFF95F86000D9
:10D0F000C1070ED495F8602002F00801CBB243B10D
:10D10000286F064B53F820000121BDE83840FFF797
:10D11000B4BE38BD2080001010640240F0AA03089D
:10D120002DE9F043044685B000200E46F4F736FFA3
:10D13000364F036F0546002157F82300FFF796FE90
:10D14000B846334B95F86020002E50D042F00102D3
:10D1500085F860202F4FEA6E57F822004FF080517B
:10D16000D86099605CB1052C09D0062C07D0072C3B
:10D1700005D0294B294F082C08BF1F4600E0264F39
:10D18000B7FBF6F10B0C5F1CB1FBF7F77E1E0296A6
:10D19000234EADF8043000201021ADF80C00ADF89E
:10D1A000061056F8220001A9FEF73AFCB14664B118
:10D1B000052C0AD0062C08D0072C06D0164A174892
:10D1C000082C14BF0446144600E0134CE96E59F8CD
:10D1D0002100FEF771FCEB6E461C94FBF6F459F847
:10D1E00023002021B4FBF7F6FEF7E7FD04E066F329
:10D1F000000285F860209E602A6F054958F82200D9
:10D20000FDF706FE304605B0BDE8F083F0AA03083E
:10D21000E41000207CA90308007A030A00BD010580
:10D22000ACAA03082DE9FF4100214FF00060FDF793
:10D23000D5FD4FF4E060FDF78FFD01200024FF22B3
:10D240008DF802008DF8030068468DF800208DF8F7
:10D250000140FDF78BFDAA4838210223017044707C
:10D260008370C470FDF782FDA64EA74DA059012121
:10D27000FEF728FB6846FEF7A0FA605969460434B9
:10D28000FEF75EFA142CEFD1042100229F48FEF72E
:10D29000AFFA032100229D48FEF7AAFA0D210022D1
:10D2A0009B48FEF7A5FA0E2100229948FEF7A0FA46
:10D2B0004FF4604700220F2195480124FEF798FAA9
:10D2C000022500970326002791488DF807406946FC
:10D2D0008DF804508DF805608DF80670FEF730FA71
:10D2E00018228A4800926946FEF72AFA894B586844
:10D2F00040F00301596010202146FEF7FBFA214659
:10D300004FF40030FEF7EAFA21464FF48020FEF792
:10D31000E5FA21464FF40020FEF7E0FA21464FF4EB
:10D320008010FEF7DBFA20202146FEF7E3FA2146C3
:10D330004FF48050FEF7DEFA21464FF48040FEF7AE
:10D34000CDFA21464FF40040FEF7C8FA20462146A8
:10D35000FEF7D0FA21462846FEF7CCFA21464FF4D4
:10D360008030FEF7C7FA21464FF40030FEF7C2FACC
:10D3700021464FF48020FEF7BDFA20462146FEF7F5
:10D38000ADFA21462846FEF7A9FA21460420FEF709
:10D39000A5FA21460820FEF7A1FA21464020FEF713
:10D3A0009DFA21468020FEF799FA21464FF48070BD
:10D3B000FEF794FA3C4620464CF250310134FEF719
:10D3C00097FF0C2CF7D104200121FEF793FA0020DF
:10D3D000F4F7E4FD0026074630460136F4F785FEF3
:10D3E000102EF9D101214FF48070FEF783FAFDF77A
:10D3F00001FD4948DFF84C810024FDF733FD4FF46F
:10D40000403568460195009402940394FDF734FD7D
:10D4100041493A6F0C6001254FF0006358F8220033
:10D42000CB600D714C718C600C610D75FDF7F0FCDB
:10D43000396F58F821002946FDF736FD29464FF48B
:10D440008000FEF73FFA3548FDF75AFF3448FEF7F3
:10D4500013F8334933480C604FF480634FF4006293
:10D4600048608B6140374FF480734FF400504B623B
:10D47000CA618F60CC600D614C6108628C62274884
:10D48000FDF7CAFF25482849FEF710F82348274929
:10D49000FEF73CF821462648FDF761FD2946244861
:10D4A000FDF754FD29461D48FDF7F7FF2A46314692
:10D4B0001A48FEF713F821462046FFF731FE2946A9
:10D4C0004FF00070FEF70AFA1A48F4F7CBFB64201D
:10D4D000F4F7D2FB184B1949194A5960F02007217B
:10D4E00082F823009C60F3201960FEF7A3F8FEF792
:10D4F00091F8F4F769F8284604B0BDE8F08100BF60
:10D50000E010002040AA03081CAA030800040240FF
:10D5100000000240002004E0E410002010640240FB
:10D52000A41000204C200140380000102080001082
:10D5300000200140007A030A10E000E07FA21900F9
:10D5400000ED00E0F0AA030838B50020F4F726FD4E
:10D5500090F86010044601F00800C0B208BBF4F770
:10D5600021FD94F86010104841F0080584F86050DF
:10D570000E49FDF7CBFF0E480125C570FDF7F6FB00
:10D5800094F860000B4B226F10F0010F53F822004B
:10D5900004D04FF08051FFF769FC02E02946FFF705
:10D5A0006CFC012038BD00BF1064024020800010D8
:10D5B000E0100020F0AA03082DE9F04106460D46D0
:10D5C000904600240CE0315B3846FEF765F80828E9
:10D5D000014604D03A46064815F0F2FE04E0023453
:10D5E000444504EB0507EED32046BDE8F08100BFBB
:10D5F000A4A9030808B5064B022133F81000FEF772
:10D6000069F8A0F1080EDEF1000040EB0E0008BD45
:10D610008CA903080020704700F01F00704700002D
:10D62000034951F820309889C0F34000704700BF8B
:10D63000B4AB030870B50E46094951F820402021CB
:10D640002046FEF7B6FCA0F101035D4245EB030561
:10D650001EB120462021FEF7B2FC284670BD00BF57
:10D66000FCAA030808B5064B40F2255153F82000E8
:10D67000FEF7A8FCA0F10102504240EB020008BDF9
:10D68000FCAA030870B50D460646FFF7EBFFA5F1AF
:10D690000103044605485A4250F8260040F225513D
:10D6A00042EB0302FEF76CFC204670BDFCAA0308A7
:10D6B000084B70B553F820400E4620460221FEF775
:10D6C00065FB05461EB120460221FEF765FB284694
:10D6D00070BD00BFB4AB030870B50D460646FFF73A
:10D6E0009FFFA5F101030446054802215A4250F864
:10D6F000260042EB0302FEF740FB204670BD00BF50
:10D70000B4AB0308F8B5044608461546FFF784FF96
:10D710000F4B53F8206007463046FDF757FF0128AE
:10D7200011D110FA07F70B48012C0CBF8068C068B4
:10D7300007420CBF0020012040B135B13046FDF753
:10D740004FFF0120F8BD0020F8BD0120F8BD00BF4B
:10D75000ECAB0308003C014003460A460220194690
:10D76000FFF7D0BF03460A4601201946FFF7CABF9C
:10D7700038B5114B53F82050044602212846FEF7D5
:10D780000EFBB8B102212846FEF714FB631C02D140
:10D79000F4F74AF803E00320A1B2F4F709F80749C7
:10D7A000085D022806D0284602210022BDE8384044
:10D7B000FEF7E3BA38BD00BFB4AB0308FC1000208D
:10D7C00081B20420F3F7F4BF2DE9F84383089F1CCE
:10D7D0001F4E00F0030556F82720A90032FA01F386
:10D7E0005F011C49FEB246EA00058B680126ADB216
:10D7F00006FA00F94FEA551219EA030F044602F03F
:10D800000F0805F01F070AD0404616FA07F102225A
:10D81000FEF7A8FD18B130462946F3F7C9FF0D49B8
:10D82000C86819EA000F0BD0012212FA07F140462E
:10D830000222FEF797FD18B902202946F3F7B8FF38
:10D84000054B53F82400BDE8F843FDF7DDBE00BFEB
:10D8500000380140003C0140ECAB030810B5064A1B
:10D860001468FFF7D9FE012111FA00F323420CBF1F
:10D870000020012010BD00BF003C0140FFF7EEBFBB
:10D88000FFF7ECBF2DE9F341044608460E469046EB
:10D89000FFF7E4FF07463046FFF7BEFE012585404F
:10D8A000B8F1010F06462AD16846FDF787FE2148E8
:10D8B000002350F826608DF804301F4B00969A68BC
:10D8C000154201D0022C04D0D9680D4205D0012C9C
:10D8D00008D110228DF8052007E0012C0CBF082488
:10D8E0000C2400E00C248DF80540012368468DF8D7
:10D8F0000630FDF723FE3046FDF786FE17E0012CCB
:10D900000D4B6FEA050204D1996802EA01009860A4
:10D9100002E0D8680240DA60074B9A68D86840EAAB
:10D9200002010D4203D1196821EA05051D60384640
:10D93000BDE8FC81ECAB0308003C014003460A460D
:10D9400002201946FFF79EBF03460A4601201946EA
:10D95000FFF798BF0020FFF733BF0120FFF730BF6C
:10D960000220FFF72DBF0320FFF72ABF0420FFF797
:10D9700027BF0020FFF728BF0120FFF725BF0220A7
:10D98000FFF722BF0320FFF71FBF0420FFF71CBFD4
:10D9900038B5074D052455F8040FFDF727FE10B1E3
:10D9A0002046FFF711FF01340A2CF4D138BD00BF27
:10D9B000FCAB030838B5074D0A2455F8040FFDF7F2
:10D9C00015FE10B12046FFF7FFFE0134102CF4D1F4
:10D9D00038BD00BF10AC03080020FFF7C9BE01200E
:10D9E000FFF7C6BE0220FFF7C3BE0320FFF7C0BE8D
:10D9F0000420FFF7BDBE0720FFF7BABE13B5012311
:10DA000000248DF805408DF806408DF80730124847
:10DA1000215C02A8013400F8041DFDF7A7F9052CCC
:10DA2000F5D100240D4B02A8E25C013400F8042D6E
:10DA3000FDF79CF9072CF5D10024094AA05C0121CF
:10DA40008DF80400013401A88DF80610FDF78EF959
:10DA5000052CF2D11CBD00BFACAB0308E4AB03083E
:10DA6000A7AB030808B5FFF7EFF9002008BD0000D9
:10DA700062B6704772B67047EFF31080704700BF10
:10DA800038B50446FFF7F8FF012C054602D1FFF731
:10DA9000EFFF01E0FFF7EEFF05F08000D0F101009D
:10DAA00038BF002038BD08B5FFF7E6FF00F0800062
:10DAB000D0F1010038BF002008BD00002DE9F04181
:10DAC00004460D4690461AB328B303782F2B22D173
:10DAD00016F082FF0C281ED800273E4607E01349A7
:10DAE0002046795816F026FB0C37B8B10136104A9B
:10DAF00013689E42F3DB102B13D00C4F0C207043A5
:10DB000039183C50581C4D60C1F8088010600AE07C
:10DB10006FF0050607E06FF0030604E04FF0FF36F4
:10DB200001E06FF002063046BDE8F081F40C002001
:10DB3000F00C0020031E08DB06480268934206DA58
:10DB4000054A0C2101FB032070470020704700208C
:10DB5000704700BFF00C0020F40C0020014B186847
:10DB6000704700BFF00C002008B500F0E3FA04484D
:10DB700003680021986816F00BF8002008BD00BF6C
:10DB8000640000202DE9F04700240746A046254602
:10DB9000264612E0254B54F803A0504616F01CFF11
:10DBA0008146514638464A4616F046FF18B9C145E7
:10DBB00084BFC846354601360C341D490868864284
:10DBC000E8D31C4CB8F1000F0CD00C26174A06FB0A
:10DBD00005FC02EB0C0852F80C0016F0FDFE6B1D64
:10DBE000014605D12368582018600020BDE8F08761
:10DBF000D8F8082053692BB92068582101601846CD
:10DC0000BDE8F08779182068D8F8042098470746BF
:10DC100048B1082015F020FA18B923681E60BDE845
:10DC2000F08705704760BDE8F08700BFF40C002066
:10DC3000F00C00206400002010B5014603780D4868
:10DC400002680D48934204DB036809211960002033
:10DC500010BD0A4A0C2404FB032293689B6923B974
:10DC6000016809200860184610BD496852680068BC
:10DC7000984710BDF00C002064000020F40C002038
:10DC800038B504460378114811490268934205DB10
:10DC90000B68092119604FF0FF3514E00D4A0C2084
:10DCA00000FB03229568EB692BB108685268616834
:10DCB0009847054604E00B68092119604FF0FF35CD
:10DCC000204615F0D1F9284638BD00BFF00C0020E1
:10DCD00064000020F40C002010B50446C012FFF7C9
:10DCE00029FF0849024610B183681B6A23B90868F6
:10DCF00058220260002010BD086852686105490D75
:10DD0000984710BD64000020F0B50E4685B0074668
:10DD1000002835D001782F2932D1013016F052FA7F
:10DD2000044628B96846194916F0B4FB3C460EE093
:10DD3000C51B0C2D24DC012D22D02A46684639460D
:10DD400015F00CFA04A84519002305F8103C00252D
:10DD500009E02846FFF7EEFE01466846096816F01E
:10DD6000E9F920B10135FFF7F9FE8542F1DBFFF754
:10DD7000F5FE854204D0627812B10134346001E0CE
:10DD80004FF0FF35284605B0F0BD00BF28720308EC
:10DD90002DE9FF410546084603A91F469046FFF7B7
:10DDA000B3FF431C044602D113232B6014E0FFF79A
:10DDB000C1FE81680E6826B9582028604FF0FF30F8
:10DDC0000AE0426803990092284642463B46B04723
:10DDD0000028A8BF40EAC42004B0BDE8F08138B5EF
:10DDE0000446C8120D46FFF7A5FE83685B6802462D
:10DDF00023B9582020604FF0FF3038BD6905204618
:10DE0000490D5268984738BD022904D84FF4005391
:10DE1000536000207047582101604FF0FF30704779
:10DE20002DE9F3410546C8121F460E469046FFF7FE
:10DE300081FE83681C6924B9582028604FF0FF30A8
:10DE400007E04268710500922846490D42463B466C
:10DE5000A047BDE8FC812DE9F3410546C8121F46E5
:10DE60000E469046FFF766FE8368DC6824B95820AA
:10DE700028604FF0FF3007E04268710500922846A5
:10DE8000490D42463B46A047BDE8FC812DE9F341E0
:10DE90000546C8121F460E469046FFF74BFE8368A4
:10DEA0009C6824B9582028604FF0FF3007E0426892
:10DEB000710500922846490D42463B46A047BDE801
:10DEC000FC8173B50546084601A91646FFF71CFFFD
:10DED000421C02D113222A6010E0FFF72BFE0346FA
:10DEE0008068446A24B901232B604FF0FF3005E0BD
:10DEF00001995B68284601393246A0477CBD000085
:10DF00000A460349034608681946FFF7DABF00BF0F
:10DF100064000020012070470020704758230360F0
:10DF20004FF0FF307047FEE74FF0FF3070470000C2
:10DF30002DE9F041061E1DDB124D134F2B6823B94E
:10DF40003868F3F7C5FB2860C0B128680D4C0E4D4A
:10DF500000EB06083868F3F7D5FB804505D92A6839
:10DF60000027511C27602960E6E720688619266093
:10DF7000BDE8F0814FF0FF30BDE8F0814FF0FF3099
:10DF8000BDE8F081B80D0020B40D00200846F4F77C
:10DF900069BA08461146F5F75BBB0846F5F74AB97A
:10DFA00008461146F5F770BB2DE9F84F3C4F9B46EC
:10DFB0003B6814462BB13B4D2A68A9460AB1022999
:10DFC00001D9092302E0002961D0162303604FF034
:10DFD000FF3561E0344B1E68721C9A4603D04FF047
:10DFE000FF30186008E0D9F8006030494FF0FF308A
:10DFF000B047064601304FD0082E01D07F2E0FD1FA
:10E00000002D45D03B6801200821984701202021A0
:10E010003A6890473B6801200821013D984737E066
:10E02000234B1A689019417811F0970F05D11A2ED9
:10E030002ED8204911FA06F32AD51A2E2BD05FFAD2
:10E0400086F801203A68414690470D2E01D00A2EED
:10E0500019D10021D9F8003042F210709847861982
:10E06000172ECAF8000003D10F494FF0FF300860A7
:10E07000C8F1170C3B6801205FFA8CF198470A221F
:10E080006255013508E004F80580013500E00D46D1
:10E090005D459FD300E000252846BDE8F88F00BF0E
:10E0A000BC0D0020C00D002054000020FFFF0F0019
:10E0B00060000020200024002DE9F8439846154B0D
:10E0C00015461A680C46994622B1134A17680FB1D3
:10E0D000022901D9092306E00139012902D847465E
:10E0E000002612E0162303604FF0FF370FE0A85D13
:10E0F0000A2804D1D9F8003020460D219847A95D9F
:10E10000D9F800202046904701364645EFD13846E1
:10E11000BDE8F883BC0D0020C00D0020014B186045
:10E12000704700BFBC0D0020014B1860704700BF56
:10E13000C00D00200248034A0021FFF7BFBC00BF0A
:10E140007EAC030884AC030800290ADD4A1EC168BE
:10E15000224B806801EBC201814234BF0846184659
:10E1600070471F4B994203DB806800EBC10070478A
:10E170001C4B994209D00133994203D09A1E914217
:10E1800015D112E00069683070474369164A5B6830
:10E190005968914203D11B680BB1DB6800E0836CC6
:10E1A00012490365416550307047483070474369F4
:10E1B0000D4A5B68586890420BD11A684AB10C4806
:10E1C00092F807C0431A634505DC991C02EBC100B5
:10E1D0007047024870470148704700BFC8B0030845
:10E1E000F1D8FFFFEFD8FFFF0800FFFF0700FFFF98
:10E1F000EED8FFFF4369826A934201D1806C704779
:10E200005B68054A5968914203D11B680BB1D86815
:10E210007047806C704700BF0800FFFF30B5164B99
:10E2200044689C4223D10368987950B100291EDDCF
:10E23000D87981421DDC881C03EBC00111600F48B6
:10E2400030BD00291C6915DD656AA94212DC03EBAB
:10E2500081000139036998681060E36953F821006F
:10E2600090F90520002AB4BF0069103030BD0020AD
:10E2700030BD002030BD00BF0800FFFF2B72030837
:10E2800038B504460D46FFF7B5FF0021024620468B
:10E2900003F065FB2B680C4A0361A1684A600860C3
:10E2A000A0680A4A00F10803A3606968C26081603F
:10E2B000A168204601F1080300220839A360BDE8E7
:10E2C000384003F027B800BF0800FFFF0400FFFF3D
:10E2D00006C903F01FB8D1E9002310B58468C4E96A
:10E2E000002383680833836010BDB1F5FA5F38B549
:10E2F000044618DC8268C368D51A01EBE505B5F55C
:10E30000FA5F10DC002910DDC569AA1ACD00AA4207
:10E3100001DC02F035FD6269A16890684D19A842E0
:10E3200005D2956001E0002038BD012038BD0120F4
:10E3300038BD884270B513D08468D300E31A836077
:10E3400000230BE0866806EBC3048E6806F108051F
:10E350008D60D4E90045C6E9004501339342F1DB05
:10E3600070BD808E888670470369186E1966704785
:10E3700010B501694A6C0B6C9A42044601D304F053
:10E3800077F9204606F082FEA368034918605960B9
:10E39000A2680832A26010BD0A00FFFF8268C3684D
:10E3A000D01AC0107047000000290CDBC90003E040
:10E3B000084A5A6008338360C268836852189342DF
:10E3C000F6D38260704783684A1C03EBC201816008
:10E3D000704700BF0000FFFF10B50446FFF7B4FE12
:10E3E00004E0D0E90223C0E900230846A36800F155
:10E3F00008018B42F5D8083BA36010BD10B5044658
:10E40000FFF7A2FEA16803E051E9022361E80223BD
:10E410008142F9D8A368D3E90023C0E9002310BDE5
:10E4200038B5284B994204460D4606D14269816AA7
:10E430008A4202D1244902F0B1FA20462946FFF768
:10E4400083FE204B9D4211D16169204A4B68586878
:10E45000904201D1196821B920461D4902F09EFA67
:10E460002BE0A06850F8083CCB600FE0A36853E9AC
:10E470000223C0E900236369144A5B68596891422A
:10E480001BD11968C9B1134A954216DAA36833F94A
:10E49000020C421C11D133F904CCBCF1050F0CDD88
:10E4A00053F8082C92F805E05FEA8E7005D04B799E
:10E4B0005B0702D5204604F066F9A1680839A1601F
:10E4C00038BD00BFEFD8FFFFACAC03080800FFFF6A
:10E4D000C3AC0308EED8FFFF10B50446FFF734FEC7
:10E4E000D0E90023A168C1E90023A3680833A36031
:10E4F00010BD000008B5FFF727FE074B984206D075
:10E50000B0F906104B1C05D1B0F9040008BD4FF05E
:10E51000FF3008BD052008BDC8B003084B1C16BF5E
:10E52000024B034853F82100704700BF80B5030831
:10E53000EFAC030808B5FFF707FE084A43689342AB
:10E5400002D10168887938B9054AC2EB030CDCF1C5
:10E55000000343EB0C0008BD012008BD0800FFFFCD
:10E560000300FFFF07B5FFF7EFFDB0F9062001320A
:10E570000AD1B0F90430052B06D0694608F064FAD8
:10E58000003018BF012000E001200EBD08B5FFF7E4
:10E59000B1FF053801288CBF0020012008BD000014
:10E5A00008B5FFF7D1FD064A4368934205D0054AF6
:10E5B000991A484240EB010008BD012008BD00BF88
:10E5C0000900FFFF0400FFFF70B516460446FFF781
:10E5D000BBFD314605462046FFF7B6FD064B9D4282
:10E5E000014606D0984204D02846BDE8704004F0A9
:10E5F000F9BE002070BD00BFC8B0030870B5164654
:10E600000446FFF7A1FD314605462046FFF79CFD75
:10E61000064B9D42024607D0984205D02046294627
:10E62000BDE8704008F052BC002070BDC8B00308BF
:10E6300007B5FFF789FDB0F906200132034608D17E
:10E64000B0F90410052904D0694608F0FDF9034625
:10E6500010B1D3E9000101E00020002103B000BDAA
:10E6600007B5FFF771FDB0F906200132034608D166
:10E67000B0F90410052904D0694608F0E5F903460D
:10E6800018B1D3E9000122F0F3FD0EBD08B5FFF784
:10E690005BFD436813F5803F07D0064A934206D1DD
:10E6A0000068003018BF012008BD002008BD01200F
:10E6B00008BD00BF0100FFFF70B50D4616460446B9
:10E6C000FFF742FD134B42689A42014613D02046A1
:10E6D00008F054FA10B9D6B1306070BD2269506CA0
:10E6E000116C884202D3204603F0C2FF294620461F
:10E6F000FFF72AFD014616B10868C3683360086851
:10E7000090F905100029B4BF0069103070BD304683
:10E7100070BD00BF0600FFFF38B50546FFF714FDCA
:10E72000B0F906300133044619D1B0F90420911E26
:10E7300007291CD8DFE801F00E1B1B1304091B0678
:10E74000036812E00068006938BD0068BDE8384021
:10E7500007F07ABC0068BDE8384007F0CFBC284617
:10E76000214608F00BFA18B12368D86838BD00209C
:10E7700038BD08B5FFF7E8FCB0F9063001330AD11F
:10E78000B0F90430042B04D0092B06D100681830EE
:10E7900008BD006808BD002008BD002008BD0000BD
:10E7A00008B5FFF7D1FC034B42689A420CBF0068E2
:10E7B000002008BD0A00FFFF38B505460C46FFF7EC
:10E7C000C3FCB0F90630013313D1B0F90420911E17
:10E7D000082910D8DFE801F00B0B050F0F0B0B0514
:10E7E0000B0028462146BDE83840FFF7C2BF00684D
:10E7F00038BD002038BD002038BD00008168034AC4
:10E800004A60836808338360704700BF0000FFFFE1
:10E810008168C1E90023836808338360704738B595
:10E8200004468568084622F023FAC5E90001A3687A
:10E830000833A36038BD0000F8B50F4601691646DD
:10E840000B6C4A6C9A42044601D303F011FF324626
:10E8500020463946A56806F023FE034A28606A6010
:10E86000A0680830A060F8BD0600FFFF38B5044678
:10E870000D4619B9BDE83840FFF7C0BF084616F08D
:10E88000ABF8294602462046BDE83840FFF7D4BF22
:10E8900070B50E46016915460B6C4A6C9A420446E7
:10E8A00001D303F0E5FE204631462A46BDE870401C
:10E8B00004F002BE0EB417B501694A6C0B6C9A42A3
:10E8C000044601D303F0D4FE06AA2046059901921E
:10E8D00004F0F2FDBDE81E4003B07047F8B50C46E9
:10E8E000016917460B6C4A6C9A42064601D303F045
:10E8F000BFFE3046FFF77EFC39460246304603F045
:10E900002EF80461B168FB00CA1AB26008E0B5686D
:10E91000EC18D4E90045013F00EBC702C2E9064507
:10E92000083B002FF3D1B368034918605960B06801
:10E930000830B060F8BD00BF0800FFFF8368054ADB
:10E94000003118BF012119605A6083680833836061
:10E95000704700BF0100FFFF8368034A19605A60D7
:10E9600083680833836070470400FFFF8368034AAD
:10E9700019605A6083680833836070470200FFFFA4
:10E980008368034A19605A6083680833836070475C
:10E990000300FFFF8368064A18605A6081680269B5
:10E9A00008318160136F191A484240EB010070472B
:10E9B0000A00FFFF10B50446FFF7C6FBA268083A3D
:10E9C000014613462046BDE8104008F0FDB800009F
:10E9D00073B504461646FFF7B7FB637943F0080C9E
:10E9E00084F805C00546304615F0F6FF314602466C
:10E9F000204606F055FD6179074A009021F0080095
:10EA000001926071A368204629466A4608F0DCF846
:10EA1000A3680833A3607CBD0600FFFF10B5044661
:10EA2000FFF792FB094B4268A16800689A42A1F186
:10EA3000080102D107F016F801E007F057F8D0E915
:10EA40000023A16841E9022310BD00BF0700FFFFBA
:10EA500038B515460446FFF777FB0A4B4268006855
:10EA60009A42294602D106F093FF01E006F0BAFF70
:10EA7000D0E90023A168C1E90023A3680833A3609B
:10EA800038BD00BF0700FFFFF8B50F460169164605
:10EA90000B6C4A6C9A42044601D303F0E9FD3246FE
:10EAA00020463946A56806F011FF034A28606A60CF
:10EAB000A0680830A060F8BD0700FFFF38B5044625
:10EAC000FFF742FBC28813B2013310D1B0F9043012
:10EAD000072B04D0092B02D0022B08D102E00068DA
:10EAE00085680FE000680EF057FE05460AE012B296
:10EAF000013208BFB0F90430216918BF052324335F
:10EB000051F8235028466DB10EF0A8FEA3681D6091
:10EB100008B1054A00E0054A5A60A3680833A360BB
:10EB2000012038BD38BD00BF0200FFFF0700FFFF16
:10EB300010B50446FFF708FBB0F90630013314D1D5
:10EB4000B0F90430A168092B03D00A2B07D0082B99
:10EB50000BD103680848DA6848600A6008E000687A
:10EB6000D0E91223C1E9002302E0A2680349516001
:10EB7000A3680833A36010BD0700FFFF0000FFFF7C
:10EB800010B50446FFF7E0FAA3680146A3F11002AE
:10EB90002046083B08F0B0F8A368103BA36010BD06
:10EBA000F8B504461746FFF7CFFA0646384615F083
:10EBB00013FF394602462046A56806F071FC084955
:10EBC00028606960A26802F10800A060A2F1080351
:10EBD0002046314608F090F8A368103BA360F8BDCA
:10EBE0000600FFFF70B50446FFF7AEFA6379A6682A
:10EBF00043F0080305466371A6F110022046296818
:10EC000007F0BEF956E90223C0E90023637923F037
:10EC100008036371A36833F9022C01320FD133F971
:10EC2000042C052A0BDD53F8080C43799A0706D00B
:10EC300029684A79530702D5204603F0B6FDA1683A
:10EC40001039A16070BDF8B504461746FFF77CFA8D
:10EC50006379A66843F00803054663713A46204687
:10EC6000296806F06DFF56E90223C0E900236379A5
:10EC700023F008036371A36833F9022C01320FD12A
:10EC800033F9042C052A0BDD53F8080C43799B0754
:10EC900006D029684A79500702D5204603F085FD41
:10ECA000A1680839A160F8BD38B50446FFF74CFAF1
:10ECB000A36853F8042C12F5803F08D023498A42F8
:10ECC00053F8082C01D1002303E0012301E00023C5
:10ECD0001A46C1880DB2013528D1B0F90450072D6C
:10ECE00002D0092D22D10EE001688A604AB343BBED
:10ECF0005379990725D001684879420721D52046E4
:10ED000003F053FD1DE001688A60D2B1CBB992F8DF
:10ED100005C05FEA8C7314D0016891F805E05FEAE2
:10ED20004E700ED5204603F02EFD0AE009B20131E7
:10ED300008BFB0F90430256918BF0523243345F80E
:10ED40002320A268083AA260012038BD0700FFFF17
:10ED500010B50446FFF7F8F9B0F90630013323D1B6
:10ED6000B0F90420A368092A03D00A2A06D0082A89
:10ED70001AD1026853F8081CD16005E053F8081C4A
:10ED800002680D4B9164D364A26852F8082C92F883
:10ED900005C05FEA8C7309D001684879400705D542
:10EDA000204603F0F0FC01E0002000E00120A36811
:10EDB000083BA36010BD00BF0700FFFF38B58368A4
:10EDC000C943154603EBC101044602F0A3FA6A1CCD
:10EDD00005D16069A26881688A4228BF826038BD17
:10EDE0007FB504460E4615462BB11946FFF7ACF920
:10EDF000236AC01A00E01846A168236A0090F6430F
:10EE000001EBC60620460849029602AAF31A0395AA
:10EE100002F0FEFA691C05D16369A26899688A420A
:10EE200028BF9A6004B070BDD1E2000830B585B04B
:10EE30008568036A0392002202910092034902AAA4
:10EE4000EB1A02F0E5FA05B030BD00BF81E2000820
:10EE5000F0B50A4C87B00F4616460546002B18BF82
:10EE60001C4669463A46334608F0CAFF28466946BA
:10EE7000224602F0FFFA07B0F0BD00BF81BF0308D1
:10EE800037B5134682680C4652F8045C07498D4238
:10EE900009D152F8082C917929B9009111692246BB
:10EEA00002F032FD00E001203EBD00BF0800FFFF80
:10EEB0008079704770B50446056909294ED8DFE8A6
:10EEC00001F005090F1214183134374AAB7D43F0B5
:10EED000010302E0A87D20F00103AB75002070BDA6
:10EEE00003F01BFCFAE7686C36E06A6C9105880D4C
:10EEF00070BD95F816C01CF0010332D16E6C900203
:10EF0000B0429ABFC0EB060028642B6405E020469F
:10EF100003F0AEFB6B7D002B25D0296C6A6C91420F
:10EF2000F5D9DBE7686D6A6570BDA86DAA6570BD2F
:10EF300096020DD06B6C9E420AD203F0EEFB6B6C16
:10EF40009E4205D203F5806020F47E7626F0070607
:10EF5000AE64B00A70BDA86C800A70BD4FF0FF307F
:10EF600070BD012070BD012070BD08B501F0E0FC4E
:10EF7000002008BD10B50446FFF7E6F80B4A4168CB
:10EF800003469142A26819682046A2F1080202D104
:10EF900006F00CFC01E006F08DFCA36810B108330C
:10EFA000A36010BD083BA36010BD00BF0700FFFFBA
:10EFB000012970B504460D4616DD01694A6C0B6CDB
:10EFC0009A4201D303F054FBA068E268811ACB1087
:10EFD000204629465A1E08F001F8A068EA00C2F14E
:10EFE00008054519A56070BD51B9064986682A46CD
:10EFF00006F056FA044930607160A3680833A360D4
:10F0000070BD00BF2B7203080600FFFF03691A6181
:10F010000369D9607047000038B50D4601694A6C34
:10F020000B6C9A42044601D303F022FB2046FFF703
:10F03000E1F829460246204606F06FFAA368044923
:10F0400018605960A2680832A260183038BD00BF4D
:10F050000900FFFF37B515460446FFF775F8294646
:10F0600001AAFFF7DBF840B1019BA168D3E90023B7
:10F07000C1E90023A3680833A3603EBD73B51546FC
:10F080000446FFF761F8294601AA0646FFF7C6F8CD
:10F090000546E0B1A3680199A3F10802A26053E913
:10F0A0000223C1E90023A368B3F9062001320ED17F
:10F0B000B3F90420052A0ADD1A6853799B0706D0A4
:10F0C00031684879400702D5204603F05CFB2846AA
:10F0D0007CBD0378052B09D101694B1C08D143691C
:10F0E000A3F1FF32504240EB02007047002070470E
:10F0F00000207047CA0506D490F83230994202DBEE
:10F10000426A511E416270470B780C2B02D189680C
:10F11000FFF7F0BF7047000070B5CE439619056841
:10F1200086EAE673A3EBE673B3F5003F0C46ED68A1
:10F1300003DBC068064903F0F7FC55F824000549D5
:10F1400083047218990C41EA823045F8240070BD9E
:10F15000F8AC0308FFFF01002DE9F7430546D0F89E
:10F1600010800C46164640462246696806F008FFA5
:10F17000B0F906302C6801338146A76A04D0D0E983
:10F18000000122F075F83FE0A86A21F071FDC9E99D
:10F190000001AA6AA36A9A420BDB1C491C48009131
:10F1A0000190A168404604F12802082304F0A8F861
:10F1B000A060FB0004E0D218164801375060083305
:10F1C000A16AA2688F42F6DBA96A02EBC101D6E907
:10F1D0000023C1E90023B6F90630013311D1B6F995
:10F1E00004C0BCF1050F0CDD326892F805E05FEA5F
:10F1F0008E7006D06379590703D54046214603F047
:10F20000C2FAA86A421CAA62BDE8FE83FFFF03009F
:10F2100013AD03080000FFFFC06850F82120044828
:10F22000930B1818431C01D001310818704700BF18
:10F230000100FEFFC068002900EB810008DD10F826
:10F2400004CC044A0CF03F015356002BB8BF0438DD
:10F25000704700BFE9B1030870B506460C460EE0E2
:10F26000356821462846FFF7E5FF007800F03F03A8
:10F270001B2B08D121462846FFF7CEFF0446621C0F
:10F28000EED1002070BD012070BD000010B50068F7
:10F290001446FFF7CFFF036803F03F021B2A16D185
:10F2A000FF2C09D0B4EBD35F06D0A40123F47F5325
:10F2B00004F47F54234307E0064A03EA020E4EF0AB
:10F2C0001A0CD90D4CEA81130360012010BD0020F7
:10F2D00010BD00BF00C07F0038B505460C4609E0F0
:10F2E0002146FF222846FFF7D1FF21462868FFF775
:10F2F00093FF0446611CF3D138BD2DE9F843089F04
:10F3000005460C461646984614E021462868FFF745
:10F3100083FF2146814642462846FFF7B7FF18B1D2
:10F3200028462146324602E0284621463A46FFF763
:10F33000F3FE4C46601CE8D1BDE8F883F7B51646ED
:10F340008269056800920446FF230F46016AFFF7B1
:10F35000D4FF4FF0FF302062A269EB6A9A420BDBC8
:10F36000134A1449009201912069E96805F12C02C1
:10F37000042303F0C5FFE860A169EA6842F8217040
:10F38000A0692B6B98420BDB094B0A480093019054
:10F390006969206905F13002042303F0B1FF686157
:10F3A0006869A26940F82260A069411CA161FEBDA4
:10F3B000FDFFFF7F2BAD030808B50068FFF73AFF9C
:10F3C00001688B0913F0FF0F21F47F5214BF002155
:10F3D000402141EA0203036008BD8369C361184606
:10F3E0007047531C70B50446164612D00D68681C51
:10F3F00002D10A6070BD054620682946FFF70CFF60
:10F40000431CF8D1204629463246BDE87040FFF73C
:10F4100083BE70BD38B505460C46FFF7DEFF2846B3
:10F4200005F120012246BDE83840FFF7DABF13B5E9
:10F430008469A24204D102B0BDE81040FFF7EABFE0
:10F44000FF230092FFF759FF02B010BD38B5456A9F
:10F450004D19016891F84B309D42044608DDF92DA5
:10F4600003DDC068034903F05FFB206880F84B5060
:10F4700038BD00BF3EAD030838B504460D46FFF762
:10F48000E5FF636A5D19656238BD000007B5044B8E
:10F4900000916A4669460193FFF75EFE0EBD00BF0C
:10F4A0000600FFFF07B502A961E9022369466A4623
:10F4B000FFF752FE0EBD000070B50C780D2C11D177
:10F4C00000688D68C0681A49531C9A0350F82530AB
:10F4D00023F4FE0C11402CF4404241EA020340F8B0
:10F4E000253070BD0E2C21D105688E68ED6855F869
:10F4F000263023F07F44013224F4000C4CEAC2533E
:10F5000045F8263002688968D268436A52F821407B
:10F510009B0124F47F5403F47F5C44EA0C0342F81B
:10F5200021300121BDE87040FFF7A6BF70BD00BFCC
:10F5300000C07F000B780D2B0AD10C230B700268E2
:10F540008868D36853F820209009C3B28B60704755
:10F550000E2B0ED102688868D26852F8203023F052
:10F560007F4323F4000C4CF0807342F820300B20D2
:10F5700008707047036880695B69421E43F8221077
:10F58000704710B5C46841EA8212029942EAC35337
:10F59000A26843EA8131BDE81040FFF7CFBEF7B55E
:10F5A0000D46144606461F46FFF717FF3046022158
:10F5B0002A4623460097FFF7E4FFFEBD13B5531C10
:10F5C0000C46002200921E212246FFF7DAFF1CBDE6
:10F5D000F7B58569C3699D420C4624DD25B990F8CD
:10F5E00032C061451FDB26E00168013DCE6856F858
:10F5F000251001F03F03032B15D18B095FFA83FC23
:10F60000A44510DCCF0D7B1C9C420CDCA218013AF7
:10F61000BA4210DD21F07F4323F4000141EAC250D9
:10F6200046F8250007E0A318002200920321224695
:10F63000013BFFF7A6FFFEBD10B59C0344EA821311
:10F64000C468A2681943BDE81040FFF777BE37B51C
:10F650000A78931F05460C46082B2BD8DFE803F0E9
:10F6600005080C122A2A2A2525000C20087021E002
:10F6700000220092042111E005210022A368FFF777
:10F68000DBFF0EE0C968FFF735FD2846A168FFF7EC
:10F6900031FDE1682846009100220621A368FFF7AA
:10F6A00070FF0B23A060237004E003B0BDE830407E
:10F6B000FFF740BF03B030BD73B50D461446064694
:10F6C000FFF7C5FF2B785A1E0B2A45D8DFE802F05A
:10F6D000060C0C181D444444444429383046214645
:10F6E0000122FFF775FF34E00221C1EB030E002079
:10F6F000DEF1000300902246304643EB0E0326E085
:10F70000304601212246AB6808E0D5E902233046A5
:10F71000FFF7C8FE0121034622463046FFF78CFF63
:10F7200017E03368AA68DB6853F82200A10101F4EE
:10F730007F5E20F47F5C4EEA0C0143F8221008E063
:10F74000AB689C4205D00021009130462246FFF76D
:10F7500018FF0C22AC602A707CBD38B50B780C2BDE
:10F7600005460C460AD00121FFF786FE6A6A284644
:10F770002146013ABDE83840FFF79EBF38BD000082
:10F7800037B54FF0FF33056A036216210022064B9E
:10F790000446FFF751FF02A92A4641F8040D20460E
:10F7A000FFF71FFE01983EBDFEFF010037B5069D25
:10F7B00004460095FFF7E5FE204603B0BDE8304063
:10F7C000FFF7DEBF73B50B780B2B04460D461646CC
:10F7D00014D103688A68DB6853F8222002F03F01E5
:10F7E00013290BD18369591ED6F1010638BF0026B3
:10F7F0008161D20D00961A2100230CE02046294693
:10F80000FFF7ABFF20462946FFF77EFCAB6800966A
:10F8100020461B21FF22FFF7C9FF7CBD38B50C46EF
:10F820000546FFF714FF2078831E082B0CD8DFE86D
:10F8300003F0120B12120B0B0B0B05002846A168EC
:10F84000FFF7BAFDA26808E0002228462146FFF72C
:10F85000B9FF024601E04FF0FF32284604F11401DF
:10F86000FFF7BFFD21692846FFF7D4FD4FF0FF31B8
:10F87000216138BD2DE9F7430C4605461646FFF7D2
:10F880001BFF23780A2B05D1284604F11001A2683A
:10F89000FFF7A7FD21696769B9423BD02846FFF70A
:10F8A000DBFC20B928463946FFF7D6FCE0B12078CA
:10F8B0000A2804D02846FFF763FF804601E04FF096
:10F8C000FF383146002201232846FFF768FE314603
:10F8D0008146012228460023FFF761FE4146074684
:10F8E0002846FFF797FD02E04FF0FF37B94628465C
:10F8F000FFF773FD80466169CDF8009028464246C7
:10F900003346FFF7FAFC2846216900974246334602
:10F91000FFF7F3FC4FF0FF320C2122616261A66019
:10F920002170BDE8FE8338B504460D46FFF78FFE13
:10F9300020462946FFF7E8FB20460121FFF79CFD02
:10F94000626A20462946013ABDE83840FFF792BF77
:10F9500038B50C460546FFF77AFE23780C2B10D1FC
:10F96000226960698242A26801D1104638BD95F8CB
:10F9700032108A4205DB28462146FFF77BFFA0684C
:10F9800038BD28462146FFF7CEFFA06838BD0A697A
:10F990004B699A4201D0FFF7DBBFFFF758BE00006A
:10F9A00030B50C4685B00546FFF7F1FF23785A1EA7
:10F9B000042A32D8DFE802F00303032B0300A86A0D
:10F9C000FF282ADC012B09D1174A6968174B0392DB
:10F9D000009101932846694602AA12E0052B05D141
:10F9E0002846D4E90223FFF75DFD0CE0A3F10202F3
:10F9F00051420F4841EB020302A9039002932846AB
:10FA00000A46FFF7A9FB0423A060237002E0A06868
:10FA1000FF2802DC40F4807003E028462146FFF70F
:10FA200097FF05B030BD00BF0000FFFF0700FFFFDC
:10FA30000100FFFF2DE9F04F85B007461046039106
:10FA400016469946FFF745FB002871D04846FFF758
:10FA500040FB00286CD0039AB468F568A2F10C034F
:10FA6000D9E902AB082B4FD8DFE803F0050C1118D9
:10FA700027424B4E65002046294652465B4620F001
:10FA8000ABFF3BE02046294652465B462DE0204630
:10FA9000294652465B4621F051F92FE0504659461F
:10FAA0000022002321F0B2FB002844D12046294641
:10FAB00052465B4621F06CFA20E05046594600223F
:10FAC000002321F0A3FB002835D152465B46204697
:10FAD000294621F05DFA22F03FFC52465B4621F0B8
:10FAE0002DF902460B462046294620F073FF05E01B
:10FAF0002046294652465B4623F0B0F804460D46A0
:10FB000004E005F1004501E0002425462046294691
:10FB100022462B464FF0010821F078FB00B98046C1
:10FB200018F0FF0F04D022462B46C6E902232BE033
:10FB30000398122808D00399142905D0384649465D
:10FB4000FFF72EFF054600E0002538463146FFF757
:10FB500027FFA8420446384605DD3146FFF7D4FAB0
:10FB60003846494604E04946FFF7CEFA3846314662
:10FB7000FFF7CAFA23463846039900950022FFF79B
:10FB800000FD0B23B060337005B0BDE8F08F2DE9A8
:10FB9000F3470E461946054690461C46DDF828A058
:10FBA000FFF7FEFE514607462846FFF7F9FE51468D
:10FBB00081462846FFF7A8FA28462146FFF7A4FA0F
:10FBC000B8F1000F06D1172E04D03B464FF00108C4
:10FBD0004F4699462846314642463B46CDF800906E
:10FBE000FFF7E4FDA0600A202070BDE8FC87F7B5B0
:10FBF000044615461F460E297DD8DFE801F055570B
:10FC0000595B5D5F2969666C6F737608170039462A
:10FC1000FFF71DFD20466A6907F114013C46FFF716
:10FC2000E0FB0FCC0FC594E803000EE0394607F166
:10FC30001006FFF70CFD20462A6931463C46FFF7C7
:10FC4000D0FB0FCC0FC596E8030085E8030052E017
:10FC50003946FFF79CFE3E780B2E20461DD12168C9
:10FC6000BA68CB6813F8221001F03F03152B14D1AA
:10FC70002946FFF749FA2268B968D26852F821008C
:10FC800020F07F43A86823F4000C4CEAC05342F8EC
:10FC900021302E70B868A8602DE03946FFF743FE8A
:10FCA000204615212A460AE00C2108E00D2106E035
:10FCB0000E2104E00F2102E0102100E011213B465B
:10FCC00003B0BDE8F040FFF7B5BE0097172107E08D
:10FCD000009717210BE00097182101E000971921E8
:10FCE000012205E00097182101E000971921002268
:10FCF0002B46FFF74CFF03B0F0BD38B50546144660
:10FD00000E293DD8DFE801F0353535353535303C45
:10FD10003C3C3C3C3C080D001146BDE83840FFF738
:10FD20007DBD1146FFF793FC2378032B0DD00A2BE2
:10FD300002D0012B02D108E0A26808E00122284687
:10FD40002146FFF73FFD024601E04FF0FF32284613
:10FD500004F11001FFF745FB28466169FFF75AFBE4
:10FD60004FF0FF33636138BD1146BDE83840FFF7FF
:10FD7000DABD1046FFF7ADF938B92846214600E054
:10FD80001146BDE83840FFF70BBE38BD10B50C4634
:10FD90001146FFF705FE0923E060237010BD30B562
:10FDA00089B0052314464FF0FF32079206928DF872
:10FDB00008300022002301290546CDE904230ED096
:10FDC00002D302294AD140E02046FFF782F918B950
:10FDD00028462146FFF7BCFD284612213AE021467D
:10FDE000FFF735FC2178481E0B2822D8DFE800F009
:10FDF0000608060808212121210A0F0F022317E017
:10FE0000032315E02846A168FFF7D6FA11E028463B
:10FE10002146FFF7A2FC28462146FFF775F900228C
:10FE2000A368009228461321FFF7ABFB0B23A060C9
:10FE3000237021696369616128462361FFF74CFAE9
:10FE400028462169FFF748FA08E02146FFF780FDC0
:10FE500028461421224602ABFFF7ECFD09B030BD65
:10FE60002DE9F34104460D461746FFF771FD204684
:10FE70002946FFF749F920460221666AFFF7FCFA96
:10FE800039462046D5F80880FFF78AFD43460090A2
:10FE90000B2132462046FFF774FB20463946FFF718
:10FEA00033F90C23AE602B70BDE8FC8173B50E46B0
:10FEB00009788B1F04461546032B2CD8DFE803F086
:10FEC000020D17212946FFF71FF9B268204629467F
:10FED00002B0BDE87040FFF7CDBC2946FFF738FD02
:10FEE00002460020009008212046B36811E0294610
:10FEF000FFF72EFD07210246B3682046FFF79CFB63
:10FF000009E02946FFF74CFDB268F368009009212B
:10FF10002046FFF736FB2046294602B0BDE8704078
:10FF2000FFF7F2B873B5013A0D46322192FBF1F6B4
:10FF30000136B3F1FF3F08BF0023B6F5007F04464A
:10FF400005DA22212A460096FFF71BFB0BE0002270
:10FF5000009222212A46FFF714FBE368204631462F
:10FF60009A68FFF7EBF9013565627CBD10B54B6807
:10FF70000F4A5C68944214D11A689279A2B9426916
:10FF8000914204BF8269CA60C868094A59689142AF
:10FF90000CBF1B6800231A69D368C11A8810013886
:10FFA00010BD4FF0FF3010BD4FF0FF3010BD00BF4F
:10FFB0000800FFFF38B50C46FFF7D8FF051E13DB1E
:10FFC00063680B485A6882420CBF186800200169B8
:10FFD000486958B106498A420CBF1B6800231A6958
:10FFE000536953F8250038BD4FF0FF3038BD00BFCE
:10FFF0000800FFFF022A07D0032A0CD0DAB9D1F19A
:020000040801F1
:10000000010038BF0020704790F84B008142ACBF20
:10001000002001207047CB0504D5836A21F480714C
:10002000994202E090F84B008142B4BF00210121C7
:1000300081F0010070470120704700004268064BC4
:100040009A4204D10368987918B91869704700205A
:1000500070470020704700BF0800FFFFF8B5064654
:1000600048680C461546FFF7E9FF074648B12146A8
:100070003046FFF77BFF29460246384601F09AFDDD
:1000800078B97069226884420CBFB068E069831A4D
:10009000B5EBE30F04DC0348002DD8BF0020F8BD0A
:1000A0000020F8BD61AD0308CA0511D503680A4AEE
:1000B00021F4807103EBC100406890420AD153F8EB
:1000C000310090F90530002BB4BF00691030704743
:1000D00002487047014870470600FFFF81BF0308D0
:1000E00019B1002A08BF002100E00A464164C36339
:1000F000036480F8382001207047406C704790F806
:1001000038007047C06B704770B543690FE05C689A
:10011000124E65680139B54208D00536B5420CBFAC
:1001200024680024A4790CB95C69091B183B0029D8
:1001300004DD846AA342EAD8002070BD09D1806A38
:10014000834204D91B1A0648DB10434302E00846E9
:1001500070BD00231366012070BD00BF0300FFFFC8
:10016000ABAAAAAA2DE9F0410B6E866A18255D4359
:10017000711904461746FFF771FF804630B1725976
:10018000791E204602EBC101FEF7A5F84046BDE806
:10019000F081F8B50B6E856A18245C432919064670
:1001A0001746FFF75BFF38B1B1682A5951E902459C
:1001B00002EBC70747E90245B368083BB360F8BDE7
:1001C00000F03F031C3B062B08D84FF062429A40D8
:1001D00004D5C00D14BF00200120704700207047D7
:1001E0002DE9F04F07468BB097F84B90C06A089105
:1001F000B9F1FA0F1346029000F2B08197F84A0065
:1002000097F849100490049800F0010C01EB0C02DF
:100210004A4500F3A38100F00502042A00F09E8104
:1002200097F84810786A0791884200F397813A6BF3
:1002300002998A4202D0002A40F090810299002956
:1002400040F38C81481ED7F80CB005901BF8202095
:1002500002F03F0CBCF11E0F40F080811946DDF822
:1002600014A05B4600248B466FE103EB84060996DD
:1002700053F8246006F03F012529039100F26E81B6
:100280004FEA96125FFA82F8C84580F267819A4D6C
:1002900015F801C00CF00302012A23D0022A2CD049
:1002A000002A53D14FEA1C1EF50D384629460EF0A0
:1002B00003028DE80810FFF79DFEDDF804C000285A
:1002C00000F04D81B10BC8054FEA9C03C60D03F049
:1002D000030238463146FFF78DFE9DE808100028DE
:1002E00038D13CE14FEA1C1000F00302B50B032AA1
:1002F0002FD1B96A8D422CDB30E14FEA1C12B00BD2
:100300007E4D02F00306022E054422D1611C4E19D7
:1003100000F12481029A964280F22081D6B103EB4B
:10032000860006900020069951F8042D069102F0EF
:100330003F01222906D1920BD105CA0D12B9013015
:10034000B042F0DB10F0010604D007E1002635468C
:1003500000E000261CF0400F02D0D84508BFA2469E
:100360001CF0800F0DD00298A11C814280F2F68013
:10037000601C13F8202002F03F0CBCF1160F40F077
:10038000ED80039A911E232900F2DE80DFE811F050
:1003900024003C0043004600DC0046004300DC0033
:1003A000DC004F00DC00DC00DC00DC00DC00DC00FA
:1003B000DC00DC00DC0058006F00DC00DC00DC004E
:1003C000DC00DC007B007B0093006B006B005C00BA
:1003D0009900DC00A500C900012E40F0B58002980C
:1003E000A11C814280F2BA80621C53F8220000F006
:1003F0003F0CBCF1220F40F0A780810BC805C00D57
:10040000002840F0A180AAE0D84500F39D80AB45CC
:10041000D8BFA24698E0079A954212E0BA683849D8
:1004200002EBC5056868884200F08E8096E008F10E
:100430000108C84580F29280C34508BFA24683E008
:10044000B542C0F2818089E0002E00F0858008F17D
:10045000020C66444E4580F2818008F10108D845BF
:10046000B8BFA24670E008F10308C84576DABBF1D0
:10047000FF0F69D0601C4219944265DA08998A42DC
:1004800062DC641960E015B145444D4566DC721EBE
:1004900046B9621C53F822000093FFF791FE009BBF
:1004A00028B95CE01AB108EB0200484556DCC345A8
:1004B000A8BFA24648E0013D002D45DD45444D451D
:1004C00041E0002D02DD45444D4547DA002E3BD189
:1004D000059901348C4237DB3EE07A6B95423DDA78
:1004E0003969029A51F8250090F848002118914284
:1004F00034DA0122099E0DE0E9B103080100FEFF94
:100500000600FFFF56F8225005F03F05042D00D0ED
:1005100025BB01328242F5DDBBF1FF0F18BF0C464F
:1005200012E0049A02F0060CBCF1020F16D16E1E06
:100530003DB9601C53F820000093FFF741FE009B7B
:1005400068B1B044C84509DC013408998C42FFF613
:100550008CAE53F82A0002E0304600E000200BB0D9
:10056000BDE8F08F2DE9F84306460D46144698463F
:100570006B68384A5968914263D11B6898790028A2
:100580005FD1294630461F69FFF7F0FC8146611CA8
:1005900038464A4601F00EFBC8F80000002853D147
:1005A000384649462246FFF71BFE00F03F030B2B5F
:1005B0004DD8DFE803F0164C4C4C28061C4C4C4C34
:1005C0004C3A800BBA6852F83010234891F905C0B4
:1005D000BCF1000FB4BF09691031C8F80010BDE8C4
:1005E000F883C40DC0F38713A342C1DC29E0820B5A
:1005F000D10507F10800C90DFFF756FDC8F8000046
:100600001648BDE8F883FB694BB1C10D53F82130A2
:1006100093F905000028B4BF1B69103300E0104BAC
:10062000C8F800300F48BDE8F883820BD30507F106
:100630000800D90DFFF738FDC8F800000A48BDE8EA
:10064000F8830020BDE8F8830848BDE8F88300205F
:10065000BDE8F8830800FFFF6EAD030875AD030821
:1006600081BF03088AC003087BAD030875C0030877
:100670002DE9F04F0B783E2B85B005468946144690
:1006800012D18068874A01F1010950F8041C914297
:100690000BBF50F8086C50F8088C4FF0000800268B
:1006A0000838A86000270FE0166EC6B1836A7D483F
:1006B000182707FB06377B685E68864201D11E68F3
:1006C00005E0D3F800800026B8F1000F02D136B162
:1006D0004FF00008CDF80C904FF0010AA3E04FF066
:1006E000FF317148714A6161E16121627049A06026
:1006F0006060E260216104F124003C2202F0AAFF64
:10070000B046A6614FF0010A94E0662B00F08B80A2
:1007100006D84C2B00F08780532B40F0828006E0F7
:100720006E2B3ED0752B36D06C2B7AD129E0B8F1E8
:10073000000F01D1B3793BB15E4A5F4B22614FF0AC
:10074000FF31E161216214E03269116A91F905C05B
:10075000BCF1000FB4BF09691031216130695749FC
:10076000C06BE06133691A6C554B2262002808BFE8
:100770000B46E36004F1240021693C2202F06AFF89
:1007800051E027B128463946FFF714FC01E04FF04D
:10079000FF30606147E00EB1F37900E03346A361BA
:1007A00041E0002F36D07B683E495868884205D129
:1007B0001B68987910B97A69002A2CDC57F8143C28
:1007C00038495868884221D119688A79F2B908698C
:1007D000A7F11803D0F80CB00192194628460293ED
:1007E000FFF7C4FB5BF82010019A01F03F00A0F175
:1007F0001C03012B029B01D9212809D18A09284613
:100800001946D2B2231DFFF7ADFE04E0002002E03E
:10081000104600E03846A06028B923496060A16016
:1008200001E04FF0000A039810F8013B0390002B01
:100830007FF46BAF4846662113F0C4FCD8B1AB68B7
:1008400016B11E60174A07E0B8F1000F03D0C3F8D5
:1008500000801C4A00E01C4A5A60EA69AB68C3EB9E
:10086000020EBEF1080F03DC2846012100F088FAD1
:10087000A9680831A96048464C2113F0A3FC002860
:1008800043D00EB1B47914B1AB680F4A30E02846BA
:100890002146224605F01AF807463069D0F8148040
:1008A0001FE000BF0800FFFF2B72030887AD03089D
:1008B0008CAD030899AD03081CD6030882AD03086C
:1008C00019B603080300FFFF0000FFFF3946284662
:1008D00058F8042B05F034F90E4B012180E80A008A
:1008E00001343269136B9C42F0DBAB680A4A1F602B
:1008F0005A60EB69A868191A082903DC2846012107
:1009000000F03EFAAA680832AA60504605B0BDE879
:10091000F08F00BF0100FFFF0700FFFF08B5FF22B7
:10092000C16AFFF75DFC003018BF012008BD000060
:1009300038B5436E0446002B27D0056A164AED18D9
:100940006B68934205D0053A934202D0052100F02E
:10095000C7F9A16851E90223C1E90023D5E90023C1
:10096000A16841E90223E269A368D31A082B03DCDA
:100970002046012100F004FAA16801F10803A360F8
:1009800020460839012200F0C5FC20460221BDE8BE
:10099000384000F0A5B900BF0800FFFF0EB4F0B565
:1009A00092B017AA044652F8041B119202F084FD7B
:1009B0006769164A7B685968914206461DD11868D6
:1009C0008379D3B939462046FFF7F4FA05467868AB
:1009D000FFF734FB016A91F90520002AB8BF0969C5
:1009E00002A8A8BF10313C2202F034FE204608497C
:1009F000009602AA2B4602F021FE2046FFF798FF40
:100A000012B0BDE8F04003B0704700BF0800FFFF20
:100A10009EAD030810B51346B1F90640621CB3F948
:100A2000064008BFB1F904200C4918BF0522013463
:100A300008BFB3F9043051F8222018BF0523947879
:100A400051F8233099788C4203D10549FFF7A6FF6E
:100A500002E00449FFF7A2FF002010BD80B50308A3
:100A6000A8AD0308C9AD03087FB50446B1F9060077
:100A700000251646421C08BFB1F90420039518BF93
:100A800005220B46124951F8225061690A688868AC
:100A900002E0934203D008328242FAD311E0E268C6
:100AA0009B1ADA10204603ABFFF75CFD034640B10A
:100AB000039A08498DE8240020463246FFF76EFF6E
:100AC00005E02046044932462B46FFF767FF7FBD0D
:100AD00080B50308E7AD03080AAE030873B5054601
:100AE0000C4608466946164605F0AEFF044A002843
:100AF00014BF314621462846FFF7B6FF7CBD00BF34
:100B000023AE030810B5084B4C689C4206D0B1F9DF
:100B100006C0BCF1FF3F18BF114600E01146034A72
:100B2000BDE81040FFF7A0BF0600FFFF39AE030885
:100B300002392DE9F0410646174603291CD8DFE8A3
:100B400001F016160209046A0D49151B04EB05088D
:100B5000112205E0046A0B49151B04EB0508172256
:100B600004F09EFC084B6051C8F8043004E0806833
:100B700050E90245C2E900450837B760BDE8F08199
:100B80009CD1030845AE03080600FFFF00B59FB0E7
:100B90001EAB0392026E019043F8642D029103662E
:100BA000002106A81D9112F0FBFF18B901980399C6
:100BB000029B98470198059A02661D981FB000BDD8
:100BC000F8B5CB1D8F1DB3F1005F04460E46056AD4
:100BD00006D2C26A2946D200FB0002F079FB01E08E
:100BE00002F06EFBA3682062C5EB030C2CF007013A
:100BF00000EBC6064018E762E661A060A36D08E05E
:100C00009A68216AC5EB020E2EF007000A189A6056
:100C10001B68002BF4D1A36A20E053F8102C216A42
:100C2000C5EB020E2EF0070C01EB0C0053F8182C4C
:100C300043F8100C216AC5EB020E2EF0070C01EBF5
:100C40000C0053F8142C43F8180C216AC5EB020E63
:100C50002EF0070C01EB0C0043F8140C61691846E8
:100C600018338842D9D9E068236A421B22F007056D
:100C70005D19E560F8BD000070B50F4B866A4A1C2F
:100C80009A4204460D4607D8026B18235A43314650
:100C90006B4302F01DFB01E002F012FB6369256368
:100CA0009A1B22F00706013D18218619A06201FB5C
:100CB00005006661606270BDAAAAAA0A026B44F6CA
:100CC00020618A4208DD836A4269C3EB020C034B50
:100CD0009C4501DCFFF7D0BF704700BFE75207001B
:100CE00070B590F805C003692CF0080242719D7D33
:100CF00025F001029A75056E04460E462DB129664F
:100D0000006E0121043012F051FF03698171196EE8
:100D1000C1B1816A41610968C16000F0BAFE314623
:100D20002046E268FFF704FFE08E0122A08684F8E7
:100D300039202046FFF7C2FF6566256625692046F3
:100D40002E6EB047012010F013FD000038B5016B86
:100D500044F62065A942044602DD0521FFF7C0FFE5
:100D60004900FFF789FF236BAB4203DD20460349AF
:100D7000FFF714FE60691830606138BD5FAE03088C
:100D8000C36A994201DC590000E05918FFF718BF07
:100D90002DE9F041044608680E4607F020F80746A2
:100DA0002069426C036C9A4202D3204601F060FC39
:100DB0002369204993F816C01F4D4CF0010883F8B1
:100DC00016801B2F08BF0D46321D3168336920463F
:100DD000A8470546A26C95F84810204600F0D5FDBE
:100DE000002706460561804605E0204600F0F0FD3C
:100DF0000137C8F8100095F84820974208F1040818
:100E0000F3DBA0680D4A06604260E369A168581AE6
:100E1000082803DC20460121FFF7B2FFA2682369FE
:100E20000832A26093F816E02EF001019975BDE832
:100E3000F08100BFD16701087D4E01080800FFFF67
:100E400070B545692D680446856008460E4613F066
:100E5000C3FD31460246204604F022FB08492860C3
:100E60006960E269A068131A082B03DC204601219F
:100E7000FFF786FFA3680833A360022070BD00BFA0
:100E80000600FFFFF0B5456C9BB00446002D37D03F
:100E900090F83930002B33D0076A8368406901919C
:100EA000D0F808E006920429C7EB0306C7EB0E074B
:100EB00002D10022199205E0A16A421A1149D0100C
:100EC00048431990E069C3EB000CBCF1A00F03DCB0
:100ED00020461421FFF754FFA16862690023A03166
:100EE0009160204684F8393001A9A847226A6169D7
:100EF0000120D71984F839008F60236A9E19A660F3
:100F00001BB0F0BDABAAAAAA70B590F838309A070A
:100F1000044626D5056A4FF0FF324D1B0121FFF72D
:100F2000B1FF6069234943685A688A4217D04E1D51
:100F3000B2420CBF1B680023997931B10FE0204603
:100F400004214FF0FF32FFF79DFF94F838209307FC
:100F500005D561694B69581E4861002BEFD1266A9F
:100F600071196369A3F11800606153F8182C1869AE
:100F70005E68E26053F80C5CA561054604E0F1E8A8
:100F80000223E6E80223013D15B932462B4607E06D
:100F9000A3689942F3D3F8E70749013B42F8041CE0
:100FA0000832002BF8DC25EAE57506EBC506A660DD
:100FB000013070BD0300FFFF0000FFFF2DE9F74F78
:100FC000DFF86C824B680192434504460D462BD0F6
:100FD000954A934228D0102205F0E6F84368276A24
:100FE00043450646C7EB050704D0204629468F4AED
:100FF000FFF73AFDA16803E051E9022361E802230B
:10100000A942F9D8E569A168681A082803DC2046D6
:101010000121FFF7B5FEA368226A0833A360D51942
:10102000D6E90023C5E90023206A6A6861692B1AA2
:1010300000937F4BA0699A4208BF2B68C86018BF15
:101040000023002B00F0DD809D79002D40F0D98039
:101050001D69E269A76895F84B10D61BB6EBC10F66
:1010600002DC2046FFF78CFE206A009B95F84A10B0
:10107000C61859B995F84910A26806F1080707EB98
:10108000C1039A4240F28780A36084E0A06895F88B
:1010900049B0871BFE10013E05E0A368654A5A600F
:1010A0000833A36001365E45F7DB95F84A1011F06E
:1010B00004084FD023695F6C186C8742CBEB060A9B
:1010C00002D3204601F0D4FA01225146204604F012
:1010D000FDFBA3688046186057485860E769A1681F
:1010E0007A1A082A03DC20460121FFF749FEA76887
:1010F0006179083741F00802A7606271002710E0AB
:10110000A3686FEA0A0909EB0700013703EBC0097E
:101110003A462046414604F013FDD9E90023C0E9D0
:1011200000235745ECDB607920F008016171012252
:101130004249204604F0B4F941460246204604F0F4
:101140006BFF074650461FF093FDC7E90001A268F8
:10115000083AA260A768F600BE1B00230BE0A26855
:1011600002F10801A160F6E80201C2E90001314A7A
:10117000013346F8042C5B45F1DBB8F1000F07D0D2
:10118000A3682D4803F10806A660C3F800805860E4
:10119000226A009956186069636A984203D1204612
:1011A000FFF7D4FD01E01830606107604660E7603A
:1011B00095F84B2007EBC2078760EB68019AA361A3
:1011C000002141610261A36802E01A4943F8041C4E
:1011D00082689C4608339445F7D394F83800A2609F
:1011E00010F0010060D0A069011DA16120464FF000
:1011F000FF320021FFF746FEA269131FA361002002
:1012000052E0E269A368D51AA02D03DC2046142120
:10121000FFF7B6FD6569616A8D4211D12046FFF77F
:1012200095FD05460EE000BF0300FFFF36B503083D
:101230000800FFFF0000FFFF0700FFFF38D303088F
:1012400018356561206A009BC11869600831296002
:10125000A268019BE160A032AA602B6194F838007B
:10126000C10705D5204600214FF0FF32FFF70AFEE7
:101270006B680E495A688A4208D1616948684368B8
:1012800093420CBF00680020036900E01B68204601
:101290009847002807DBA268C300D11A2046FFF751
:1012A00033FE012000E00220BDE8FE8F0800FFFFB2
:1012B00070B582794369044632B908394FF0FF327C
:1012C000FFF77CFEB8B170BD0022827158680F4EE6
:1012D0004568B54205D00536B54208BF0268907929
:1012E00038B12046FFF710FE28B161698B68A36012
:1012F00001E01A68E260A16A6269501A0449C310E9
:1013000059432046BDE8704005F02EBF0300FFFFA3
:10131000ABAAAAAA70B50D46818E4B1C9BB2C72BF7
:101320000446164683860AD9C82B03D11049FFF715
:1013300035FB04E0E02B02D90521FFF7D1FC204664
:1013400029463246FFF73AFE18B92046012105F03A
:101350000BFFA28E2369511EA1865A6C186C824223
:1013600004D32046BDE8704001F082B970BD00BFD3
:101370005DAE030838B58279012A044607D01AB950
:101380004269836A9A4202D02046134904E0A28E41
:10139000C72A05D911492046BDE83840FFF750BD9E
:1013A000A568501CCA00A086E086AA1A20460C49EF
:1013B000FFF7ECFB054648B1A07129462046A2681C
:1013C000FFF7B6FB6369A168996000E0A579A08E7C
:1013D000421EA286284638BD6EAE03085DAE0308E5
:1013E000B112010838B5828EC38E9A4204460D466A
:1013F00002D90649FFF7D2FAA168ED0001204D1B82
:10140000A071E5604FF0FF3038BD00BF94AE030817
:101410002DE9F84F99460A9BD0F864B0436604461C
:10142000B0F834804769866A90F839A0FFF7AEFBC0
:101430000546C8B1206A81444946204600F029FB90
:10144000204629464A46FFF773FBA36AA4F8348076
:10145000BE1B991961619A59E260C86884F839A085
:10146000A0612046FFF72AFCC4F864B02846BDE816
:10147000F88F000070B588B086680792036A426EE4
:10148000039100240092F31A03AA08490494054624
:1014900005940694FFF7BCFF0499069A0646234676
:1014A000284601F015FF304608B070BD910D0108C7
:1014B00070B51446126903460D464AB919462A46C4
:1014C000A36894E84100B047E36A20615D19E562D2
:1014D00070BD07B502AB0A4603F8010D012118469D
:1014E000FFF7E6FF0EBD10B5044603E000202146DD
:1014F000FFF7EFFFE36A9B07F8D110BD012AF7B5AC
:101500000CD000224D08134605E04418C65CA75CC9
:10151000C754A6540133013AAB42F6D1FEBD0229AD
:1015200037B514460DD004291DD001292FD100F163
:101530008003FF2B01D9652111612146FFF7C9FF07
:1015400025E000F50045B5F5803F01D36523136123
:1015500002AD022125F8040D62692846FFF7CEFF8F
:101560002846022110E000F10045691ECB1C01D97C
:101570006523136102AD042145F8040D6269284614
:10158000FFF7BCFF284604212246FFF791FF3EBD2E
:101590000A468969FFF7C3BF37B5CB69022B0C46F2
:1015A0000BD0042B19D0012B28D1FF2801D965239A
:1015B0000B612146FFF78DFF20E0B0F5803F01D39E
:1015C00065220A6102AD022125F8040D62692846F0
:1015D000FFF794FF284602210DE0421C01D165254A
:1015E0000D6102AD042145F8040D62692846FFF73C
:1015F00085FF284604212246FFF75AFF3EBD70B5FD
:101600000D46044640B190F90530002B02DA00691E
:1016100040B901E0103005D100202946BDE87040F6
:10162000FFF7BABFE668013630462946FFF7B4FF38
:1016300094F905100029B4BF206904F11000314667
:101640002A46BDE87040FFF733BF2DE9F04F036A2B
:101650008B4287B00546144605D0D06800280CBFE1
:101660001846002000E000202146FFF7C8FFE86B85
:101670002146FFF78DFF286C2146FFF789FF95F87B
:1016800048002146FFF725FF95F849002146FFF75E
:1016900020FF95F84A002146FFF71BFF95F84B0005
:1016A0002146FFF716FFE86A2146FFF771FF204643
:1016B000FFF719FF00260EE0EB68626953F8261069
:1016C00001A801910421FFF719FF01A80421224676
:1016D000FFF7EEFE0136EA6A9642EDDBD5F8288088
:1016E00021464046FFF754FF00266CE0D5F808A0DD
:1016F0004FEAC6090AEB0907B7F906104B1C08BFE9
:10170000B7F90400214618BF0520FFF7E2FEB7F93C
:101710000600431C0DD1B7F90430052B09D0062B68
:101720004BD0012B4ED15AF809002146FFF7D1FECC
:1017300048E0D7E900AB676AAFB1594650461FF0A1
:1017400097FD07461FF0E6FE1FF0A4FA52465B46DF
:101750001FF05CFD08B9662323613846216A2246E2
:10176000FFF7DDFE2EE0276A042F02D0082F29D1D3
:101770000FE0594650461FF0C3FD0DF118093946D8
:1017800049F8080D62694846FFF7B8FE48463946F1
:101790000FE0A26ACDE904AB22B10498059901904B
:1017A0000491059004A808216269FFF7A7FE04A828
:1017B00008212246FFF77CFE04E05AF80900214682
:1017C000FFF71DFF0136464590DB6F6B214638461B
:1017D000FFF7DEFE002607E02B69296A53F8260092
:1017E0002246FFF732FF0136BE42F5DBE6680EB94E
:1017F0002F6B00E0002738462146FFF7C9FE204640
:10180000FFF771FE002606E06A69214652F82600BD
:10181000FFF7BEFE0136BE42F6DBE76817B9D5F822
:10182000388001E04FF00008404621460026FFF7CF
:10183000AFFE374612E0A86921468059FFF7DFFE68
:10184000AA69931921465868FFF7A2FEA969881969
:1018500021468068FFF79CFE01370C364745EADBDE
:10186000E6680EB96F6A00E0002738462146FFF7A8
:101870008FFE002606E0E96951F826002146FFF7B1
:10188000BEFE0136BE42F6DB07B0BDE8F08F0000B9
:10189000F0B591B016AE0D4656F8044B0190029289
:1018A00003930FCE06AF0FC796E80300154A079BB8
:1018B0000D9287E803000698089A8DF83A005121A6
:1018C00009988DF838108DF83B3004210A9B049458
:1018D0008DF83C2000248DF83D108DF83E000C2141
:1018E0000DA801AA05940C948DF839408DF83F306D
:1018F000FFF7DEFD2846214601AAFFF7A6FE059860
:1019000011B0F0BD1B4C7561F0B591B00124099484
:101910000F941E466C46169B84468E460020174642
:10192000082104220D900E900A920B920C9144F81B
:10193000043B09AD0FCD0FC495E803003A4684E897
:101940000300334660467146FFF7A2FF11B0F0BDB9
:10195000426901691161036942695A617047F8B5CA
:10196000CF1C0C460021FB0015460A46064601F036
:10197000AFFC074639463046082200F02CFF012311
:10198000BB71FD60FC713846F8BDF8B50C464B1DC7
:1019900000219B0015460A46064601F099FC0746C1
:1019A00008223046394600F016FF0023BB71FD6067
:1019B000FC71224606E007EB840C0CEB03010020CF
:1019C000013A4861043B002AF5D13846F8BD0000D1
:1019D000002138B50A461823044601F079FC054673
:1019E000294620460C2200F0F6FE034B05F11000BC
:1019F000A8606B61284638BD0000FFFF2DE9F0416B
:101A000004460F46056900F158060CE00AD14379F7
:101A1000297D23EA0102920726D083F00303437154
:101A2000BDE8F0811E4633681BB19A68BA42184679
:101A3000ECD200210A461823204601F049FC0C2173
:101A400001718760326805F17803026030600361DC
:101A5000D5F88C10804641610861C5F88C0041467C
:101A6000204600F0ACFE4046BDE8F08170B58A68C3
:101A700001F110039A4204460D4602D00846FFF7D2
:101A800067FF2046294618220023BDE8704001F078
:101A90001FBCF8B504460E4605691AE03968A16511
:101AA0002A7D787920EA0203990704D02046394636
:101AB000FFF7DCFF0DE03846FFF74AFFBB68D3E9CC
:101AC00000233846E0E904233946B860204600F098
:101AD0008CFEA76D17B1BA68B242DFD2F8BD002103
:101AE00038B50A464C23044601F0F2FB0546294668
:101AF00020460B2200F06FFE0023AB60AB622B612F
:101B00006B63EB60EB622B636B6285F84830EB61D3
:101B100085F8493085F84A3085F84B306B61AB6306
:101B2000AB61EB632B642B62284638BD70B54B6B01
:101B30000C469A0009690023054601F0C9FBA26A18
:101B4000A168D2000023284601F0C2FBA36BA16963
:101B50000C225A432846002301F0BAFB626AE1696D
:101B600000239200284601F0B3FB94F90530002BC6
:101B70000DDBE36AE1689A002846002301F0A8FB28
:101B8000226B616928469200002301F0A1FB2846E0
:101B900021464C220023BDE8704001F099BB8B79AF
:101BA000CA7913B10332D20001E0531D9A00002319
:101BB00001F08EBBF0B50023866B1D460EE0A768D2
:101BC000BA4209DA013907D1206890F90530002BB3
:101BD000B4BF00691030F0BD01350C33B54206DAF0
:101BE0008469E41867689742E9DD0020F0BD0020B1
:101BF000F0BD0000B0F90E30013305D1B0F90C1082
